S01300006170706C69636174696F6E2E737265637D
S31508004000E04A0020FDCE010875D401088DAF0108ED
S3150800401091AF010895AF010899AF010800000000AB
S3150800402000000000000000000000000029B301089D
S3150800403079D401080000000095B30108A5B301086A
S315080040407DD4010881D4010885D4010889D40108E2
S315080040508DD4010891D4010895D4010899D4010892
S315080040609DD40108A1D40108A5D40108A9D4010842
S31508004070ADD40108B1D40108B5D40108B9D40108F2
S31508004080BDD40108C1D40108C5D401083B9F000866
S31508004090359F0008C9D40108419F0008CDD40108FE
S315080040A0D1D40108D5D40108D9D40108DDD4010832
S315080040B0E1D4010895650008E5D40108E9D40108AA
S315080040C0EDD40108F1D40108F5D40108F9D40108A2
S315080040D0FDD4010801D5010805D5010809D501084F
S315080040E00DD5010811D5010815D5010800000000F5
S315080040F02DE9FE4304460E4660694088002836D0FE
S31508004100B4217143621802F12C0529780818A169AF
S31508004110498881422BDB616851F83000806B07784B
S3150800412002F1D8084FF0FF30A8F800008520A870E3
S31508004130DFF8A892CDF80490A87A00902B892A78FF
S315080041406978204600F013FAC5F80490D8F80420D8
S31508004150002A02D03946204690476868484506D165
S315080041603146C9B2204603B0BDE8F043CEE0BDE80B
S31508004170F78310B50446002004E00021204600F02D
S31508004180C5F801200028F8D010BD1FB5B422514348
S31508004190421802F134046168002901D1A1686160FE
S315080041A06168039101210291019103A9009102F12D
S315080041B04003A278218801F0F9FE002800D10020EA
S315080041C004B010BD10B586B080220592B4225143C2
S315080041D0014401F1340401220392029204AA0192D5
S315080041E005AA009201F14003A278218801F076FE23
S315080041F0002803D1059860600020A06006B010BDB5
S3150800420030B4B42461430844C16B5418812C02D2DB
S31508004210856BA54201D2FF200EE0002406E0651852
S31508004220054495F840501D55641CE4B29442F6D3F3
S31508004230C16B5218C263002030BC704770B4B424F6
S3150800424061430844C16B5418812C01D3FF200EE04A
S31508004250002406E01D5D6618064486F84050641C76
S31508004260E4B29442F6D3C16B5218C263002070BC04
S3150800427070472DE9FF4705460E461746984602AB96
S3150800428000F0C4F8040007D13846012804D19DF887
S315080042900810284600F03AF8DDF83490002C22D1B0
S315080042A0384602281FD105F1D8044FF0B40A9DF804
S315080042B008000AFB00F0205E01F093FF9DF8081045
S315080042C00AFB01F160529DF808000AFB00F0284439
S315080042D0852180F82E109DF808000AFB00FA05EBE8
S315080042E00A00C0F83090CDF804909DF83000009090
S315080042F0434632463946284600F039F9002801D0A7
S31508004300FF2000E0002004B0BDE8F0873EB5044673
S315080043100D4600200190009003460246204600F014
S3150800432012F8002004E00022014481F84020401CD5
S315080043302946B422514321448028F4D3002081F829
S315080043402D00086337BD2DE9F84305460E46174686
S315080043509846099C2046022805D0032803D004283D
S3150800436001D005280FD1B4204143681800F1C009CF
S31508004370002000901A4B1B4A3146284601F0E2FEFF
S31508004380A9F818000AE0B4204143681800F1C009EA
S31508004390B9F9180001F025FFA9F818000898B42102
S315080043A04E43A91901F12C021770A2F808809072E1
S315080043B094700020D070D060106101F1C000002117
S315080043C0017041708170416081600173417381732E
S315080043D0C175C1610846BDE8F28300000000040506
S315080043E040420F00F140000810B4002300F12D04EC
S315080043F000E00123002B07D16378002BF9D10020B8
S315080044001070217010BC7047FF20FBE770B40C4693
S315080044100021264600E00121002913D100F12C05D0
S31508004420A9780029F7D08529F5D02978B142F2D1A3
S3150800443069781546A942EED1002B01D000201870E4
S31508004440002000E0FF2070BC704770B40C460021C5
S31508004450264600E00121002911D100F12C05A97892
S315080044600029F7D02978B142F4D169781546A942CE
S31508004470F0D1002B01D000201870002000E0FF20AA
S3150800448070BC704738B50446154601F0C7FB0146AF
S31508004490FE2901DB852032BD6B462A462046FFF7FA
S315080044A0D4FF002801D0FF2032BD9DF80010204619
S315080044B0FFF72CFF002032BDB42359430144886B13
S315080044C0002802D10020106002E0C96B401A106073
S315080044D000207047812A01D3FF207047B42359432F
S315080044E008448263002070471FB590F8E040052C09
S315080044F001D07F2C1AD1446901290FD121880029BE
S3150800450014D052188169098891420FDB416851F825
S315080045103210896A0968ADF8021010E0618800292E
S3150800452004D0521881694988914201DAFF201CE0BB
S31508004530416851F8321089690968ADF802100021FE
S315080045408DF8041008218DF80510002104E05A5C46
S315080045506C460C44A271491C0829F8DBD0F84802BD
S315080045608DF80000684601F0C7FE04B010BD7CB5A2
S31508004570069C079D80268DF800601E468DF8016012
S315080045801B0A8DF802308DF803402B468DF804304F
S315080045901B0A8DF805302B461B0C8DF806302D0EA0
S315080045A08DF807506B46FFF79FFF76BD2DE9F84F4C
S315080045B086B004468B4600208DF808008DF8040066
S315080045C04FF0030860690088A1690988002200285D
S315080045D003D116E0521C401C80B2814211DB63688D
S315080045E01E1D16F83060012E41F3088353F830304B
S315080045F09B691B68BBF80260B342EBD14FF0010818
S3150800460015464046032823D160694188A069428837
S31508004610002300291CD0002002E05B1C491C89B23B
S315080046208A4213DB6668371D17F83170042FC1F20A
S31508004630E58256F83160B76A3F68BBF802C067453D
S31508004640EBD14FF002081D46B06B00788DF80400D8
S315080046504046032801F0D2829BF8050008280DD0B1
S315080046604FF000600190002000900346424629461C
S31508004670C9B22046FFF7FDFDFF20C7E002AB424660
S315080046802946C9B22046FFF7C1FEFF21B4260028F5
S315080046901CD14246012A07D19DF8082072432244BC
S315080046A092F82E20042A0AD04246022A0ED19DF8F4
S315080046B008207243224492F82E20052A06D19BF838
S315080046C00610802901D1042100E006210A46FF2AA6
S315080046D002D19BF806104909062901F27282DFE821
S315080046E011F007002901580260039F04E3048A07B2
S315080046F04146012940F08D80002808D19DF8081010
S315080047007143214491F82E10022900D00120002877
S3150800471041F0CC819DF8080070432044CE30B0F9B2
S315080047200A0010F1010F16D001F05BFD04F1D8075D
S315080047309DF808107143785200200090DFF8083D74
S31508004740DFF8082D9DF80810204601F0FBFC9DF8BF
S315080047500810714378529DF80810714304F134002B
S315080047600844078890F802A09BF8060004F12F0277
S31508004770515CC0F30012914240F05883C0F34200E6
S31508004780C0F1070003900BF10703039A9DF8081080
S315080047902046FFF753FD002840F0E48604F12F0079
S315080047A09DF808107143405C000140F020008DF828
S315080047B010000120002104AA01E01154401C07281A
S315080047C0FBD904AB2A46D2B201212046FFF78CFE5C
S315080047D09DF80800464304F12F00805D401E804185
S315080047E0C00F04F12F0188559BF80600C0070CD5A9
S315080047F09DF808102046FFF7C8FC002840F09C8466
S315080048009DF808102046FFF781FD002007B0BDE897
S31508004810F08F002808D19DF808107143214491F8BB
S315080048202E10032900D00120002841F03F819DF871
S31508004830080070432044CE30B0F90A0010F1010F89
S3150800484016D001F0CEFC04F1D8079DF80810714384
S31508004850785200200090DFF8F03BDFF8F02B9DF847
S315080048600810204601F06EFC9DF808107143785236
S315080048709DF80810714304F134000844078890F83D
S3150800488002A09BF8060004F12F02515CC0F3001247
S31508004890914240F0CB82C0F34200C0F1070003907A
S315080048A00BF10703039A9DF808102046FFF7C6FC8C
S315080048B0002840F057869DF80800704304F12F0140
S315080048C0095C491E8941C90F04F12F0211549DF84C
S315080048D0080070439BF80610C9071AD504F1D805D5
S315080048E0285E01F07EFC9DF808107143685204F1B9
S315080048F02E009DF8081071430122425404F1DC0091
S315080049009DF808107143405800283FF47EAF01F027
S315080049104CB904F12F01085C000140F060008DF8E5
S3150800492010000120002104AA072801F2448011542E
S31508004930401CF9E74146012975D19BF808109BF8F8
S31508004940077047EA01279BF809A0002800F06D8642
S3150800495002AA01212046FFF747FD002840F0658698
S3150800496002200190504600903B462A46D2B29DF856
S3150800497008102046FFF7E7FC9BF806100A46C2F324
S315080049804000002824D0C2F38100C0F1040003903F
S3150800499004F138009DF808104E43039981510BF134
S315080049A00A03039A9DF808102046FFF747FC0028DB
S315080049B040F0D8859DF808102046FFF7E6FB00284A
S315080049C040F0BA839DF808102046FFF79FFC19E0CF
S315080049D0C80717D59BF80A009BF80B1000EB0120B7
S315080049E09BF80C1000EB01409BF80D1000EB0160E2
S315080049F00390039A9DF808102046FFF76BFD0028E0
S31508004A0040F0B08560208DF8100004A94F703F0A69
S31508004A108F7081F803A004200022072800F2CB87B4
S31508004A200A54401CF9E7002808D19DF8081071437C
S31508004A30214491F82E10022900D00120002841F0C7
S31508004A4035809DF8080070432044CE30B0F90A003E
S31508004A5010F1010F16D001F0C4FB04F1D8079DF838
S31508004A6008107143785200200090DFF8DC39DFF82F
S31508004A70DC299DF80810204601F064FB9DF8081013
S31508004A80714378529DF80800704304F134010144DB
S31508004A900F8891F802A004F12F01085C9BF8061014
S31508004AA0C1F30011884240F0C18103AA9DF808109D
S31508004AB02046FFF701FD9DF808107143039800286A
S31508004AC01AD104F1D805685E01F08BFB9DF8081031
S31508004AD07143685204F12E009DF8081071430122B3
S31508004AE0425404F1DC009DF8081071434058002830
S31508004AF03FF48BAE01F059B804F12F00405C039ADD
S31508004B00072A1BD9401E8041C00F04F12F025054BA
S31508004B1004F12F009DF808104E43805D00018DF8C2
S31508004B2010000DF1110307229DF808102046FFF723
S31508004B3067FB002840F0168500F03DBF401E804107
S31508004B40C00F04F12F02505404F12F009DF80810ED
S31508004B504E43805D0399C1F10701490041EA0011FE
S31508004B6041F001018DF810100DF11103039A9DF81B
S31508004B7008102046FFF744FB002840F0F38403980A
S31508004B80401C002104AA072800F215871154401C6E
S31508004B90F9E7414601296AD19BF808109BF8077086
S31508004BA047EA01279BF809A0002800F03E8502AADB
S31508004BB001212046FFF718FC002840F0368503201F
S31508004BC00190504600903B462A46D2B29DF80810FE
S31508004BD02046FFF7B8FB9DF808102046FFF7F2FAC3
S31508004BE0002840F0A98203AA9DF808102046FFF77E
S31508004BF063FC3846000A04AE0399042919D94121F1
S31508004C008DF810107770B07086F803A0039830718D
S31508004C100398000A70710398000CB0710398000E8F
S31508004C20F07104AB2A46D2B201212046FFF75CFC9C
S31508004C30EBE5C1F10401890041F043018DF810103C
S31508004C407770B07086F803A005AB039A9DF8081034
S31508004C502046FFF7D5FA002840F084840398001D03
S31508004C600021072800F23D813154401CF9E700284D
S31508004C7008D19DF808107143214491F82E10032994
S31508004C8000D00120002840F011879DF808007043E5
S31508004C902044CE30B0F90A0010F1010F16D001F009
S31508004CA0A0FA04F1D8079DF808107143785200203D
S31508004CB00090DFF89437DFF894279DF8081020460F
S31508004CC001F040FA9DF808107143785204F1340057
S31508004CD09DF8081071430844078890F802A09BF8CD
S31508004CE006100A46C2F34000002834D0C2F38100F9
S31508004CF0C0F1040003900BF10A03039A9DF808100B
S31508004D002046FFF79BFA002840F02C8404F1D805CA
S31508004D109DF808007043285E01F063FA9DF80810B4
S31508004D207143685204F138009DF808107143039ADC
S31508004D30425004F12E009DF8081071430122425496
S31508004D4004F1DC009DF808107143405800283FF430
S31508004D505CAD00F02ABFC80717D59BF80A009BF878
S31508004D600B1000EB01209BF80C1000EB01409BF8A0
S31508004D700D1000EB01600390039A9DF80810204679
S31508004D80FFF7A8FB002840F0ED8360208DF810009F
S31508004D900120002104AA072800F20D861154401CA0
S31508004DA0F9E74146012940F0A980002808D19DF875
S31508004DB008107143214491F82E10032900D00120D0
S31508004DC0002840F073869DF8080070432044CE30D2
S31508004DD0B0F90A0010F1010F16D001F002FA04F139
S31508004DE0D8079DF808107143785200200090DFF824
S31508004DF05836DFF858269DF80810204601F0A2F923
S31508004E009DF80810714378529DF80800704304F124
S31508004E10340101440F8891F802A004F12F01085CBF
S31508004E209BF80610C1F3001188420DD0DFF8D40DA7
S31508004E300190CDF800A03B4642462946C9B2204615
S31508004E40FFF717FAFF20E1E403AA9DF808102046A9
S31508004E50FFF732FB04F12F009DF808107143405C00
S31508004E6000010399072920D98DF810000DF11103C7
S31508004E7007229DF808102046FFF7C2F9002840F0DF
S31508004E8071839DF80800464304F12F00805D401E9B
S31508004E908041C00F04F12F01885504AB2A46D2B2CF
S31508004EA001212046FFF720FBAFE4C1F1070140EAE4
S31508004EB0410040F001008DF810000DF11103039A2E
S31508004EC09DF808102046FFF79BF9002840F04A8312
S31508004ED00398401C002104AA01E01154401C07282D
S31508004EE0FBD904AB2A46D2B241462046FFF7FCFA64
S31508004EF09DF808102046FFF709FA86E4002808D12D
S31508004F009DF808107143214491F82E10022900D00B
S31508004F100120002840F0CA859DF808007043204407
S31508004F20CE30B0F90A0010F1010F16D001F059F988
S31508004F3004F1D8079DF808107143785200200090B4
S31508004F40DFF80435DFF804259DF80810204601F03F
S31508004F50F9F89DF808107143785204F134009DF869
S31508004F60081071430844078890F802A003AA9DF820
S31508004F7008102046FFF7A0FA9DF808107143039819
S31508004F8000281AD104F1D805685E01F02AF99DF8BF
S31508004F9008107143685204F12E009DF808107143F9
S31508004FA00122425404F1DC009DF808107143405870
S31508004FB000283FF42AAC00F0F8BD04F12F00405C4D
S31508004FC00001039907290ED98DF810000DF1110378
S31508004FD007229DF808102046FFF712F9002840F02E
S31508004FE0C18200F0E8BCC1F1070140EA410040F087
S31508004FF001008DF810000DF11103039A9DF80810B1
S315080050002046FFF7FDF8002840F0AC820398401CC4
S31508005010002104AA072800F2CE841154401CF9E79F
S315080050209BF80A509BF80B1045EA01259BF80C10D3
S3150800503045EA01459BF80D1045EA0165B8F1010FEF
S3150800504009D100287FF4E1AB9DF808102046FFF748
S315080050505DF9FFF7DABB00287FF4D7AB9DF80800A7
S3150800506070432044CE30B0F90A0001F0BAF804F1D2
S31508005070D8019DF808207243885204F12E009DF845
S3150800508008107143802242549DF80800704320445A
S31508005090056304F1DC009DF80810714340580028A8
S315080050A03FF4B3AB00F081BD9BF8069009F0030905
S315080050B04146012940F05F81B9F1000F73D19BF891
S315080050C008109BF8077047EA01279BF809A00028F3
S315080050D000F0AB829BF80A00802880F2A68102AA1B
S315080050E001212046FFF780F9002840F09E8205201E
S315080050F00190504600903B462A46D2B29DF80810C9
S315080051002046FFF720F904F1C0009DF80810714306
S315080051109BF80620C2F38002425404F1C1009DF8B0
S31508005120081071439BF80A2042549DF8081020463F
S31508005130FFF748F800280CD00190CDF800A03B46B0
S3150800514042462946C9B22046FFF793F8FF20FFF7E3
S315080051505DBB03AA9DF808102046FFF7ADF904F1D8
S31508005160C4009DF808104E4303998151C2208DF85A
S31508005170100004A847703F0A877080F803A00399B7
S3150800518001710399090A41710399090C81710399FF
S31508005190090EC17104AB2A46D2B201212046FFF797
S315080051A0A3F9FFF732BBB9F1010F14D1002808D1D2
S315080051B09DF808104E43A11991F82E10052900D024
S315080051C00120002840F072849DF808102046FFF759
S315080051D09DF8FFF71ABBB9F1020F03D0B9F1030F17
S315080051E07FF413AB002808D19DF8081071432144B9
S315080051F091F82E10052900D00120002840F0568489
S315080052009DF8080070432044CE30B0F90A0010F12A
S31508005210010F14D000F0E5FF04F1D8079DF8081037
S315080052207143785200200090874B884A9DF80810F1
S31508005230204600F087FF9DF80810714378529DF8C4
S315080052400800704304F1340101440F8891F802A064
S31508005250B9F1020F3DD19BF8081004F1C1021154AF
S315080052609BF8079009F07F0903AA9DF808102046C5
S31508005270FFF722F99DF80810714304F1C800421897
S315080052800398002811D1107981450ED150798000F4
S3150800529040F0C1008DF810000120002104AA07285B
S315080052A000F289831154401CF9E71068C9EBC90953
S315080052B0814404F13C0040F801909DF808007043D1
S315080052C004F13801095804F13C0210588142C0F033
S315080052D0ED839DF80800704304F13C01095804F178
S315080052E0C80211504FF0010915E08DF810900DF124
S315080052F0110307229DF808102046FEF781FF0028B3
S3150800530040F0308104AB2A46D2B201212046FFF78D
S31508005310EBF809F1010904F1C1009DF80810714381
S31508005320084401784A46D2B29142FFF46EAA80F840
S315080053300B9003AA9DF808102046FFF7BDF80398BE
S315080053400728D2D849F080098DF810900DF111037D
S31508005350039A9DF808102046FEF752FF002840F0F1
S3150800536001810398401C002104AA072800F20D8138
S315080053701154401CF9E7B9F1000F03D0B9F1020F37
S3150800538040F01581002808D19DF808107143214482
S3150800539091F82E10042900D00120002840F08683B9
S315080053A09DF808007043204400F12E01CF8891F83B
S315080053B008A0CE30B0F90A0010F1010F16D000F09F
S315080053C010FF04F1D8019DF8082072438852002086
S315080053D000901D4B1D4A9DF80810204600F0B2FEAD
S315080053E004F1D8019DF8082072438852B9F1000FDC
S315080053F016D19BF80A00802817DA04F1C0009DF838
S31508005400081071439BF80620C2F38002425404F147
S31508005410C1009DF8081071439BF80A20425456E0D3
S315080054209BF808000146802912DBDFF8DC070190AB
S31508005430CDF800A03B4642462946C9B22046FEF7AB
S3150800544018FFFF20FFF7E2B940420F00F1400008BD
S315080054509DF8081071432144C03148709BF80790A5
S3150800546009F07F0903AA9DF808102046FFF724F8DB
S315080054709DF80810714304F1C800421803980028E3
S3150800548011D1107981450ED15079800040F0C100C4
S315080054908DF810000120002104AA072800F28B824B
S315080054A01154401CF9E71068C9EBC909814404F195
S315080054B03C0040F801909DF80800704304F138015B
S315080054C0095804F13C0210588142C0F0AE809DF89C
S315080054D00800704304F13C01095804F1C802115050
S315080054E04FF0010914E08DF810900DF11103072211
S315080054F09DF808102046FEF783FE002832D104AB3B
S315080055002A46D2B241462046FEF7EEFF09F10109C6
S3150800551004F1C1009DF808107143084401784A4611
S31508005520D2B29142FFF471A980F80B9003AA9DF8B4
S3150800553008102046FEF7C0FF03980728D3D849F07D
S3150800554080098DF810900DF11103039A9DF8081043
S315080055502046FEF755FE002804D10398401C00217A
S3150800556004AA10E04FF000600190CDF800A03B4679
S3150800557042462946C9B22046FEF77BFEFF20FFF7C2
S3150800558045B91154401C0728FBD904AB2A46D2B2A8
S3150800559041462046FEF7A8FF04F1CD009DF8081005
S315080055A04E430399C1F107018155FFF72EB9B9F1A9
S315080055B0010F40F07B829DF8080070432044CE30EE
S315080055C0B0F90A0000F00DFE04F1D8019DF8082094
S315080055D07243885204F12E009DF808107143012287
S315080055E0425404F1DC009DF8081071434058002825
S315080055F03FF40BA9D9E24146012940F07D810028F4
S315080056006ED09BF80600C00700F150829BF8080090
S315080056109BF8077047EA00279BF809A002AA012110
S315080056202046FEF7E1FE00280ED0DFF8E0050190DF
S31508005630CDF800A03B4642462946C9B22046FEF7A9
S3150800564018FEFF20FFF7E2B80420019050460090AC
S315080056503B462A46D2B29DF808102046FEF773FE4E
S3150800566004F1CE009DF8081071430122425404F15A
S31508005670C0009DF8081071439BF80620C2F380020B
S3150800568042549BF80600800713D504F1C4009DF820
S3150800569008104E439BF80A109BF80B2001EB0221D9
S315080056A09BF80C2001EB02419BF80D2001EB0261EF
S315080056B08151A0208DF8100004A847703F0A877012
S315080056C080F803A0102101710021C180417104AB4B
S315080056D02A46D2B201212046FEF706FFFFF795B803
S315080056E09DF8080070432044CE300178012940F027
S315080056F08A80B0F90A0010F1010F16D000F071FD8A
S3150800570004F1D8079DF808107143785200200090DC
S31508005710DFF8FC34DFF8FC249DF80810204600F07A
S3150800572011FD9DF80810714378529BF8063003F076
S315080057307F0904F1CC079DF80800704338440178C6
S315080057404A46521E1B062FD58A4211D10221817064
S315080057509DF80800704307F8009008220BF106012F
S3150800576004F1CF009DF808307343184400F032FE68
S31508005770A2208DF8100004A89DF808107143795CE2
S3150800578041701021817000214160C17004AB2A4626
S31508005790D2B201212046FEF7A7FE00209DF8081088
S315080057A04E43B855FFF731B88A420CD180F80090BD
S315080057B00BF1070307229DF808102046FEF73EFD69
S315080057C0002840F08E81B9F1100F7FF41EA8A220A0
S315080057D08DF8100004A89DF808107143795C417093
S315080057E01021817000214160C17004AB2A46D2B2F3
S315080057F001212046FEF778FE00209DF808104E434A
S31508005800B855FFF702B802297EF4FFAF9BF80610D9
S31508005810C90740F14B81B0F90A0010F1010F16D003
S3150800582000F0DFFC04F1D8079DF8081071437852A0
S3150800583000200090DFF8D833DFF8D8239DF8081049
S31508005840204600F07FFC9DF808107143785204F159
S31508005850D0009DF80810714343189BF80600C0F362
S315080058608202C2F107029DF808102046FEF7E6FC00
S31508005870002840F036819DF80810714304F1C400F1
S315080058804058002805D004F13C025158884240F09F
S315080058904A81A1208DF810000120002104AA01E008
S315080058A01154401C0728FBD904AB2A46D2B2012161
S315080058B02046FEF719FE9DF808102046FEF765FCFF
S315080058C0002812D004F134019DF8082056433144CB
S315080058D00190887800900B8801222946C9B2204693
S315080058E0FEF7C7FCFF20FEF791BF9DF8081020467B
S315080058F0FEF70CFDFEF789BF002840F0D7809DF81B
S31508005900080070432044CE30B0F90A0010F1010FA8
S3150800591014D000F066FC04F1D8079DF8081071430E
S31508005920785200200090BA4BBA4A9DF808102046D3
S3150800593000F008FC9DF80810714378529DF808009D
S315080059407043221802F1CC01887800283CD19BF8D4
S315080059500600C0073EF559AF0120887004F1C00063
S315080059609DF8081071439BF80620C2F38002425442
S315080059709BF80600800713D504F1C4009DF80810AB
S315080059804E439BF80A109BF80B2001EB02219BF86B
S315080059900C2001EB02419BF80D2001EB02618151BD
S315080059A0A3208DF810000120002104AA01E011545B
S315080059B0401C0728FBD904AB2A46D2B241462046EA
S315080059C0FEF792FDFEF721BF012868D19BF8060075
S315080059D000F07F0904F1CC070A784B465B1E0006E7
S315080059E02FD5934211D1022088709DF80800704384
S315080059F007F8009008220BF1060104F1CF009DF884
S31508005A0008307343184400F0E5FCA2208DF8100016
S31508005A1004A89DF808107143795C417010218170C3
S31508005A2000214160C17004AB2A46D2B241462046E5
S31508005A30FEF75AFD00209DF808104E43B855FEF7AC
S31508005A40E4BE93420BD181F800900BF107030722BD
S31508005A509DF808102046FEF7F1FB002841D1B9F160
S31508005A60100F7EF4D2AEA2208DF8100004A89DF87F
S31508005A7008107143795C41701021817000214160E2
S31508005A80C17004AB2A46D2B241462046FEF72CFD29
S31508005A9000209DF808104E43B855FEF7B6BE0228FA
S31508005AA07EF4B3AE9BF80600C1070DD457480190A3
S31508005AB000200090034642462946C9B22046FEF712
S31508005AC0D8FBFF20FEF7A2BE02F1D003C0F3820284
S31508005AD0C2F107029DF808102046FEF7AFFB002822
S31508005AE014D004F134009DF808104E4330444FF0AA
S31508005AF00061019181780091038842462946C9B21E
S31508005B002046FEF7B6FBFF20FEF780BE9DF808107C
S31508005B10714304F1C4004058002818D004F13C022F
S31508005B205158884213D004F134009DF808104E43AA
S31508005B3030443649019181780091038842462946C6
S31508005B40C9B22046FEF795FBFF20FEF75FBEA120EF
S31508005B508DF810000120002104AA01E01154401C10
S31508005B600728FBD904AB2A46D2B241462046FEF79F
S31508005B70BBFC04F1D8059DF808007043285E00F0C8
S31508005B8030FB9DF808107143685204F12E009DF809
S31508005B90081071430122425404F1DC009DF80810F4
S31508005BA07143405800283EF430AE9DF80410204654
S31508005BB004F1DC029DF808305E4392599047FEF7DF
S31508005BC024BE154900280FD19DF808004643A019A0
S31508005BD02E300191017A0091C38842462946C9B2FE
S31508005BE02046FEF746FB09E0019100200090034697
S31508005BF042462946C9B22046FEF73BFBFF20FEF780
S31508005C0005BE000000000305020004052100000887
S31508005C1040420F00F140000801000405F0B40024DA
S31508005C204269538882695588002B13D0224609E0B9
S31508005C3056F83360B66B36780F46BE420CD05B1CFE
S31508005C409BB2521C9D4208DB4668371D17F8337015
S31508005C50042FEDDAFF2006E00124002C01D1FE20F6
S31508005C6001E01046C0B2F0BC70472DE9F04F85B090
S31508005C70054617461C46FFF7D1FF0646FE2880F262
S31508005C80828002AB022231462846FEF7BFFB002877
S31508005C9001D1FF2077E002AA02212846FEF7A4FBDD
S31508005CA0002801D0FF206EE01098B8464FEA182861
S31508005CB005F1D7090DF10C0ADDF838B0002826D011
S31508005CC005200190204600903B4632469DF8081074
S31508005CD02846FEF738FB9DF80810B420414309F81A
S31508005CE001B0A0208DF80C008AF801708AF80280AD
S31508005CF08AF8034010208AF804000520002201468D
S31508005D00C9B2082927DA0AF80120401CF7E7032058
S31508005D100190204600903B4632469DF808102846DA
S31508005D20FEF711FB9DF80810B420414309F801B0AD
S31508005D3040208DF80C008AF801708AF802808AF8EB
S31508005D4003400420002202E00AF80120401C014614
S31508005D50C9B20829F8DB0F999DF80820B4204243F8
S31508005D60A818C0F8DC1003AB324602212846FEF715
S31508005D70BBFB002806D09DF808102846FEF7C6FA91
S31508005D80FF2000E0002005B0BDE8F08F1FB59DF8A4
S31508005D9020400294079C01949DF818400094FFF750
S31508005DA064FF04B010BDF8B5044615461E46069FA6
S31508005DB0002038602046FFF731FF0146FE2906DA43
S31508005DC06B4602222046FEF721FB002803D000205E
S31508005DD030608520F2BDB4219DF800004843204478
S31508005DE090F82E20012A0ED0802A01D0852A03D1C8
S31508005DF0006B38600020306004F12E009DF800200A
S31508005E005143405CF2BD00F130029068002801D190
S31508005E10D068906004F138009DF800204A43805805
S31508005E203268824203D2002030608A20F2BD306098
S31508005E30002008E09DF800204A432244024492F8D4
S31508005E4040202A54401C32689042F3D39DF8001033
S31508005E502046FEF75BFA0120F2BDF0B40246106850
S31508005E6095681318506803EB5004C00748BF4D44A3
S31508005E70A3422DD013F8016B16F0030004BF13F8E4
S31508005E80010BC01C31090F2907D113F8011B0F316B
S31508005E9003E013F8017B05F8017B401EF9D10029C0
S31508005EA0E6D013F8010BC6F38106032E08BF13F8D4
S31508005EB0016B00EB0620404228440026B71E8F429D
S31508005EC01EBF10F8017B05F8017B761CF6D1CFE7DB
S31508005ED0F0BC02F10C007047002070472DE9F8432A
S31508005EE00F4615461C466A46D0F84C329847064671
S31508005EF00098002858D128463179884209D3794C28
S31508005F00009400231A4629463846FFF7E5FF20463F
S31508005F104AE00A9800280FD0306829460901405CF3
S31508005F20C00709D5704C009400231A4629463846FE
S31508005F30FFF7D2FF204637E0002C02D14FF0006071
S31508005F4032E0089F2D013068011D49593A688A4296
S31508005F5002D23960654827E0DDF824802844407875
S31508005F6088F800003068011D51F805904A46284413
S31508005F708168204600F02EFA98F80000092802D019
S31508005F80C7F800900FE03068001D4059396888420C
S31508005F9007D2002004F8090009F10109C7F80090A2
S31508005FA001E0C7F800900020BDE8F2832DE9FE4F16
S31508005FB004460D4616469B4601AAD4F84C32984725
S31508005FC08046019800286FD10C9F304698F8041037
S31508005FD0884209D3434C00943B6800223146284640
S31508005FE0FFF77AFF20467BE00D98002806D0D8F800
S31508005FF0000031460901405C022806D0324629468F
S315080060002046A36A9847002809D0394C00943B6873
S31508006010002231462846FFF75FFF204660E0B1467A
S315080060204FEA0919D8F80000484441788DF800105D
S3150800603043689A46C06802903868002801D08245AD
S3150800604044D359469DF80000626A9047019000289B
S3150800605008D000903B68524631462846FFF73CFF79
S3150800606001983DE03A685946D8F8000048448068E7
S3150800607000F0B0F99DF80000092808D138685045A5
S3150800608005D2D8F800104944896800220A54C7F88E
S3150800609000A00298002809D0324641462046029BB5
S315080060A098470190002801D0019819E0D8F8000017
S315080060B010F80900400707D532462946204604F558
S315080060C013735B6898470BE0002009E0C7F800A047
S315080060D0084C0094524631462846FFF7FDFE2046F6
S315080060E0BDE8FE8F1100090601000106050004053A
S315080060F0020001061000070638B515461C466A4612
S31508006100D0F84C32984701460098002807D128460F
S315080061100A79904203D2086800EB0510C46000981B
S3150800612032BD00207047002070478268521C82608A
S31508006130426832B10268531C036011704168491EF7
S31508006140416070472DE9F84F0746884600245A4DA6
S31508006150DFF86891B9F900108C4601E0641C18351F
S31508006160A6460FFA8EFE0CF10100704535DBBEF12E
S31508006170180F32DA1000F1D028780028EED116462A
S31508006180AEF1010EE64502D1491CA9F800109A465F
S3150800619000F02AFA834650464FF6FF718A4500D327
S315080061A00846D9F804108B4509D2A1EB0B018842A1
S315080061B005D200EB0B01C9F8041000F0FCF90A98A7
S315080061C0AE606F60C5F80C80DA44C5F810A0686147
S315080061D001202870204600B201E04FF0FF30BDE8EC
S315080061E0F28F10B401464FF0FF3291420ED0334978
S315080061F0B1F9002003461446A34201D1521E0A8073
S3150800620000212D4A00EB4003D80011544FF0FF300F
S3150800621010BC7047F8B54FF6FF7600F0E5F9014671
S31508006220264C62688A180023234D2F4615E0801AEB
S3150800623038613869B0420ED806460CE0A0EB010C6E
S31508006240B1FBF0FE00FB0EC03861032038703869D8
S31508006250B04200D806465B1C1837B4F900009C46C5
S315080062600FFA8CFC60450BDB3878C007F3D5386924
S315080062708242DCD378690028E0D102203870EAE748
S315080062806660304600F097F900260DE02878810709
S3150800629008D500F0FD002870AA68002A02D0E9682F
S315080062A068689047761C1835B4F90000314609B27B
S315080062B08842EBDAF1BD0000503200205818002061
S315080062C010B5334C204600F0B1F904F5217000F002
S315080062D0BDF904F5F260BDE8104000F0C3B9002826
S315080062E002D0012803D005E02A4800F0C7B92A4899
S315080062F000F0F8B9FF20704718B587B00446207833
S3150800630000F05AFA002801D1FF2019E00020019078
S31508006310207900906379A21D618802A800F02EFCFE
S3150800632001462078002803D11A4800F036FC07E019
S31508006330012804D102A9184800F072FC00E0FF20E9
S3150800634008B010BD38B50446114D05F5217000F0AA
S31508006350AAFC05F5F26000F0B5FC00F0C5FC28467D
S3150800636000F0E2FC002803D100F0CFFCFF2032BD8C
S31508006370284600F0E7FC01462046142200F03AF8C9
S315080063800121284600F0E5FC00F0BFFC002032BDE4
S31508006390FC1A0020801D00208C22002010B40269FF
S315080063A00A7002684A80027B4A71827B0A7100225F
S315080063B00CE000238C18A37107E0037B5B1E934255
S315080063C0F7DB83181B798C18A371521C082AF4DB97
S315080063D010BC704762B38B0708D0521E11F8013BF8
S315080063E000F8013B00F024808B07F6D1830740F0C4
S315080063F0208000BF103A07D330B4B1E83810103AFD
S31508006400A0E83810F9D230BC530724BFB1E8081009
S31508006410A0E8081044BF51F8043B40F8043BD207F3
S3150800642024BF31F8022B20F8022B44BF0B780370E7
S315080064307047121F17D35B0009D151F8043B20F8A7
S31508006440023B1B0C121F20F8023BF6D20BE051F858
S31508006450043B00F8013B1B0A20F8023B1B0C121FE9
S3150800646000F8013BF3D238BF121D521E24BF11F8A3
S31508006470013B00F8013BF8D870470268531C0360DB
S3150800648011707047010007D4012200F01F018A40ED
S315080064905D49400941F8202070470901020002D4ED
S315080064A05A48815470475A4802F00F02104400F8BF
S315080064B0041C704781B057490A6802430A60096894
S315080064C008400090009801B070475348006800F4EF
S315080064D0E0607047016841F001010160704701689A
S315080064E04908490001607047026822F070021143AA
S315080064F00160704741627047406A70478162704721
S31508006500C16270476FF0010101617047006900F0D0
S3150800651001007047C16841F00101C16070477047CA
S3150800652038B50220FFF7C6FF3C4C00212046FFF78E
S31508006530DBFF00F059FE0546FFF7C7FF002800D02D
S315080065406D003748854203D3B5FBF0F1491E00E0DC
S3150800655000212046FFF7D2FF4FF6FF712046FFF7CE
S31508006560CFFF00212046FFF7C5FF2046FFF7D2FFE1
S3150800657000211D20FFF791FF1D20FFF783FF20460E
S31508006580FFF7ADFF002000900346264A0146FFF7B5
S31508006590D9FD31BD10B5214C2046FFF7B7FF0128BC
S315080065A002D12046FFF7AEFF01201F490860BDE86B
S315080065B0104000F0F6B838B5044600F095FB174DC4
S315080065C02846FFF78CFF4FF6FF70041B2146284626
S315080065D0FFF790FF0020144908602846FFF77AFF66
S315080065E0BDE8314000F091BB10B50C4C2046FFF7D2
S315080065F083FF0D480068002803D02046BDE81040F8
S315080066007AE7002010BD000000E100E000E400E0A9
S3150800661018ED00E01C10024004100240000400407F
S3150800662040420F001F650008E03F002010B50446F1
S3150800663020231422044900F038FE04F520700021B6
S3150800664001804180204610BDF592000810B5044629
S3150800665000202060201D00F055FE002084F8080563
S31508006660204610BD10B5044600202060201D00F00D
S3150800667049FE002084F80805204610BD1FB50446CB
S31508006680002901D1FF2027E021601146206800F08B
S31508006690BDFE002801D1FF201EE01048D0E90023E6
S315080066A02146684600F052FF00226946206800F03D
S315080066B0F6FE684600F04CFF0948D0E9002321465B
S315080066C0684600F043FF01226946206800F0E7FEAD
S315080066D0684600F03DFF002004B010BDFCCB010861
S315080066E00CCC01081FB50446002901D1FF2027E07C
S315080066F021601146206800F089FE002801D1FF209C
S315080067001EE01048D0E900232146684600F029FF1C
S3150800671000226946206800F0C2FE684600F018FFAD
S315080067200948D0E900232146684600F01AFF0122ED
S315080067306946206800F0B3FE684600F009FF0020AD
S3150800674004B010BD04CC010814CC010838B5DFF834
S31508006750A843002104F1100000F006FFDFF89C535F
S315080067602A46DFF89C1300F0C7FD04F1E80000F0A4
S3150800677061FF2A46DFF88C1300F0BEFD0FF2C83021
S31508006780009004F584734FF48062282104F12400F4
S3150800679000F0D4FF2A46DFF87013BDE8384000F051
S315080067A0ABBDDFF8540301210170103000F022BFA1
S315080067B0DFF8580300F01EBF0120704780B501F0CE
S315080067C091F8401E8041C043C00F02BD10B5DFF8E6
S315080067D028430020607008E001F083FA00F027F9EA
S315080067E0052104F1100000F0E1FEA078002804D08D
S315080067F06078002801D1012060706078012804D1F2
S31508006800A078002801D10020607060780028E3D0C5
S31508006810642001F0E7FAE8E710B5B74CA088814292
S315080068200FD1A068042803DAA068401CA06002E023
S31508006830012001F04DFC04F1E800BDE8104000F02D
S315080068406ABF10BD01F0DFB9F0B585B00746B04D97
S315080068500FF26520C5F8500201F0EDFB0446A64E7E
S3150800686001F049F8B080002803D0802801DA002C0E
S3150800687001D02020B08000200190FF200090B3882E
S3150800688003F5C0734FF4A0520021284602F0B1F870
S315080068905FF00603AEA24FF4B051284602F0ECF8BA
S315080068A000200190FF200090B38803F5207341F281
S315080068B001420021284602F09CF80223AAA241F2CE
S315080068C00161284602F0D8F800200190FF200090C8
S315080068D0B38803F5607341F202420021284602F0AC
S315080068E088F80423A2A241F20261284602F0C4F8FD
S315080068F005F58270874901613179090441F4FA7115
S3150800690000680160FFF70CFE00F0E9FF02464FF44D
S315080069107A7042438048824208D08048824205D035
S315080069207F48824202D07F48824201D1002C00D0A3
S315080069307A4A39460020FFF7D2FC00F0CDFF00283E
S3150800694003D0802801DA002C00D014200146C9B2F1
S31508006950284602F0F3F90021284602F097F90021AB
S31508006960284602F037F80121284602F033F80221BA
S31508006970284602F02FF80321284602F02BF801AA30
S3150800698041F20901284602F0AAFA044601980028AD
S3150800699007D101F07EFB024666A12068806802F0F6
S315080069A053FB01AA41F20A01284602F098FA044666
S315080069B00198002809D10220009005235FF0010202
S315080069C05EA12068806802F03FFB00F08BFF00287C
S315080069D011D000F08AFFADF80C00022004900020C8
S315080069E00290019004A8009003AB002241F217011F
S315080069F02846FFF7DBFA0521284602F047F9B08852
S31508006A0001F0FBF806F1E80000F039FE00F061FF3E
S31508006A10F0604549684602F037FB014606F1240056
S31508006A2002F089FB684600F093FD05B0F0BD30B56D
S31508006A3089B0314C2078002803D000202070FFF759
S31508006A40E9FB04F1E805284600F030FE374988429C
S31508006A5006DB0020A06001F03BFB284600F05BFE49
S31508006A6004A802F047FC03E000F042FF00280CD01F
S31508006A7004A8FFF767FC00280FD1694604A8FFF7AA
S31508006A808DFCBDF80200C009EED021480021C0F8EF
S31508006A904812694602F024F8EAE709B030BD012039
S31508006AA015498870704714484078012801D101209B
S31508006AB0704700207047000038B50D4614466A46F0
S31508006AC002F00DFA01460098002810D142F6FF7030
S31508006AD0854206D1084AD068154B002809D118689E
S31508006AE0D060086800EB0410806800F08CFE002077
S31508006AF032BD1860FBE7000010050020E83F0020C3
S31508006B00FB7500085B7600084F92000820050020F8
S31508006B10B41500201968000848E8010090D0030061
S31508006B2020A1070040420F00CD67000880841E00A0
S31508006B309C3F0020312E25750000000025752E2566
S31508006B40752E25750000000063616E6F70656E0016
S31508006B5008010040100200400803004008040040F5
S31508006B6008050040100600402007004020080040A5
S31508006B7020090040100B0040100D00401CB50446CB
S31508006B809DF8140001909DF810000090204602F030
S31508006B90B9FB00202061204616BDF8B505460F460C
S31508006BA02868002801D1FF20F2BD284600F07BF8AE
S31508006BB0002495F80805002813D102F01DFD0646A5
S31508006BC083B068460ECF0EC0396801600C3F0EBC14
S31508006BD0286800F02CFC012800D10124304602F078
S31508006BE021FD200016D100F07FF8281D02F04AFD8D
S31508006BF000280DD0281D02F04BFD0446394602F048
S31508006C004EFD002020610121281D02F059FD0124B6
S31508006C1000F07BF8002C01D00020F2BDFF20F2BD69
S31508006C20F8B505460F462868002801D1FF20F2BDB1
S31508006C30284600F047F8002495F80805002813D1DF
S31508006C4002F0DAFC064683B068460ECF0EC03968F5
S31508006C5001600C3F0EBC286800F0E9FB012800D152
S31508006C600124304602F0DEFC200016D100F03CF884
S31508006C70281D02F007FD00280DD0281D02F008FD8A
S31508006C800446394602F00BFD012020610146281D05
S31508006C9002F016FD012400F038F8002C01D000207F
S31508006CA0F2BDFF20F2BD10B504462068002808D0C2
S31508006CB000F0D7FB7F2804DA2068BDE8104000F012
S31508006CC0DFBB10BD10B504462068002808D000F0C8
S31508006CD0C8FB7F2804DA2068BDE8104000F0D0BB66
S31508006CE010BD6FF01C00704780B502F0F1FC0C482F
S31508006CF0016811F1010F05D10A48402200F134015B
S31508006D0002F0F4FC491C016001BD05490868002829
S31508006D1004D0401E086001D102F0F4BC70470000A0
S31508006D20CC3F002074BA010800F520714A88104645
S31508006D3009880B46914201D3181A7047C0F1200002
S31508006D4018187047B0F8821201EB810200EB820036
S31508006D507047B0F88222891801F01F01A0F8821244
S31508006D60704725002DE9FC410546DFF800452878DF
S31508006D70C00757D5606800F00C00042807D0606883
S31508006D8000F00C0008280AD16068C00307D52068FF
S31508006D90800347D56868002844D1012069E16868FE
S31508006DA0B0F5803F04D1206840F4803020601DE0B3
S31508006DB0002808D1206820F480302060206820F45C
S31508006DC08020206012E0B0F5A02F206807D140F49B
S31508006DD080202060206840F48030206006E020F49F
S31508006DE080302060206820F48020206068680028B1
S31508006DF00CD002F0A4FC06462068800312D402F0E8
S31508006E009EFC801B6528F7D3032032E102F097FC2D
S31508006E1006462068800305D502F091FC801B65288C
S31508006E20F7D3F1E72878800718D5606810F00C0FBB
S31508006E3007D0606800F00C00082825D16068C003F8
S31508006E4022D42068800702D528690128A5D12068A0
S31508006E5020F0F800696940EAC10020602878000738
S31508006E603ED5DFF81414A869002860D00120086010
S31508006E7002F065FC0646606A80072ED402F05FFCC5
S31508006E80801B0228F7D9BFE7DFF8F0132869002826
S31508006E9015D00120086002F052FC064620688007DB
S31508006EA005D402F04CFC801B0228F7D9ACE7206811
S31508006EB020F0F800696940EAC1002060CEE70020AA
S31508006EC0086002F03CFC064620688007C6D502F03A
S31508006ED036FC801B0228F7D996E7012000F0B4F9A2
S31508006EE0287840077BD50026E069C00009D4E06908
S31508006EF040F08050E061E06900F080500090009812
S31508006F000126DFF87C733868C0051ED4386840F45B
S31508006F108070386002F013FC80463868C00514D4C7
S31508006F2002F00DFCA0EB08006528F6D36CE70020FC
S31508006F30086002F004FC0646606A8007D0D502F0B5
S31508006F40FEFB801B0228F7D95EE7E868012804D112
S31508006F50206A40F0010020621CE0002808D1206A5F
S31508006F60400840002062206A20F00400206211E0F8
S31508006F700528206A07D140F004002062206A40F004
S31508006F800100206206E0400840002062206A20F0E6
S31508006F9004002062E86800280DD002F0D0FB0746FE
S31508006FA0206A800715D402F0CAFBC01B41F289315A
S31508006FB08842F5D328E702F0C2FB0746206A800715
S31508006FC007D502F0BCFBC01B41F289318842F5D3D4
S31508006FD01AE7012E03D1E06920F08050E061E869E4
S31508006FE0002845D0616801F00C0108293FF4D5AEA8
S31508006FF0DFF8886202282DD10020306602F09FFB58
S3150800700007462068800105D502F099FBC01B0228B7
S31508007010F7D9F9E6286AB0F5803F05D1616821F409
S315080070200031A86801436160616821F47411286A17
S315080070300143686A014361600120306602F07FFB04
S3150800704005462068800113D402F079FB401B02280C
S31508007050F7D9D9E60020306602F071FB05462068AC
S31508007060800105D502F06BFB401B0228F7D9CBE659
S315080070700020BDE8F6812DE9F04105460E46814F10
S31508007080386800F00700B04209D23868C00856EAE6
S31508007090C0003860386800F00700B04261D1734C10
S315080070A02878800705D5616821F0F001A8680143B2
S315080070B061602878C00745D56868012803D121682A
S315080070C0890308D44DE00228216802D1890102D437
S315080070D047E0890745D56168890850EA81006060FC
S315080070E002F02DFB8046686801280ED1606800F022
S315080070F00C00042826D002F022FBA0EB080041F27F
S3150800710089318842F2D303204EE002280DD1606807
S3150800711000F00C00082815D002F011FBA0EB0800BF
S3150800712041F289318842F2D3EDE7606810F00C0F1E
S3150800713008D002F004FBA0EB080041F2893188422E
S31508007140F3D3E0E7386800F0070086420BD23868C8
S31508007150C00856EAC0003860386800F00700B04238
S3150800716001D0012020E02878400705D5616821F480
S31508007170E061E868014361602878000706D5606821
S3150800718020F46050296940EAC100606000F00EF8FA
S315080071903D496268C2F30312895CC84035490860F4
S315080071A00F2002F0C7FA0020BDE8F08137490A68C7
S315080071B002F00C00082812D137A0C2F38343C05C42
S315080071C0D20309D538A20968C1F34041525C28495F
S315080071D04843B0FBF2F070472D49484370472448AE
S315080071E0704724480068704780B5FFF7FAFF2949B9
S315080071F0264A1268C2F30222895CC84002BD80B5DD
S31508007200FFF7EFFF2349214A1268C2F3C222895CBD
S31508007210C84002BD0F2202601C4A136803F003032C
S315080072204360136803F0F0038360136803F4E063B4
S31508007230C3601268D20802F4E0620261114800686D
S3150800724000F007000860704781B00A490968C90854
S315080072504FF47A72B1FBF2F14843009000BF0098F0
S31508007260411E00910028F9D101B070470010024074
S3150800727000127A00F01800208004424200004242C0
S315080072800070004000200240045501080410024026
S3150800729000093D00B8D301080203040506070809DA
S315080072A00A0B0C0D0E0F101001022DE9F0410646CF
S315080072B00F4690461C463546380018BF002D05D0A7
S315080072C024B13046B847641E4644FAD12846BDE87C
S315080072D0F0812DE9F0411646044673430D46E7183A
S315080072E07642A046B84503D237443846A847F9E758
S315080072F0A4F10800BDE8F0810B460146184602F0E5
S315080073004FBA250010B50446402314220449FFF756
S31508007310CCFF04F5A060002101804180204610BD05
S31508007320F5920008002101F0AFBE2DE9FF4107469E
S315080073300C4615461E463248386000224C21381D38
S3150800734002F072FA092310222E4907F15000FFF7BE
S31508007350ACFF07F1E00002F085FA4FF000080FE0F5
S315080073600021684601F090FE014607F1500000EB47
S31508007370081002F00DFB684600F0EAF808F101086B
S31508007380B8F1090FECD333462A462146381D02F0D8
S315080073903EFB3A460FF28911381D02F0B5FB384616
S315080073A004B0BDE8F08138B584B0044614482060BE
S315080073B000250EE00021684601F066FE01462846D3
S315080073C00246D2B2204600F06AF8684600F0C0F8D5
S315080073D06D1C082DEEDD201D02F09DFB201D02F020
S315080073E0A7FB04F1E00002F0A9FA092310220649D6
S315080073F004F15000FFF76DFF204605B030BD0000D0
S31508007400BCCE0108257300085175000838B5044636
S315080074100D462168896888472946201D02F0D5FB54
S31508007420054620462168C9688847284632BD0EB4F5
S315080074301EB504460020019005A883B06946D0E928
S315080074400023C1E90023D0E90223C1E902230EBCC7
S31508007450201D02F00AFC1EBC5DF810FB001D02F0A0
S3150800746063BC38B50446216889688847201D02F040
S315080074709FFC054620462168C9688847284632BDCC
S3150800748038B50446216889688847201D02F094FCAF
S31508007490054620462168C9688847284632BDF8B59A
S315080074A084B004460D4616462168896888473046E2
S315080074B014EB0017284602F0D5FD002807F1500006
S315080074C010D002F0CFFD002801D102F0D2FD2946E6
S315080074D007F1500002F05CFA01223146201D02F045
S315080074E033FD16E002F0BEFD002801D002F0C2FD11
S315080074F00021684601F0C8FD014607F1500002F078
S3150800750047FA684600F024F800223146201D02F0AA
S315080075101BFD20462168C968884705B0F0BD0000F4
S3150800752010B510EB011404F1500002F09BFD002881
S3150800753005D004F15000BDE8104002F09DBD10BD15
S31508007540E03002F0BDB9E03002F0D8B902F0A6BDCD
S3150800755010B50446E168002901D0896888472046A5
S3150800756010BD02F0A7BD2E0010B504464FF6FF72F7
S3150800757000F002F8204610BD7FB504460D461646B3
S315080075806846102102F0A2FD201D029010200390EB
S315080075906A462946304602F027FF2060002804D1B3
S315080075A02F22124920A002F0A1F87FBD1CB50C4677
S315080075B0006802F033FF002801D1012016BD10F142
S315080075C0030F01D1002C02D010F1020F01D10121C5
S315080075D000E00021002907D1002100910B46024650
S315080075E00AA1034802F06AFF002016BDC0C40108BC
S315080075F014010280006802F027BF10B5044620680F
S3150800760002F036FF204610BD0000000053656D618C
S3150800761070686F726520616371756972652066614D
S31508007620696C6564000000005F696420213D204E96
S31508007630554C4C0010B50446002020600146C4E9AC
S315080076400201C4E9040102F063FFA061012020776A
S31508007650204600F060F8204610BD10B50446FFF736
S3150800766043FB2068002804D0207F002801D002F0C0
S3150800767001FD00202060FFF748FB204610BD10B52D
S315080076800446FFF731FB206800280BD1207F00282D
S3150800769001D002F0EEFCA06903F089F9C4E9020101
S315080076A001202060BDE81040FFF72FBB0CE080B535
S315080076B000F00AF803F08CF90249BDE8044003F02B
S315080076C0ABB900000024744938B50446FFF70CFB33
S315080076D0204600F00AF8D4E90423141843EB010500
S315080076E0FFF713FB2046294634BD70B5064600242D
S315080076F02546FFF7F9FA3068002807D0B06903F085
S3150800770056F9D6E90223841A61EB0305FFF7FDFA59
S315080077102046294670BD10B50446FFF7E5FAA0696C
S3150800772003F045F9C4E9020100200146C4E9040151
S31508007730BDE81040FFF7E9BAB9E77047F8B504465F
S315080077400D4616461F460C4820600021201D01F0F4
S315080077509BFC002104F14000FFF706FF04F15400EA
S3150800776002F080F8069800903B46324629462046A5
S3150800777001F0D7FC2046F2BDF8D00108E220DFF878
S31508007780481208607047DFF844225060117070474D
S31508007790704710B5DFF8384203E0204600F005F8D8
S315080077A00C3460680028F8D110BDFEB5044665683B
S315080077B02089801C232801DB0020FEBDDFF80C622F
S315080077C07768C117CDE900012268002306F1080190
S315080077D038463F687F69B847002801D00020FEBDBB
S315080077E02189891C89B206F1080000F03FF90028B2
S315080077F001D10020FEBD228906F108012846FEF7C0
S31508007800E9FD0120FEBD024670480078C00708D58C
S315080078106F4800E00C304168002902D09142F9D146
S3150800782000E070477FB5044622891046801C23284D
S3150800783001DB00204BE0654D616805F10800FEF7A5
S31508007840C9FD02A803F074F9228905F1080102A806
S3150800785003F082F902A803F08FF905F108002189DF
S315080078600844BDF808100170BDF80810090A4170EF
S315080078706E682089801CC117CDE9000122680023A3
S3150800788005F1080130463668B669B047002801D0C8
S3150800789000201CE06E682089801CC117CDE9000114
S315080078A02268002305F10801304636687669B04734
S315080078B0002801D000200AE02189891C89B205F137
S315080078C0080000F0D3F8401E8041C043C00F04B042
S315080078D070BD5748006870473E48008870473E4864
S315080078E0008870473D48008870473D4800887047C3
S315080078F03C48008870473C48008870473B480088E9
S3150800790070473B48008870473A48008870473A48AD
S31508007910008870473948008870473948008870479A
S3150800792038480088704738480088704737480088C4
S315080079307047374800887047364800887047364889
S315080079400088704735480088704735480068704792
S315080079503448006870473448006870473348006800
S3150800796070473448007870473348B0F900007047CC
S31508007970324890F900007047314890F90000704786
S315080079803048007870473048008870472F480068AC
S3150800799070472F48006870472E48006870472E4881
S315080079A0008870472D48008870472C490880704722
S315080079B02B48008870472A4908807047294800885C
S315080079C07047294800887047943F0020AC3B002048
S315080079D0E09E0108C81A0020CA1A0020CC1A002006
S315080079E0CE1A0020D01A0020D21A0020F43F002018
S315080079F0F63F0020F83F0020FA3F0020FC3F002019
S31508007A00D41A0020D61A0020FE3F0020D81A0020DB
S31508007A10DA1A0020DC1A0020DE1A0020E01A0020FC
S31508007A20401200204412002048120020983F0020EF
S31508007A309C3F002039400020024000203A400020A8
S31508007A403B4000203C40002004400020A03F00208E
S31508007A50A43F0020A83F0020064000200A4000203E
S31508007A600C4000200E400020104000207CB5044643
S31508007A700D462E46032E17DB684603F059F8AA1E54
S31508007A8092B22146684603F067F8684603F074F830
S31508007A90A019801EBDF800100278407842EA00223C
S31508007AA0914201D1012076BD002076BD80B5C1483E
S31508007AB0FFF7C0FDC04AC149BDE80840FFF71CBC36
S31508007AC00120BF49087070470120BD4948707047BA
S31508007AD030B4426952880B46446854F83240A46967
S31508007AE003F5C0652560446854F83240A46A03F576
S31508007AF0B0632360406850F83200806B017030BC78
S31508007B00704741694988426852F8312092694FF4B2
S31508007B10C0631360426852F83120926A4FF4B0632A
S31508007B201360406850F83100806B0021017070477F
S31508007B307FB504460D460020019004200390A04E10
S31508007B4002A8009003AB01AA2046FEF72CF90128EB
S31508007B502AD10198B0F5D17F11D106F110014FF461
S31508007B60827003F00AF8002802D003F009F800E052
S31508007B7000207060934A944904F09AFE14E040F29B
S31508007B80A511884210D106F110014FF4847002F055
S31508007B90F4FF002802D004F095FE00E00020706093
S31508007BA0884A894906F03CFC022229462046FCF709
S31508007BB069FC2046FFF7A5FF0220F060012030701F
S31508007BC07FBD3EB504460D46FCF7D3FA2946204646
S31508007BD0FFF77EFF002002907C4801900620009067
S31508007BE000234FF4805229462046FEF7CFF8002896
S31508007BF002D002207249C86037BD7149488001F534
S31508007C008C70FFF73CBD7248704738B56C4C60689D
S31508007C10002801D0012032BD04F58C752846FFF7EF
S31508007C208BFDE168002905D002290DD1694906F0C6
S31508007C3001FC09D82846FFF76EFD0120E06061883F
S31508007C40C9B26548FFF7BDFF002032BD70B55C4C70
S31508007C5004F58C752846FFF76FFD627821780029B0
S31508007C6005D0002A03D15D4906F0E4FB09D9002AAC
S31508007C7003D05B4906F0DEFB03D9564906F0DAFB6A
S31508007C8001D8012600E00026606806F07CFC002882
S31508007C9026D0002E24D02846FFF73DFD0020607030
S31508007CA020704D4D02226188C9B22846FCF7EAFBCE
S31508007CB02846FCF75EFA6188C9B22846FFF708FF2E
S31508007CC0606806F044FC01286188C9B2284603D1D9
S31508007CD0BDE8704004F0CCBCBDE8704006F064BA5C
S31508007CE070BD2DE9F04F8FB0354CA068002802D042
S31508007CF0012807D05BE0FFF788FF002857D001204E
S31508007D00A06054E0606806F020FC0546606806F04E
S31508007D101EFC012802D1FFF718FE01E0FFF71BFE43
S31508007D202860606806F011FC0546606806F00FFCDE
S31508007D30012802D1FFF70CFE01E0FFF70FFE68608D
S31508007D4060680790FFF728FE0890FFF722FE0446B2
S31508007D50FFF71CFE0546FFF716FE0646FFF710FE60
S31508007D600746FFF709FE8046FFF702FE8146FFF742
S31508007D70FBFD8246FFF713FE8346FFF7F2FD014639
S31508007D80089806900594049503960297CDF8048002
S31508007D90CDF8009053465A4609A806F060FB0146FE
S31508007DA007980246126892699047FFF74FFF0FB08F
S31508007DB0BDE8F08FF0040020E83F00205B7600085D
S31508007DC0D8030020C97A0008C17A0008317B000868
S31508007DD0DC03002001000040B4150020CECC4C3E48
S31508007DE00100803F80B506F03FFF002805D06C22D1
S31508007DF0DFF8081002A001F079FC01BD00B1010806
S31508007E00737461747573203D3D206F734F4B00008A
S31508007E10F8B588B0DFF86843DFF868330C220B2121
S31508007E20201DFFF782FADFF860532A46DFF85C1355
S31508007E30FFF762FA4FF48063D54AD64904F57270A3
S31508007E4006F02CFF2A46D449FFF756FA192104F5FD
S31508007E50847007F017F80122152104F5927007F0CF
S31508007E601EF80122162104F5A07007F018F8012261
S31508007E70172104F5AE7007F012F8182104F5BC7046
S31508007E8007F01CF804F5CA7007F026F82A46C34915
S31508007E90FFF732FA06200790052006901020059075
S31508007EA00720049012200390112002901B200190B5
S31508007EB01A2000901F231E221D2104F5037007F0C7
S31508007EC02FF800200090042301221C2104F552708B
S31508007ED007F0F4FA082104F5597007F002FBB04ED2
S31508007EE02A463146FFF708FA04F560770021384636
S31508007EF007F0F7FA2A463146FFF7FEF90F2104F58F
S31508007F00677006F0BFFF0246394604F56E7009B081
S31508007F10BDE8F04007F0F4BA0268002902D080688C
S31508007F2002607047C0680260704741680968006867
S31508007F3001400846401E8041C043C00F704730B517
S31508007F4085B09848016821F0100101608C4C00F05A
S31508007F50A0F82070002104F5847007F011FB04F5E1
S31508007F6059754FF47A71284607F010FB0021284608
S31508007F7007F019FB04F56075FA21284607F006FB99
S31508007F800021284607F00FFB002104F5677007F06B
S31508007F90F7FA04F5727006F0A1FE04F5037007F00F
S31508007FA03DF8002104F5BC7007F00AFB7E480090F6
S31508007FB000220121684607F011FB05B030BD0120FB
S31508007FC07A4908607A487B490160062141604FF486
S31508007FD04071816007F00ABB754807F02DBB7648EB
S31508007FE0704776487047014681F00101744807F0EA
S31508007FF0C7BA10B5724C204607F024FB411E8941CA
S31508008000C90F2046BDE8104007F0BABA002802D0CA
S315080080104FF07C5100E000216A4807F015BB80B597
S31508008020684807F021FB684906F004FA01D80120E0
S3150800803002BD002002BD80B5644807F021FB401E42
S315080080408041C043C00F02BD6149002802D002200A
S31508008050087070470120087070475D480078401E18
S315080080608041C043C00F704759480078002800D1A6
S31508008070704700B585B04C4900910022022800D10E
S3150800808001220121684607F0A9FA07F016FB05B098
S3150800809000BD38B53A4C04F5927007F0F1FA451E62
S315080080A0AD4104F5A07007F0EBFA002801D00020D6
S315080080B000E0022050EAD57504F5AE7007F0E0FA44
S315080080C0002801D0002000E004200543284632BDE0
S315080080D018B42B4C6070002801D0032100E002215F
S315080080E000231A4604F5CA7001B010BC07F0EEBAB0
S315080080F023484078704700231A461146354807F04A
S31508008100E5BA00231A460121324807F0DFBA1FB53F
S31508008110044600222F49684607F0E2FA009810281C
S3150800812003D101982060012000E0002004B010BDB2
S3150800813070B50446124D05F50376304606F0FAFF8B
S315080081402146884216D0200007D0002105F5527036
S3150800815007F0EDFA3220FFF745FE2146304606F0D5
S31508008160A5FF002C06D1012105F55270BDE8704027
S3150800817007F0DDBA70BD0146174807F0D1B900000F
S315080081801028002090D00300E83F0020A7730008BD
S3150800819000E4010800E00108C5EC000811D2010856
S315080081A079CD0108002002400028004080044242A0
S315080081B0703F00200030004014280020D82B0020F3
S315080081C018290020742B0020CECCCC3D882900200D
S315080081D038400020A4290020C82B00202DE9F84F9C
S315080081E088B044694568238905EBC30303EBC103DB
S315080081F0648905EBC40404EBC1074FF00008C146C7
S315080082003968D1F808A01968896C09781170196855
S3150800821089690968C1F30A01518041461171054609
S3150800822016460022082106A801F0FEFA38684146DB
S31508008230C9B200EB0110806904682146090C04F0F4
S31508008240FF04002C29D004EB090BBBF1410F24D203
S31508008250621ED208521C0592012203920022029243
S3150800826004AA019205AA009206AB0268120AD2B2C3
S315080082702846FDF733FE002818D10020029009F0A1
S315080082800700019006EBD900801D009000231A46CE
S3150800829006A9204600F03DF9D94608F101084046EE
S315080082A09AF80010C0B28842BBD303E0FF2009B099
S315080082B0BDE8F08FA9F101094FEAD90909F10109C9
S315080082C086F805900020F2E72DE9F84F88B00223DA
S315080082D04FF000094D46AA460A79002A40F0A480C4
S315080082E0426992888469A488002A04D1484609B05C
S315080082F0BDE8F08F04239442F8DB1E46022E02D016
S31508008300042E0CD0F7E7466856F83260B669366828
S315080083104F88BE42EED06D1C521C92B2EBE7426902
S31508008320B2F806B0A8465FFA88F8426802EBCB02B4
S3150800833052F83820926806460F468DF80C50079278
S3150800834038E02C78002C33D07879C00004EB09018A
S3150800835088422DDB00200290019005A8009000239A
S315080083604A46921009EB527202F0F802A9EB020291
S31508008370D2B2484607EBE000811D204600F0C9F856
S31508008380601EC010401C049029680120029000203D
S31508008390019004A8009005AB0A46120AD2B2090C4D
S315080083A03046FDF703FE00281DD14C44E4B2A14631
S315080083B00AF1010A504607990978C0B2884214D2D0
S315080083C00022082105A801F02FFA706800EBCB00FF
S315080083D050F8380018305146C9B209014558002DE1
S315080083E0AFD1FF2083E7FF2081E7F068002819D086
S315080083F0716851F83B10896D0C88002C12D030F941
S315080084001800FDF7EEFE002000904FF47A70444302
S31508008410234632699DF80C103046FDF793FEF16845
S3150800842021F81800002062E7012A7FF45FAF0126D1
S315080084304269128983691B89002A3FF457AF0446AB
S3150800844000E004269342FFF651AF3046012804D0D7
S3150800845004280ED005284DD0F4E7606850F832009D
S31508008460806900684F88B842EBD06D1C521C92B2E6
S31508008470E8E7606850F83200806A0078FD280AD07C
S31508008480FC2810D12846C0B200EB8006B000A668CA
S31508008490375CFF0701D40526D4E73044801DFDF775
S315080084A02BFF484623E7FF2801D0FE2820D128467F
S315080084B0C0B200EB80018E00A068801C805FFDF7CB
S315080084C090FEA168891C8853A068001D805FFDF78F
S315080084D088FEA168091D8853A068815D01F0FE0128
S315080084E08155EDB22946204600F00EF94846FEE6CB
S315080084F0FF20FCE66A462946C9B22046FFF76EFE0B
S31508008500002801D0FF20F2E66846FDF7F5FE48464A
S31508008510EDE62DE9F043079E089C099D14E04FF00F
S31508008520010C0FE04FF0010C6144A4465FFA8CFC85
S31508008530BCF1080F07DB0024AC46BCF1000FEED0F7
S315080085404FF0FF3C6644C01B0746FFB2002F3ED0E3
S31508008550A71A7FB291F800C0012F02DB0CFA07FCBC
S3150800856003E0C7F1000E4CFA0EFCC4F1080E01DB5D
S31508008570F04601E0C2F108080746FFB25FFA88F83C
S31508008580474500D947463C194FF0FF0808FA04F951
S3150800859048FA0EF848EA090896F800E008EA0E0EC6
S315080085A086F800E02CEA080C4CEA0E0C86F800C0A7
S315080085B0BA1894465FFA8CFCBCF1080FB5DB0022AA
S315080085C09C46BCF1000FADD04FF0FF3CACE7BDE8D0
S315080085D0F08310B51446806801EB810200EB820037
S315080085E0801D21460E22FDF7F5FE2046BDE8104007
S315080085F0FDF782BE2DE9F84185B006460F4696F985
S31508008600E600002838D0384600EB80014FEA81089A
S31508008610B06810F80800C0072ED470690489384677
S315080086200419A4B2706850F83400806900680028FC
S3150800863022D400220E2101A801F0F6F801AA394633
S315080086403046FFF7CBFD002816D1B06800F10801C7
S3150800865031F80810BDF8062091420FD14044C17A7E
S315080086609DF80920914209D108220DF10A010C3022
S3150800867007F064F8002801D1002041E0706850F83E
S315080086803400816D0C88806B0588002C14D0B06886
S315080086904044B0F90200FDF7A4FD002000904FF415
S315080086A07A70444323460FF2610239463046FDF795
S315080086B049FDB16841444880002D1BD0B068001DB3
S315080086C030F90800FDF78DFD002000906420454331
S315080086D02B460FF2550239463046FDF733FDB16891
S315080086E0091D21F80800B06810F8081041F00101CA
S315080086F000F8081001AA39463046FFF76AFF01203C
S3150800870006B0BDE8F081000018B401EB81029200C2
S315080087104FF0FF3384681444638000238468083468
S31508008720A352C9B214BC65E718B401EB81029200E2
S315080087304FF0FF3384681444A38083689C5C04F07C
S31508008740FE049C54C9B214BC54E770472DE9F8439B
S3150800875084B005460E4600274FF003096869048968
S31508008760A869B0F8088095F9E600002800F09D8011
S31508008770002C00F09A803A460E21684601F054F81B
S3150800878001E04FF00B09A045C0F28F80B9F1030F45
S3150800879006D0B9F1050F77D0B9F10B0F7CD082E07E
S315080087A0686850F83400816909680029E9D4816A43
S315080087B0300027D00878002824D0F12822DAAA68C1
S315080087C007EB87008000135C5B1C1354AA68135CD4
S315080087D091F800C0634515D1002111540A460E21AF
S315080087E0684601F021F86A4638460146C9B2284665
S315080087F0FFF7F4FC002802D04FF00B09C3E74FF04F
S315080088000509C0E7300020D00878FC281DD107EB01
S3150800881087004FEA8009A8684844821D3846014601
S31508008820C9B22846FFF7DAFC0028A86810F809102C
S3150800883004D001F0FE0100F8091003E041F001013F
S3150800884000F809104FF00B099DE7300002D00878B0
S3150800885000280DD0300014D10878FF2801D0FE2852
S315080088600FD1A86807EB87018900405CC00708D4C8
S3150800887038460146C9B22846FFF7BCFE4FF00B0939
S3150800888081E74FF00B097EE76A4639462846FFF727
S31508008890A0FE4FF00B0976E77F1CFFB2641CA4B25A
S315080088A04FF003096FE7FF2000E0002005B0BDE8A0
S315080088B0F08370B504460D4694F9E60000282AD0E0
S315080088C0921E012A01D9D21E25D1606861690989DB
S315080088D000EBC1002D1AED10EDB205EB8500860000
S315080088E0A0683044B0F90200FDF77BFCA16831446A
S315080088F04880A0683044B0F90400FDF772FCA1680E
S31508008900314488800020A168885529462046FFF70B
S31508008910FBFE002070BD002070BDF8B504464FF47C
S31508008920C05560690689A0690789300014D117E027
S315080089306A46294689B22046D4F84C3298470146F9
S315080089400098002806D109480A68D0620A68D063E8
S315080089500968C8656D1C761C304680B28742E7DA1E
S3150800896000212046FFF7F2FEF1BD0000B38800089B
S315080089702DE9F0410446002560690689A069078942
S31508008980300021D124E005EB85004FEA8008A06875
S315080089904044B0F90200FDF724FCA1684144488030
S315080089A0A0684044B0F90400FDF71BFCA1684144E7
S315080089B088800020A16801F80800A168083121F81C
S315080089C008006D1CEDB2761C304680B28742DADAB2
S315080089D0BDE8F08142691289002A09D0891889B24E
S315080089E0406850F831008069016841F00041016033
S315080089F070472DE9F84185B006460F4690460C9C0F
S31508008A000D9D04930420039000200290019003A872
S31508008A10009004AB012241463046FDF7C7FA04949C
S31508008A200120039000200290019003A8009004AB57
S31508008A30022241463046FDF7B9FA04970120039011
S31508008A4000200290019003A8009004AB042241463E
S31508008A503046FDF7ABFA04950220039000200290F9
S31508008A60019003A8009004AB052241463046FDF765
S31508008A709DFA06B0BDE8F0812DE9F84185B00446B7
S31508008A800D4616461F4638460490012003900020DE
S31508008A900290019003A8009004AB00222046FDF73F
S31508008AA085FA4FF0000814E056F8280004900420D0
S31508008AB0039008F1010800200290019003A8009095
S31508008AC004AB4246D2B229462046FDF76FFA5FFA52
S31508008AD088F838468045E7DB06B0BDE8F081704780
S31508008AE04A881346DB1130D05B1E08D09B1E072B25
S31508008AF015D9083B012B1AD9DB1E1ED0704700F189
S31508008B00E203802A05D193F90210002923D006F042
S31508008B10B1BE93F90120002A1DD006F0ECBE00F183
S31508008B20E20292F90420002A15D0FFF7CDBB90F98E
S31508008B30E220002A0FD0FBF739BD00F1E20292F9D4
S31508008B400320002A07D006F002BF026A1278002A1C
S31508008B5001D007F0B0B8704770B504460E4696F9CE
S31508008B60010004F1E105002806D095F90110002955
S31508008B7002D1012068700AE0002808D195F90100A1
S31508008B80012804D1002068702046FBF7F2FA96F90E
S31508008B900300002809D095F90310002905D1012002
S31508008BA0E870204606F004FE0AE0002808D195F988
S31508008BB00300012804D10020E870204606F028FEAC
S31508008BC096F90400002809D095F90410002905D162
S31508008BD001202871204607F05AF80AE0002808D133
S31508008BE095F90400012804D100202871204607F0D1
S31508008BF056F896F90200002809D095F902100029BE
S31508008C0005D10120A870204606F065FE0AE0002876
S31508008C1008D195F90200012804D10020A870204641
S31508008C2006F068FE96F90500002809D095F90510A2
S31508008C30002905D1012068712046FFF76EFE0AE07B
S31508008C40002808D195F90500012804D1002068718B
S31508008C502046FFF78DFE96F90000002806D095F904
S31508008C600010002902D10120287070BD00280AD101
S31508008C7095F90000012806D1002028702046BDE895
S31508008C80704007F076B870BD000000003EB5044697
S31508008C9004F1E00528780A4603469A4224D00029BA
S31508008CA006D0042933D0052920D07F290ED040E0EC
S31508008CB076A0D0E90023CDE9002300202870694674
S31508008CC02046FFF749FF2046A968884771A0D0E9E2
S31508008CD00023CDE900237F20287069462046FFF748
S31508008CE03BFF2046E968884728783EBD002820D003
S31508008CF06AA0D0E90023CDE900230520287069463B
S31508008D002046FFF729FF204629698847ECE700280F
S31508008D100FD000BF63A0D0E90023CDE900230420CB
S31508008D20287069462046FFF717FF20466969884775
S31508008D30DAE7FF203EBD0068007870472DE9F84362
S31508008D4084B004460D006069008800F090802F46C4
S31508008D50802F80F28C80002821D0616851F830106D
S31508008D608969226812780B68164606F5C066B3420A
S31508008D7001D0FF2A02D107F5C0620A60616851F87E
S31508008D803000806A2168097802680B4603F5B063EB
S31508008D909A4201D0FF2902D107F5B06101604FF070
S31508008DA0000960698688A069B0F804804FEA0D005A
S31508008DB03EA11022FDF71EFB002E19D11DE06068AA
S31508008DC050F836008069216809786A4652F82920E1
S31508008DD003688C469444634501D0FF2902D129468D
S31508008DE08A18026009F101095FFA89F9761CB6B298
S31508008DF0B04502DBB9F1040FE1DB60690689A069B9
S31508008E00B0F808804FEA0D002CA11022FDF7F2FAFF
S31508008E100020002E18D11BE0616851F836108969C8
S31508008E20226812786B4653F82030D1F800C096466F
S31508008E309E44F44501D0FF2A02D12A46D3180B6076
S31508008E40401CC0B2761CB6B2B04501DB0428E3DB91
S31508008E5020680078D4F87C120A68034680339A4260
S31508008E6001D0FF2801D180370F602068057005B052
S31508008E70BDE8F0837047016A0978002903D1812289
S31508008E80002106F096BF7047704770470100000042
S31508008E9000000000000101010100010000010101BC
S31508008EA001010000000000000100010000020000AE
S31508008EB00003000000040000000500008001000017
S31508008EC08002000080030000800400009F2804D16F
S31508008ED00878002801D059487047002070474FF499
S31508008EE08050091A56D0491E5BD0091F5BD0491E0F
S31508008EF05BD0891E5BD0491E5BD0491E5BD00C39FE
S31508008F005BD0491E5BD0491E5BD04FF4F470091A3A
S31508008F1059D0803959D04FF4C070091A57D0491E14
S31508008F2057D0491E57D0491E57D040F2FD10091A8E
S31508008F3055D0491E55D0491E55D0491E55D0091A37
S31508008F4055D0491E55D0491E55D0491E55D0091A27
S31508008F5055D0491E55D0491E55D0491E55D040F208
S31508008F60FD50091A53D0491E53D0491E53D0491EE5
S31508008F7053D0491E53D0491E53D040F6FA70091AE9
S31508008F8051D041F20100091A4FD04FF48050091A06
S31508008F904DD04EE0002000211160294901EBC000A8
S31508008FA070470120F7E70220F5E70320F3E70420DE
S31508008FB0F1E70520EFE70620EDE70720EBE70820B5
S31508008FC0E9E70920E7E70A20E5E70B20E3E70C20B5
S31508008FD0E1E70D20DFE70E20DDE70F20DBE71020B5
S31508008FE0D9E71120D7E71220D5E71320D3E71420B5
S31508008FF0D1E71520CFE71620CDE71720CBE71820B5
S31508009000C9E71920C7E71A20C5E71B20C3E71C20B4
S31508009010C1E71D20BFE71E20BDE71F20BBE72020B4
S31508009020B9E72120B7E72220B5E72320B3E72420B4
S31508009030B1E70448106000207047000030000906B8
S3150800904050A10108000002060CB430B583B00A46E8
S3150800905006A90291044600250194009502AB01A9D0
S31508009060084878441E3006F0D2FE019A157000288A
S315080090704EBF04460198041B204603B030BC5DF879
S315080090800CFB00BFF7D3FFFF13B5044608460028BC
S3150800909005D100221021204600F0C6FB03E001A9F5
S315080090A0204607F007FE204616BD70472DE9F8430F
S315080090B005460E46174699460898014611F0070FC9
S315080090C006D001F1080201F00708A2EB080800E043
S315080090D08846A8EB0101A9EB010909F00701A9EBEC
S315080090E0010900216961002801D1012000E0084634
S315080090F0099C85F83C00084685F8BC0002462421F0
S3150800910005F1180000F090FB2F63C5F82C90002C91
S3150800911001D10FF2C414AC61C5F828806E63BDE8AE
S31508009120F1831CB5049C0194009313460A4600215A
S31508009130FFF7BCFF13BD38B504460D4604F15400CD
S3150800914000F0BEFB6069002803D194F8BC00002833
S3150800915006D004F1540000F0D1FB6FF0030032BDD5
S31508009160A06A00280ED1E06A8008800007F0FCFE9D
S31508009170A062002806D16322DFF810110FF2401012
S3150800918000F0B4FA002005E0DFF80411A26A42F8FC
S315080091902010401CE16AB0EB910FF5D30022442160
S315080091A004F1780000F040FB4420606204F1780086
S315080091B020622946201D00F0EBFB04F11802214627
S315080091C00FF2D50008F02CFB6061002813D194F843
S315080091D03C00002804D0A06A07F0D6FE0020A06252
S315080091E004F1540000F08AFB04F14000FEF702FA8D
S315080091F06FF0020032BD04F1540000F07FFB00203E
S3150800920032BD70B50546002605F1540000F058FB3E
S315080092106C6905F14000FEF7EDF93046686195F88E
S31508009220BC00002808D1012085F8BC00002C03D01A
S31508009230204608F02FFB064605F1540000F05EFBB9
S31508009240304670BD80B5FEF7CDFD002002BD10B5D5
S315080092500446104820602046FFF7D3FF94F83C00E8
S31508009260002804D0A06A07F08FFE0020A06204F14F
S31508009270540000F063FB04F14000FEF7BEF9201D20
S31508009280FEF766F9204610BD000000004CC501082F
S31508009290A52E5AE2F8D0010810B50446201D08F09C
S315080092A025FB04F1540000F00BFB0020606101204F
S315080092B084F8BC0004F14000BDE81040FEF79AB9F6
S315080092C05F617474722E737461636B5F6D656D2074
S315080092D0213D204E554C4C006170706C6963617479
S315080092E0696F6E5F756E6E616D65645F74687265D1
S315080092F06164000010B5044608F0FAFA00202061FF
S31508009300204610BD1CB59DF8144001949DF81040E8
S31508009310009408F0EFFA16BDDFF838030068C0F3CA
S3150800932002207047EFF30580401E8041C043C00FFE
S315080093307047EFF31080002806D1EFF31180401E26
S315080093408041C043C00F70470120704738B5DFF829
S315080093500843FF20E070E07860F0FF00C043B0FAF1
S3150800936080F5C5F12005FFF7D7FFA84201D30546CA
S315080093706D1CFE2000FA05F5257031BDF8B5DFF83D
S31508009380DC52287A012801D10020F2BD002806D037
S315080093904FF0FF3008F0C0FA4FF0FF30F2BD05F18C
S315080093A05406DFF8BC72F868B060388A3080B8684E
S315080093B02864FC6A396B204608F0AFFA002800D00A
S315080093C0F4627C69B969204608F0A7FA002801D03A
S315080093D0346201E0F06A3062FC69396A204608F0B6
S315080093E09CFA002801D0746201E0F06A70627C6A17
S315080093F0B96A204608F091FA002801D0B46201E063
S31508009400F06AB0627C6B002C06D0E368A26821681B
S31508009410204608F0DFFA3463BC6B002C06D0E368FC
S31508009420A2682168204608F0D5FA7463FC6B002C04
S3150800943006D0E368A2682168204608F0CBFAB46330
S315080094403C6C002C06D0E368A2682168204608F028
S31508009450C1FAF4637C6C002C06D0E368A268216824
S31508009460204608F0B7FA3464BC6C002C06D0E368D2
S31508009470A2682168204608F0ADFA7464FC6C002CDA
S3150800948006D0E368A2682168204608F0A3FAB46407
S315080094903C6D002C06D0E368A2682168204608F0D7
S315080094A099FAF464012028720020F2BD38B5DFF875
S315080094B0AC41207A012806D06FF0060008F02CFA95
S315080094C04FF0FF3032BD08F085F900280AD0FFF7C3
S315080094D03DFFDFF88C51DFF88C11686808F0C0FA98
S315080094E0002806D04FF0FF3008F016FA4FF0FF308C
S315080094F032BD08F0D9FA206108F0DAFA04F11C0046
S3150800950007F0DCFD07F0EBFE2878C00703D502203C
S3150800951080F3148802E0032080F314880220207266
S31508009520002032BD80B5DFF83401017A022902D065
S31508009530032904D005E003210172002002BD0120A1
S3150800954002BD4FF0FF3008F0E7F94FF0FF3002BDDB
S3150800955080B5DFF808110A7A921E012A0CD800286D
S3150800956002D0012804D007E002200872002002BDBC
S3150800957003200872012002BD4FF0FF3008F0CCF935
S315080095804FF0FF3002BD38B504460D4608F0A6FA7E
S3150800959029462046BDE8344008F0ACBA10B508F0B4
S315080095A017FBFFF7BFFE002803D1FFF7C2FE00280E
S315080095B005D06FF00504204608F0AEF903E02A4806
S315080095C0844600DF0446204610BD000010B5FFF7AC
S315080095D0A9FE002803D1FFF7ACFE002805D06FF0DE
S315080095E00504204608F098F903E02048844600DF81
S315080095F00446204610BD000010B5FFF793FE00286C
S3150800960003D1FFF796FE002805D06FF00504204623
S3150800961008F082F903E01648844600DF044620462F
S3150800962010BD000010B50446FFF77CFE002803D1E4
S31508009630FFF77FFE002805D06FF00504204608F0E6
S315080096406BF904E00B488446204600DF04462046B2
S3150800965010BD00000CED00E01FED00E0241A00200C
S3150800966018BE0108A5B301087D930008AD9400084B
S3150800967025950008519500085254582056352E3520
S315080096802E33000080B508F0A4FAC0F1400002BDF0
S31508009690B0F8001501EB810200EB8200704710B5A7
S315080096A00446087B2073887BA073487B6073086830
S315080096B020600A7B091D201DFCF79CFE204610BD74
S315080096C0B0F80025891801F03F01A0F80015704789
S315080096D080B508F08CFA72B603494A78012A02D096
S315080096E008700120487001BD3640002082B00B4644
S315080096F0009200220146024800F0E0FEFEE700BFA5
S315080097004401FF8080B508F072FA002804D036229A
S3150800971005490648FFF7EAFF054800214170007829
S31508009720012800D162B601BD64C101087CCC0108DC
S315080097303640002080B508F08AFA002002BD10B530
S315080097400F4C1048006800280CD000F0E1FE01F02C
S315080097502EF921680818002121604FF47A71B0FBB0
S31508009760F1F010BD08F0BFFA61682268821A92B259
S315080097705118616020604FF47A70B1FBF0F010BDAB
S31508009780843F0020D03F002038B504460D46AC4241
S3150800979005D0206820188047241DAC42F9D131BD78
S315080097A0F8B505460E46174608F0F2FA1A4908684B
S315080097B000B91A481A4A90422EBF002404460C30B3
S315080097C0086008F0EEFA0CB90120F2BD2660656063
S315080097D0A7600020F2BD80B50F49124800F001F8D5
S315080097E001BDF8B50E46054637683C0004D1F1BD03
S315080097F088470DE007463C46AC42F8D00C3C616809
S315080098000800F9D02068002200286260F0D0884756
S3150800981030688742F0D0EDE7E43F00205C40002046
S31508009820D84200205C40002062F30F2262F31F42F8
S3150800983000B500BF130096469446103928BFA0E825
S315080098400C50FAD85FEA417C28BF0CC048BF40F8E4
S31508009850042BC90728BF20F8022B48BF00F8012BA4
S3150800986000BD704710B50446002020620146204618
S3150800987000F002F8204610BD38B584B005460C46FF
S315080098806846102100F022FC002C00D139A400946F
S31508009890281D02901C2003900B200190684608F0B2
S315080098A0C3FC2860002809D108F066FD002805D108
S315080098B01F48352200F12401FFF718FF05B030BD17
S315080098C038B505464FF0FF31286808F0C3FC040098
S315080098D002D1286A401C2862002C0DD008F04CFDE5
S315080098E0002809D1002000900346224617A11148F6
S315080098F000F0E4FD204632BD002032BD38B50546ED
S31508009900286808F0C1FC040002D1286A401E2862B3
S31508009910002C0BD008F030FD002807D1002000905D
S31508009920034622460EA1044800F0C8FD204632BD73
S31508009930F4BE0108150102801701028010B504461D
S31508009940206808F0B9FC204610BD00004D75746506
S3150800995078206C6F636B206661696C656400000033
S315080099604D7574657820756E6C6F636B20666169DA
S315080099706C6564006170706C69636174696F6E5FB1
S31508009980756E6E616D65645F6D757465780000004F
S3150800999038B504460D46AC420AD0FDF7D9FD214636
S315080099A0102001F0EAF8002802D0294608F01AFE2D
S315080099B0204632BD010008D4012200F01F018A406A
S315080099C0DFF8F015400941F820207047DFF8E82550
S315080099D01268103002EB80021160704710B5044619
S315080099E008F012FE002805D00FF21460BDE81040FA
S315080099F008F024BFA16C204600F0E7F8012805D03E
S31508009A000FF21460BDE8104008F018BF10BD2DE92C
S31508009A10FC4781460C4615461E46DFF8A0753946B2
S31508009A20204608F07FFF8246DFF89485414628469F
S31508009A3008F078FF0146504608F04EFF10F1010F76
S31508009A4007D140F22922DFF87C150FF2EC50FFF718
S31508009A504DFEDFF87415884254D1DFF870050168A9
S31508009A6041F000710160006800F0007000900098F5
S31508009A700020C9F844003946204608F009FF414647
S31508009A80284608F005FF20464FF0FF31884202D0ED
S31508009A90012109F037F928464FF0FF31884202D0F4
S31508009AA0012109F02FF9DFF82005C9F80000002088
S31508009AB0C9F818000120C9F81C00C9F820000020C0
S31508009AC0C9F82400C9F82800C9F82C00C9F8080004
S31508009AD0C9F80C004FF4A020C9F810004FF4E000B4
S31508009AE0C9F814000220C9F80400C9F848604846B5
S31508009AF0FFF774FF002000900346024601464846D9
S31508009B0000F060F9BDE8F387DFF8C4345960406CAB
S31508009B1043F82020704702685369DFF8B8140B40F1
S31508009B2053610021DFF8A824406C42F820107047E2
S31508009B300068DFF8941488420DD1DFF89C040168A8
S31508009B4041F000710160016821F000710160C1688F
S31508009B5021F00071C160704770B40B460021B0FB5C
S31508009B60F3F01823B0FBF3F39BB207E0641E002C56
S31508009B7004DDE51C75438542F8D10121002907D18A
S31508009B80B3EB900F04D25B1C9BB216245E1CEEE767
S31508009B90002915D0DFF8440400EBC401496809051B
S31508009BA001F4E00150F83400000400F47020014389
S31508009BB0120602F040720A43C3F309031A4301E08E
S31508009BC04FF0FF32104670BC70472DE9F04107464A
S31508009BD08846FDF709FB01224146FFF7BDFF064609
S31508009BE03D680124C7F84880002E3ADD286840F011
S31508009BF001002860FFF7A3FD07466868C00705D47B
S31508009C00FFF79DFDC01B0328F7D30024002C23D0A3
S31508009C10E969DFF8CC030140E961E8690643EE61CA
S31508009C202868400840002860FFF789FD06466868EE
S31508009C30C00705D5FFF783FD801B0328F7D300244B
S31508009C40002C0FD1AA69002392B2A969090CDFF882
S31508009C50940308F0F3FD05E00FF2EC3008F0EEFD92
S31508009C6000E000242046BDE8F0810EB40068816853
S31508009C70490116D5002100EB011000F5C0710868EE
S31508009C8000F0010008609DF80E209DF80D000028E0
S31508009C900868009B11D140EA435050EA42020A6024
S31508009CA012E08168090101D50121E4E78168C9004C
S31508009CB001D50221DFE7002034E040EAC30050EA7C
S31508009CC0420242F004020A6048680009000148603E
S31508009CD048689DF80C2002F00F02104348609DF872
S31508009CE007009DF80620120442EA00629DF8050066
S31508009CF042EA00229DF8040002438A609DF80B00A0
S31508009D009DF80A20120442EA00629DF8090042EA18
S31508009D1000229DF808000243CA60086840F0010066
S31508009D200860012003B0704710B40068C36813F0D8
S31508009D30030F01D1002039E000EB021303F5D873B5
S31508009D401C68C4F380044C73002C1C6802D1640D93
S31508009D500C6001E0E4080C601C68C4F340048C73D2
S31508009D605C6804F00F040C739C680C719C68240AE8
S31508009D704C719C68240C8C719C68240ECC71DC6830
S31508009D800C72DC68240A4C72DC68240C8C72DB6862
S31508009D901B0ECB72002A04D1C16841F02001C160B4
S31508009DA003E0016941F020010161012010BC704700
S31508009DB000688069000E704700688069000CC0B2B0
S31508009DC07047000038B58AB01C0001D0012C28D194
S31508009DD00E9C05940025069501250795002B07D1AD
S31508009DE049010091002101915201029203910FE06D
S31508009DF00B465B0B0093C90089B241F0040101913F
S31508009E001146490B0291D20092B242F00402039223
S31508009E1000210491294608910E340994694608F0F0
S31508009E208AFC01200BB030BDF8B507460E46002067
S31508009E30014602467B69DB0728D56B4BBC681C408C
S31508009E409C4200D10120694BBC681C409C4200D151
S31508009E500121674BBC681C409C4200D101220028A6
S31508009E6001D00123BB60002902D04FF48073BB6088
S31508009E70002A02D04FF48033BB600843104305D054
S31508009E80534A012152F8260052689047F96801F0B2
S31508009E9003017869400800F00100002907D000286E
S31508009EA005D04B4A002152F8260052689047BA69F5
S31508009EB0520802F001027969490A01F0010178693C
S31508009EC0C00B00F00100002A09D0002907D000289D
S31508009ED005D03F4A052152F8260052689047BD69C9
S31508009EE0AD0805F001057C69A40A04F00104786947
S31508009EF0C00B00F00100002D09D0002C07D0002867
S31508009F0005D0334A072152F82600526890477869E7
S31508009F10C00B00F00100002D0BD0002C09D0002842
S31508009F2007D02B4A022152F826005268BDE8F840AD
S31508009F301047F1BD0021244876E70021224873E73F
S31508009F400021214870E7000000681F4B984200D0A6
S31508009F50704710B5072915D8DFE801F0041519145C
S31508009F60141E1423022314242249002A42691DD1EF
S31508009F7022EA030343612046FFF728FD2046BDE891
S31508009F80104017E510BD012313241B49EDE74FF4D4
S31508009F90004316241949E8E74FF4007316241749B5
S31508009FA0E3E74FF4806316241449DEE7134343615D
S31508009FB0E1E7000000E100E008ED00E004CB01085D
S31508009FC028CB010868C00108006400401C10024044
S31508009FD07C3F0020EC79FFFF1010024048B00108D2
S31508009FE000FC80FC6CC9010801000004000100089F
S31508009FF000000110359F00083B9F0008419F00089C
S3150800A00043616E6E6F7420696E697469616C697AF2
S3150800A010652043414E00000043616E2066726571FB
S3150800A02075656E637920636F756C64206E6F742036
S3150800A0306265207365740A0028696E742963616E07
S3150800A04020213D204E43000063616E20696E6974CD
S3150800A05020726571756573742074696D656F7574A2
S3150800A0600A000000C068002801D0012070470020BF
S3150800A070704770477047010680B5C168002905D149
S3150800A08040F23B2203490448FFF730FB0968BDE864
S3150800A09004400847E8C30108B0D301081FB50446C1
S3150800A0A0684608F08BFE0146204608F08BFE2046DF
S3150800A0B004B010BD1FB50446684608F099FE01466F
S3150800A0C0204608F099FE204604B010BD0022FFF78E
S3150800A0D0AFBB0401EFF30580401E8041C043C00FAB
S3150800A0E07047EFF31080002806D1EFF31180401E69
S3150800A0F08041C043C00F70470120704710B4024624
S3150800A100D2E85F0F814202D8BFF32F8F04E0431CC9
S3150800A110C2E8543F04B1F3E780B210BC70470000B0
S3150800A1200146D1E85F0F10B9BFF32F8F04E0421E36
S3150800A130C1E8532F03B1F4E780B270477047704700
S3150800A140DFF85C034069704780B50C30FFF7E8FF1D
S3150800A150401E8041C043C00F02BD10B50446E189C8
S3150800A16004F10C00FFF7CAFF0146E28991428041DB
S3150800A170C00F10BD10B50446A06800280FD02046B1
S3150800A180FFF7E2FF00280AD02046FFF7D8FF06F0BF
S3150800A19095FF00221146BDE8104007F0DBB810BD58
S3150800A1A0F8B505460F46002D04D0B5F5803F01D217
S3150800A1B0BD4206D26FF00301002008F033FE0020EE
S3150800A1C0F2BD002A14D016689468002C06D014F044
S3150800A1D0030006D1D06810280CD202E0D068002807
S3150800A1E008D06FF00801002008F01CFE0020F2BD20
S3150800A1F000263446002C11D1A94BD3F89800002824
S3150800A20003D007F007FC044606E001221021D3F824
S3150800A210800008F008FE0446012000E00020002C1B
S3150800A2200BD0F6212170A07066600020A060A7817F
S3150800A230E5819C489A49886604E06FF0040100208D
S3150800A24008F0F0FD2046F2BD38B50C46FFF776FF5C
S3150800A250050002D02878F62807D06FF003042146B7
S3150800A260284608F0DFFD204632BD2846FFF76CFF7A
S3150800A270002801D0002032BD002C11D021466320D1
S3150800A28007F07BF8002808D0FFF75AFF044628464F
S3150800A290FFF755FF214606F0FAFE6FF0010032BDC2
S3150800A2A06FF0020032BD38B5FFF748FF040002D050
S3150800A2B02078F62807D06FF003052946204608F0CF
S3150800A2C0B1FD284632BDA0680028204609D0FFF710
S3150800A2D036FF06F0F3FE0122002107F03BF80020C6
S3150800A2E032BDFFF73AFF002801D0002032BD6FF0DB
S3150800A2F01001204608F096FD6FF0020032BD38B511
S3150800A300FFF71CFF040002D02078F62807D06FF06C
S3150800A31003052946204608F085FD284632BDA06873
S3150800A32000280FD02046FFF70AFF06F0C7FE0022D6
S3150800A3306FF0020107F00EF8A0680028F2D100209D
S3150800A34006F0D3FF00202070A078C0070AD5564A29
S3150800A35090690028214602D007F06CFB02E01068DD
S3150800A36008F0BEFD002032BD10B50C46FFF7E6FE2C
S3150800A370002804D00178F62901D1002C06D06FF008
S3150800A3800304214608F04EFD204610BDFFF7DCFE0B
S3150800A390002801D0002010BD6FF0020010BD38B5AE
S3150800A3A0FFF7CCFE040002D02078F62807D06FF01D
S3150800A3B003052946204608F035FD284632BD2046C5
S3150800A3C0FFF7CBFE002806D02046FFF7B8FE08F0B8
S3150800A3D096FE002032BD6FF01001204608F022FDDF
S3150800A3E06FF0020032BD000070B504460D461646F1
S3150800A3F0FFF770FE002803D1FFF773FE002806D08A
S3150800A4006FF00501002008F00DFD002070BD2748FB
S3150800A410844632462946204600DF70BD38B50446D4
S3150800A4200D46FFF757FE002803D1FFF75AFE00280E
S3150800A43004D029462046BDE8344095E71C488446A2
S3150800A4402946204600DF32BD10B50446FFF742FE16
S3150800A450002803D1FFF745FE002803D02046BDE8B3
S3150800A46010409CE713488446204600DF10BD0000D4
S3150800A47038B50446FFF72EFE002803D1FFF731FE54
S3150800A480002806D06FF005052946204608F0CAFCC4
S3150800A49004E009488446204600DF0546284632BDC2
S3150800A4A0241A002075A10008A41A0020A1A10008FA
S3150800A4B049A20008A7A20008FFA200082DE9F84350
S3150800A4C004460D4616461F46DFF8409001214846C9
S3150800A4D008F030FE002816D1DDF820800020009014
S3150800A4E043463A463146204607F00AFF43463A466F
S3150800A4F0294609F13C0007F049FF00214846BDE816
S3150800A500F44308F017BEBDE8F28300BF9827002081
S3150800A51005A0704703480168002901D002A0084732
S3150800A52070470000EC180020E0CA0108103D002022
S3150800A5302DE9F8430546686800F1380108780028CF
S3150800A54070D1887800286DD1286800688047286807
S3150800A550C06980470468002C04D12D22C64993A0FF
S3150800A560FFF7C4F84FF000081F2100E0491E0A460D
S3150800A570D2B2002A04D001228A40A242F6D18846E5
S3150800A58040680746001F1D2804D33B22BA4987A006
S3150800A590FFF7ACF8072007F1FC0600FA06F60020DC
S3150800A5A0696808606968486028684068804769681B
S3150800A5B00862002001466A68C2E90A016868846080
S3150800A5C0686880F83B8001203A4608F0BBFD401ECB
S3150800A5D06968C8606868066122460023A7489046ED
S3150800A5E09946E0FB0689B8F1010069F1000108F017
S3150800A5F0BBFD6A68C2E90601002001466A68C2E92D
S3150800A6000C01696881F83900696881F83A00012007
S3150800A610696881F83800284600F009F82846BDE838
S3150800A620F243D8E0BDE8F1834068016070472DE940
S3150800A630F84F0646746804F13A052878002866D16A
S3150800A6403068406880477168096A88425FD0266A20
S3150800A650861BE1680E4000272062D4F808808748E8
S3150800A66080454ED06D7802463B46A2FB0601002D7A
S3150800A6701FD0804689462A4608F08EFE06460F46B3
S3150800A680D4E90A0110EB080841EB090930463946B6
S3150800A6902A4608F057FDB8EB000269EB0103C4E946
S3150800A6A00A23A06800218B422BD31FD8824228D3C5
S3150800A6B01CE082468B46424608F056FD06460F4683
S3150800A6C0D4E90A0110EB0A0041EB0B01A8FB0623AB
S3150800A6D008FB0733821A61EB0303C4E90A23A0685F
S3150800A6E000218B420DD301D882420AD3761C67F12A
S3150800A6F0FF37D4E90A23A068101A63EB0101C4E9FD
S3150800A7000A01D4E90C0180197941C4E90C01BDE8B4
S3150800A710F18F2DE9F0470746796801F10806D6E971
S3150800A7200A45121BAB41D1F810A05046D1E906459F
S3150800A7309D4234D301D8944231D330684F4CA0425D
S3150800A74004D1504690422AD9104628E091F83BC0D9
S3150800A7504B4C0025BCF1000F10D010461946624636
S3150800A76008F0F0FC00196941444A2B4608F0FCFC45
S3150800A77002465046904212D9104610E0A0FB0289C4
S3150800A78000FB039918EB040049EB05013B4A2B46ED
S3150800A79008F0EAFC02465046904200D91046B169D4
S3150800A7A0401871680840BDE8F087000030000000D6
S3150800A7B0904207D2914203D281428041C00F70472E
S3150800A7C001207047814204D291428041C043C00FA4
S3150800A7D0704700207047F8B5044661680D4695F83D
S3150800A7E03A00002846D191F83900002842D120467F
S3150800A7F0FFF71DFF6168486800282FD0D0E90023BD
S3150800A800D1E90C679F4207D301D8964204D3206842
S3150800A8104069BDE8F24000472046FFF77AFF064642
S3150800A8200C356869864206D113494FF4847201F1E2
S3150800A8304C00FEF75BFF30462168096988472068A7
S3150800A84040688047324601466869FFF7B1FF00282D
S3150800A85010D020684069BDE8F240004705F10C02B7
S3150800A8605069516808181168084021680969BDE8E7
S3150800A870F4400847F1BD0000A8BD010840420F009A
S3150800A8803F420F0038B504460D46FFF751FEFCF768
S3150800A8902BFA29462046FFF7C7FEBDE83140FCF7EC
S3150800A8A034BA2DE9D0430446FCF71EFA2068C0687E
S3150800A8B08047606800F139014878002803D0BDE870
S3150800A8C0D043FCF722BA0120087007E0D16841603E
S3150800A8D060680168002901D0906888476068406808
S3150800A8E000280DD02046FFF7A2FE60684268D0E92E
S3150800A8F00C67D2E900894F45E8D801D34645E5D229
S3150800A9000020616881F839002046FFF764FFBDE83A
S3150800A910D043FCF7FAB92DE9F04106460F4614462E
S3150800A9201D46DDF81880FCF7DFF93046FFF77FFE95
S3150800A930C7E90045C7F8088000217068406801E04B
S3150800A9400146C068002806D0D0E900239D42F7D802
S3150800A95001D39442F4D2F860002905D170684760A3
S3150800A9603046FFF738FF00E0CF60BDE8F041FCF75E
S3150800A970CCB938B504460D46FCF7B6F9616848689F
S3150800A980A84206D1E86848602046FFF724FF07E09A
S3150800A9900846002804D0C168A942F9D1E968C1600F
S3150800A9A0BDE83140FCF7B1B90000000000BF38B57A
S3150800A9B00446FFF7BDFDFCF797F92046FFF737FE7B
S3150800A9C06068D0E90C45FCF7A0F92046294634BD55
S3150800A9D0A9B1B1FA81F241409040C2F1200261FA70
S3150800A9E002F181EA000018BF40F0010002F19D0162
S3150800A9F0C905020672F1004241EB1020704750B1BA
S3150800AA00B0FA80F29040C2F19D02D205010671F1BA
S3150800AA10004142EB102070474FF0FF0C1CEAD05360
S3150800AA201DBF1CEAD1526345624543E09B1A5FEAA3
S3150800AA30CC7280EA010C42EA01211CEA020C42EAC5
S3150800AA400020421A38BF01EB420253F17E034FEA57
S3150800AA501121B2FBF1F001FB102260F3D63C4FEA5C
S3150800AA600222B2FBF1F001FB102260F3CE1C4FEA82
S3150800AA700222B2FBF1F006DDFF2B29DA5CEA500070
S3150800AA8040EBC3507047C3F1020301FB1022192B98
S3150800AA9040EA4C010CF0004C41F0807121DC21FAAF
S3150800AAA003F0C3F120039940114371F1004250EBC2
S3150800AAB00C00704763451ABF0CEAD152624512E092
S3150800AAC080EA010C00180CF0004C06D049181AD17F
S3150800AAD00CF0004C4CF0FF407047C94208BF6FEAC3
S3150800AAE0020C60467047634506D1B2EB0C02F5D0FE
S3150800AAF001F00041484070474A0212BF08464840E4
S3150800AB0000F0004070474AB90902B1FA81F2914053
S3150800AB1043B19B18C00140F0004092E7C90141F0DB
S3150800AB20004152420002B0FA80F39840D31A88E7EF
S3150800AB304FF6FF710180704710B40288054B144622
S3150800AB4081EA242133F8111081EA0221018010BC20
S3150800AB50704700001498010870B504460D4616465D
S3150800AB6004E015F8011B2046FFF7E6FF3046461EAF
S3150800AB7080B20028F5D170BD7047084670470804B2
S3150800AB8010B50446012103F069FCDFF8680C206063
S3150800AB9004F58170002101704170204610BD7CB516
S3150800ABA004460D4604F10C01684608F004FC2878B2
S3150800ABB0698840EA0120216B4140616320630221D4
S3150800ABC0204603F002FD002816D004F581760221FE
S3150800ABD0204603F0E6FC002807D001203070707884
S3150800ABE0002809D00020707006E0012070703078C7
S3150800ABF0002801D000203070B5F9040008F0E4FB05
S3150800AC00DFF8F41BFFF708FF206595F9060008F042
S3150800AC10DBFB606595F9070008F0D6FBA06504F133
S3150800AC205C063078297A884201D0012000E00020AD
S3150800AC307070287A3070652801DB64203070688966
S3150800AC4008F0D4FBDFF8B01BFFF7E6FE7060A16BD7
S3150800AC50E8684140E163E868A063216C28694140DF
S3150800AC60616428692064A16C68694140E164686987
S3150800AC70A064684608F0C7FB73BD102103F0D0BC7A
S3150800AC801CB5044604F10C01684608F094FB94F8D8
S3150800AC900241684608F0B7FB204616BD1CB50446B7
S3150800ACA004F10C01684608F086FB002084F80201CE
S3150800ACB0684608F0A8FB13BD1CB5044604F10C0150
S3150800ACC0684608F078FB94F80341684608F09BFB51
S3150800ACD0204616BD1CB5044604F10C01684608F06A
S3150800ACE06AFB002084F80301684608F08CFB13BD54
S3150800ACF01046012971D0022974D0042977D0082971
S3150800AD007AD010297DD0202900F08080402900F0D3
S3150800AD108280802900F08480B1F5807F00F08580EC
S3150800AD20B1F5007F00F08680B1F5806F00F087806E
S3150800AD30B1F5006F00F08880B1F5805F00F089807A
S3150800AD40B1F5005F00F08A80B1F5804F00F08B8086
S3150800AD50B1F5004F00F08C80B1F5803F00F08D8092
S3150800AD60B1F5003F00F08E80B1F5802F00F08F809E
S3150800AD70B1F5002F00F09080B1F5801F00F09180AA
S3150800AD80B1F5001F00F09280B1F5800F00F09380B6
S3150800AD90B1F5000F00F09480B1F1807F00F0958046
S3150800ADA0B1F1007F00F09680B1F1806F00F09780D6
S3150800ADB0B1F1006F00F09880B1F1805F00F09980E2
S3150800ADC0B1F1005F00F09A80B1F1804F00F09B80EE
S3150800ADD0B1F1004F00F09B809DE00C220FF24C1160
S3150800ADE0FBF7F8BA0D220FF25011FBF7F3BA0C2253
S3150800ADF00FF25411FBF7EEBA0E220FF25811FBF7B9
S3150800AE00E9BA0F220FF25C11FBF7E4BA0E22DFF85B
S3150800AE10D41BFBF7DFBA0E220FF25811FBF7DABA8A
S3150800AE2006220FF26011FBF7D5BA10220FF25C1159
S3150800AE30FBF7D0BA0E220FF26411FBF7CBBA0F223A
S3150800AE400FF26811FBF7C6BA0C220FF27011FBF766
S3150800AE50C1BA0B220FF27011FBF7BCBA0C220FF223
S3150800AE607411FBF7B7BA09220FF27411FBF7B2BADD
S3150800AE7010220FF27811FBF7ADBA0E220FF27C11F1
S3150800AE80FBF7A8BA10220FF28411FBF7A3BA0C221B
S3150800AE900FF28811FBF79EBA0A220FF28C11FBF704
S3150800AEA099BA0F220FF28C11FBF794BA0F220FF200
S3150800AEB09411FBF78FBA10220FF29811FBF78ABA92
S3150800AEC00E220FF2A011FBF785BA0C220FF2A4117D
S3150800AED0FBF780BA0E220FF2A811FBF77BBA0A22FB
S3150800AEE00FF2AC11FBF776BA0F220FF2B011FBF78F
S3150800AEF071BA0E220FF2B411FBF76CBA0F220FF2D9
S3150800AF00BC11FBF767BA042206A1FBF763BA042251
S3150800AF1005A1FBF75FBA0822DFF8781CFBF75ABAD7
S3150800AF200000000045333000453331004F76657226
S3150800AF3063757272656E7400556E646572766F6CB1
S3150800AF4074616765000000004F766572766F6C74F1
S3150800AF50616765004C6F772074656D702E204443D9
S3150800AF6048000000486967682074656D702E2044A3
S3150800AF7043480000486967682068756D69646974A4
S3150800AF8079000000576174657200000048692E2038
S3150800AF904C6F6769632074656D702E004C6F676926
S3150800AFA063206F66666C696E65000000437269749B
S3150800AFB06963616C206572726F72000043726F7705
S3150800AFC06E206572726F720043656C6C20636F75D4
S3150800AFD06E740000485947206F66666C696E650096
S3150800AFE04E6565642041434B00000000436F6D6267
S3150800AFF0696C696674206F66666C2E0053686F729A
S3150800B00074206369726375697400000048692E20AC
S3150800B010636F6E742E2074656D702E004C6F6769B1
S3150800B0206320636F756E7400414443206572726FC6
S3150800B0307200000043757272656E742073656E73D4
S3150800B0406F720000434820636F6E742E2063796325
S3150800B0506C65000044434820636F6E742E20637944
S3150800B060636C65005368756E74206F66666C696EEE
S3150800B070650000005368756E74206572726F720001
S3150800B08053657474696E6773206572722E000000CA
S3150800B0905744542072657365740000004E6F20741F
S3150800B0A0656D702E2073656E732E000053686F727F
S3150800B0B07465642074656D702E00000053706972A3
S3150800B0C06974206F66666C696E6500001046012912
S3150800B0D056D0022958D004295AD008295CD01029FC
S3150800B0E05ED0202960D0402962D0802964D0B1F58D
S3150800B0F0807F65D0B1F5007F66D0B1F5806F67D0E7
S3150800B100B1F5006F68D0B1F5805F69D0B1F5005F21
S3150800B1106AD0B1F5804F6BD0B1F5004F6CD0B1F560
S3150800B120803F6DD0B1F5003F6ED0B1F5802F6FD05E
S3150800B130B1F5002F70D0B1F5801F71D0B1F5001FA1
S3150800B14072D0B1F5800F73D0B1F5000F74D0B1F19C
S3150800B150807F75D0B1F1007F76D0B1F1806F77D05E
S3150800B160B1F1006F78D0B1F1805F79D0B1F1005FAD
S3150800B1707AD0B1F1804F7BD0B1F1004F7CD07FE01F
S3150800B180032241A1FBF726B9032240A1FBF722B906
S3150800B19003223FA1FBF71EB904223EA1FBF71AB909
S3150800B1A004223DA1FBF716B904223CA1FBF712B90C
S3150800B1B004223BA1FBF70EB904223AA1FBF70AB910
S3150800B1C0042239A1FBF706B9042238A1FBF702B914
S3150800B1D0042237A1FBF7FEB8042236A1FBF7FAB81A
S3150800B1E0042235A1FBF7F6B8042234A1FBF7F2B81E
S3150800B1F0042233A1FBF7EEB8042232A1FBF7EAB822
S3150800B200042231A1FBF7E6B80422B7A1FBF7E2B89E
S3150800B2100422B6A1FBF7DEB80422B5A1FBF7DAB81B
S3150800B2200422B4A1FBF7D6B80422B3A1FBF7D2B81F
S3150800B2300422B2A1FBF7CEB80422B1A1FBF7CAB823
S3150800B2400422B0A1FBF7C6B80422AFA1FBF7C2B827
S3150800B2500422AEA1FBF7BEB80422ADA1FBF7BAB82B
S3150800B2600422ACA1FBF7B6B80422ABA1FBF7B2B82F
S3150800B2700422AAA1FBF7AEB80422A9A1FBF7AAB833
S3150800B2800422A8A1FBF7A6B84F43000055560000B4
S3150800B2904F5600004C54440048544400424345006D
S3150800B2A04848550057485500484C54004C4F4600EE
S3150800B2B04345520043524F0043454C004859470006
S3150800B2C041434B00434F4D00534843001046012964
S3150800B2D071D0022974D0042977D008297AD0102988
S3150800B2E07DD0202900F08080402900F082808029C6
S3150800B2F000F08480B1F5807F00F08580B1F5007F8D
S3150800B30000F08680B1F5806F00F08780B1F5006F98
S3150800B31000F08880B1F5805F00F08980B1F5005FA4
S3150800B32000F08A80B1F5804F00F08B80B1F5004FB0
S3150800B33000F08C80B1F5803F00F08D80B1F5003FBC
S3150800B34000F08E80B1F5802F00F08F80B1F5002FC8
S3150800B35000F09080B1F5801F00F09180B1F5001FD4
S3150800B36000F09180B1F5800F00F09180B1F5000FE3
S3150800B37000F09180B1F1807F00F09180B1F1007FFB
S3150800B38000F09180B1F1806F00F09180B1F1006F0B
S3150800B39000F09180B1F1805F00F09180B1F1005F1B
S3150800B3A000F09180B1F1804F00F09180B1F1004F2B
S3150800B3B000F0918093E00D220FF29C11FBF70AB87A
S3150800B3C00E220FF2A411FBF705B80C220FF2A811F2
S3150800B3D0FBF700B809220FF2AC11FAF7FBBF0F22F0
S3150800B3E00FF2AC11FAF7F6BF10220FF2B411FAF702
S3150800B3F0F1BF0F220FF2FC51FAF7ECBF10220FF241
S3150800B4000461FAF7E7BF11220FF2A411FAF7E2BFB7
S3150800B41010220FF20061FAF7DDBF10220FF2046165
S3150800B420FAF7D8BF11220FF20C61FAF7D3BF102230
S3150800B4300FF29011FAF7CEBF0E220FF29811FAF713
S3150800B440C9BF09220FF29C11FAF7C4BF0A220FF2EC
S3150800B450A011FAF7BFBF0B220FF2A011FAF7BABF75
S3150800B46010220FF2A411FAF7B5BF0C220FF2A81199
S3150800B470FAF7B0BF11220FF2AC11FAF7ABBF0422EC
S3150800B48029A1FAF7A7BF042228A1FAF7A3BF042225
S3150800B49027A1FAF79FBF042226A1FAF79BBF042229
S3150800B4A025A1FAF797BF042224A1FAF793BF04222D
S3150800B4B023A1FAF78FBF042222A1FAF78BBF042231
S3150800B4C021A1FAF787BF042220A1FAF783BF042235
S3150800B4D01FA1FAF77FBF04221EA1FAF77BBF082235
S3150800B4E0DFF8B016FAF776BF484354004C4F4700CA
S3150800B4F04144430043534500434343004443430008
S3150800B50053484F0053484500534554005744540088
S3150800B5104E5453005453530053504900453330009A
S3150800B52045333100554B4E0045353200453533001D
S3150800B530453534004535350045353600453537003F
S3150800B5404535380045353900453630004536310031
S3150800B55045363200453633004C6F772074656D707A
S3150800B5602E20434800000000486967682074656D0E
S3150800B570702E2043480000004D6F756E742065726A
S3150800B580726F72004653206572726F720000000077
S3150800B590556E616C6C6F7761626C6520434800007C
S3150800B5A0537475636B20636F6E746163746F720096
S3150800B5B0496E73756C6174696F6E206661756C741B
S3150800B5C000000000436F6E742E20666565642E20A9
S3150800B5D065722E0047656E6572616C206572726FC2
S3150800B5E0720000004856206661756C740000000001
S3150800B5F0505357206572726F720000004856494CC6
S3150800B600206572726F7200005072656368617267B6
S3150800B61065206572726F7200506F77657220666179
S3150800B620756C74004375722E206C696D697420659B
S3150800B63072726F72000000001046012956D0022966
S3150800B64058D004295AD008295CD010295ED0202960
S3150800B65060D0402962D0802964D0B1F5807F65D05A
S3150800B660B1F5007F66D0B1F5806F67D0B1F5006F90
S3150800B67068D0B1F5805F69D0B1F5005F6AD0B1F5E1
S3150800B680804F6BD0B1F5004F6CD0B1F5803F6DD0CF
S3150800B690B1F5003F6ED0B1F5802F6FD0B1F5002F10
S3150800B6A070D0B1F5801F71D0B1F5001F72D0B1F519
S3150800B6B0800F73D0B1F5000F74D0B1F1807F75D0CB
S3150800B6C0B1F1007F76D0B1F1806F77D0B1F1006F1C
S3150800B6D078D0B1F1805F79D0B1F1005F7AD0B1F15D
S3150800B6E0804F7BD0B1F1004F7CD07FE004229FA130
S3150800B6F0FAF770BE04229EA1FAF76CBE04229DA139
S3150800B700FAF768BE04229CA1FAF764BE04229BA13C
S3150800B710FAF760BE04229AA1FAF75CBE042299A140
S3150800B720FAF758BE042298A1FAF754BE042297A144
S3150800B730FAF750BE042296A1FAF74CBE042295A148
S3150800B740FAF748BE042294A1FAF744BE042293A14C
S3150800B750FAF740BE032292A1FAF73CBE042291A151
S3150800B760FAF738BE042290A1FAF734BE03228FA155
S3150800B770FAF730BE03228EA1FAF72CBE03228DA15A
S3150800B780FAF728BE04228CA1FAF724BE04228BA15C
S3150800B790FAF720BE04228AA1FAF71CBE042289A160
S3150800B7A0FAF718BE042288A1FAF714BE042287A164
S3150800B7B0FAF710BE042286A1FAF70CBE042285A168
S3150800B7C0FAF708BE042284A1FAF704BE042283A16C
S3150800B7D0FAF700BE042282A1FAF7FCBD042282A170
S3150800B7E0FAF7F8BD042281A1FAF7F4BD042280A174
S3150800B7F0FAF7F0BDC0BF0108000020411046012934
S3150800B8003ED0022941D0042944D0082947D010291E
S3150800B8104AD020294DD040294FD0802951D0B1F5A2
S3150800B820807F53D0B1F5007F55D0B1F5806F57D0E2
S3150800B830B1F5006F59D0B1F5805F5AD0B1F5005F08
S3150800B8405BD0B1F5804F5CD0B1F5004F5ED0B1F555
S3150800B850803F60D0B1F5003F62D0B1F5802F64D04B
S3150800B860B1F5002F66D0B1F5801F68D0B1F5001F7D
S3150800B8706AD0B1F5800F6CD0B1F5000F6DD070E0CD
S3150800B8800E220FF2E471FAF7A5BD11220FF2E87144
S3150800B890FAF7A0BD10220FF2F471FAF79BBD0F223A
S3150800B8A00FF2F871FAF796BD0F220FF60001FAF7B4
S3150800B8B091BD0F224FA1FAF78DBD102251A1FAF7BB
S3150800B8C089BD0E220FF2F471FAF784BD0F220FF22A
S3150800B8D0FC71FAF77FBD0F220FF60001FAF77ABD61
S3150800B8E00F220FF60801FAF775BD102249A1FAF7DB
S3150800B8F071BD10224BA1FAF76DBD11224DA1FAF7C1
S3150800B90069BD0A220FF2F471FAF764BD07220FF235
S3150800B910F871FAF75FBD07220FF2F471FAF75ABD0C
S3150800B92007220FF2F471FAF755BD10220FF2F071E3
S3150800B930FAF750BD0F220FF2F871FAF74BBD112234
S3150800B9400FF2FC71FAF746BD0C220FF60801FAF75A
S3150800B95041BD042290A1FAF73DBD04228FA1FAF752
S3150800B96039BD08220FF2F871FAF734BD4C5443007A
S3150800B970485443004D4E540046534500554348002D
S3150800B980535443004343460044434600494E460049
S3150800B99050434600434446004D434600434645004F
S3150800B9A047450000485646005053450048450000A4
S3150800B9B05045000050460000434C450045353200CE
S3150800B9C045353300453534004535350045353600AF
S3150800B9D04535370045353800453539004536300098
S3150800B9E04536310068C00008453632004536330012
S3150800B9F0554B4E00434820636F6E742E206665656E
S3150800BA00642E000044434820636F6E742E206665DA
S3150800BA1065642E0050434820636F6E742E20666559
S3150800BA2065642E00432F4420636F6E742E2066656E
S3150800BA3065642E004D61696E20636F6E742E2066F4
S3150800BA406565642E00000000104601293ED00229D3
S3150800BA5040D0042942D0082944D0102946D02029AC
S3150800BA6048D040294AD080294CD0B1F5807F4DD0A6
S3150800BA70B1F5007F4ED0B1F5806F4FD0B1F5006FAC
S3150800BA8050D0B1F5805F51D0B1F5005F52D0B1F515
S3150800BA90804F53D0B1F5004F54D0B1F5803F55D003
S3150800BAA0B1F5003F56D0B1F5802F57D0B1F5002F2C
S3150800BAB058D0B1F5801F59D0B1F5001F5AD0B1F54D
S3150800BAC0800F5BD0B1F5000F5CD05FE0042234A193
S3150800BAD0FAF780BC042233A1FAF77CBC0422BDA184
S3150800BAE0FAF778BC0422BCA1FAF774BC0422BBA1FD
S3150800BAF0FAF770BC0422BAA1FAF76CBC0422B9A101
S3150800BB00FAF768BC0422B8A1FAF764BC0422B7A104
S3150800BB10FAF760BC0422B6A1FAF75CBC0422B5A108
S3150800BB20FAF758BC0422B4A1FAF754BC0422B3A10C
S3150800BB30FAF750BC0422B2A1FAF74CBC0422B1A110
S3150800BB40FAF748BC0322B0A1FAF744BC0322AFA116
S3150800BB50FAF740BC0322AEA1FAF73CBC0422ADA119
S3150800BB60FAF738BC0322ACA1FAF734BC0422ABA11D
S3150800BB70FAF730BC0422AAA1FAF72CBC042206A1C3
S3150800BB80FAF728BC042205A1FAF724BC0422A5A1C9
S3150800BB90FAF720BC60C10008493232004932330046
S3150800BBA043565200434F4E001046012971D00229D0
S3150800BBB074D0042977D008297AD010297DD0202975
S3150800BBC000F08080402900F08280802900F084807F
S3150800BBD0B1F5807F00F08580B1F5007F00F08680A2
S3150800BBE0B1F5806F00F08780B1F5006F00F08880AE
S3150800BBF0B1F5805F00F08980B1F5005F00F08A80BA
S3150800BC00B1F5804F00F08B80B1F5004F00F08C80C5
S3150800BC10B1F5803F00F08D80B1F5003F00F08E80D1
S3150800BC20B1F5802F00F08F80B1F5002F00F09080DD
S3150800BC30B1F5801F00F09180B1F5001F00F09280E9
S3150800BC40B1F5800F00F09380B1F5000F00F09480F5
S3150800BC50B1F1807F00F09580B1F1007F00F0968009
S3150800BC60B1F1806F00F09780B1F1006F00F0988015
S3150800BC70B1F1805F00F09980B1F1005F00F0998022
S3150800BC80B1F1804F00F09980B1F1004F00F0998032
S3150800BC909BE008220FF2D041FAF79CBB0F220FF265
S3150800BCA0D041FAF797BB09220FF2D441FAF792BBB3
S3150800BCB00F220FF2D841FAF78DBB11220FF2DC41A1
S3150800BCC0FAF788BB0C220FF2E841FAF783BB112278
S3150800BCD00FF2E841FAF77EBB0F220FF2F441FAF7AA
S3150800BCE079BB07220FF2F841FAF774BB07220FF265
S3150800BCF0F841FAF76FBB0D220FF2F441FAF76ABB67
S3150800BD0005220FF2FC41FAF765BB0C220FF2F84147
S3150800BD10FAF760BB11220FF2FC41FAF75BBB0E2261
S3150800BD200FF20451FAF756BB0C220FF20C51FAF730
S3150800BD3051BB0C220FF20C51FAF74CBB0B220FF237
S3150800BD401051FAF747BB0F220FF21051FAF742BB10
S3150800BD500A220FF21851FAF73DBB0F220FF21851BB
S3150800BD60FAF738BB0E220FF22051FAF733BB11222D
S3150800BD700FF22451FAF72EBB10220FF23051FAF7C0
S3150800BD8029BB10220FF23451FAF724BB09220FF20D
S3150800BD903C51FAF71FBB0B220FF23C51FAF71ABBBC
S3150800BDA00D220FF24051FAF715BB04228DA1FAF7BE
S3150800BDB011BB04228CA1FAF70DBB04228BA1FAF75A
S3150800BDC009BB04228AA1FAF705BB08220FF29031B3
S3150800BDD0FAF700BB50444E00494348004944430023
S3150800BDE04343460044434600494E530043524500E8
S3150800BDF050524500445245005043460043444600CD
S3150800BE004D434600494E5400463100004632000074
S3150800BE10463300004342530042520000434D43005C
S3150800BE2043453100554B4E001046012956D002298C
S3150800BE3058D004295AD008295CD010295ED0202968
S3150800BE4060D0402962D0802964D0B1F5807F65D062
S3150800BE50B1F5007F66D0B1F5806F67D0B1F5006F98
S3150800BE6068D0B1F5805F69D0B1F5005F6AD0B1F5E9
S3150800BE70804F6BD0B1F5004F6CD0B1F5803F6DD0D7
S3150800BE80B1F5003F6ED0B1F5802F6FD0B1F5002F18
S3150800BE9070D0B1F5801F71D0B1F5001F72D0B1F521
S3150800BEA0800F73D0B1F5000F74D0B1F1807F75D0D3
S3150800BEB0B1F1007F76D0B1F1806F77D0B1F1006F24
S3150800BEC078D0B1F1805F79D0B1F1005F7AD0B1F165
S3150800BED0804F7BD0B1F1004F7CD07FE0042245A192
S3150800BEE0FAF778BA042244A1FAF774BA032243A1EE
S3150800BEF0FAF770BA042242A1FAF76CBA042241A1F1
S3150800BF00FAF768BA042240A1FAF764BA04223FA1F4
S3150800BF10FAF760BA04223EA1FAF75CBA04223DA1F8
S3150800BF20FAF758BA04223CA1FAF754BA04223BA1FC
S3150800BF30FAF750BA04223AA1FAF74CBA042239A100
S3150800BF40FAF748BA042238A1FAF744BA042237A104
S3150800BF50FAF740BA042236A1FAF73CBA042235A108
S3150800BF60FAF738BA042234A1FAF734BA042233A10C
S3150800BF70FAF730BA042232A1FAF72CBA042231A110
S3150800BF80FAF728BA032230A1FAF724BA04222FA115
S3150800BF90FAF720BA04222EA1FAF71CBA04222DA118
S3150800BFA0FAF718BA04222CA1FAF714BA04222BA11C
S3150800BFB0FAF710BA04222AA1FAF70CBA042209A140
S3150800BFC0FAF708BA042208A1FAF704BA042207A164
S3150800BFD0FAF700BA042206A1FAF7FCB9042221A14D
S3150800BFE0FAF7F8B953323800533239005333300070
S3150800BFF0533331004C4F5300484343004348000035
S3150800C00041434800434350004443480044435000DA
S3150800C0105654480048454100434F4F00485348008E
S3150800C020494E4900504348004353480043454100A0
S3150800C03042413100424132004155580050444100C6
S3150800C040455753004D434F0053520000432F4400B9
S3150800C050525443005254440050555000455831003C
S3150800C06048415500554B4E004261747465727920FB
S3150800C070636F7665720000004368617267657220B7
S3150800C080636F6E6E6563742E00000000506F7765EF
S3150800C0907220646F776E207265712E00496E68692A
S3150800C0A06269742063686172672E0000496E686968
S3150800C0B06269742064697363682E0000496E73753B
S3150800C0C06C2E207374617475730000004368617286
S3150800C0D067652072657175657374000050726563D3
S3150800C0E06861726765207265712E00004469736322
S3150800C0F06861726765207265712E0000496E746505
S3150800C100726C6F636B000000467573652031000022
S3150800C1104675736520320000467573652033000046
S3150800C1204369726375697420627265616B65720032
S3150800C13042616C616E63696E67207265712E0000DC
S3150800C140436C6F7365204D61696E20636F6E742E44
S3150800C15000000000436C6F7365204578742E31002B
S3150800C160554E4B4E4F574E004C6F7720534F43005A
S3150800C170486967682063682E20637572722E00000E
S3150800C1804368617267696E6700000000416C6C6FF6
S3150800C19077206368617267696E67000043482063A9
S3150800C1A07572722E2070726573656E7400000000D9
S3150800C1B04469736368617267696E6700444348201F
S3150800C1C06375722E2070726573656E7400000000C8
S3150800C1D0566F6C742E20746F6F206869676800004C
S3150800C1E04865617465720000436F6F6C6572000084
S3150800C1F04859472073687574646F776E00000000AD
S3150800C200496E697400000000507265636861726760
S3150800C210696E6700436F6D62696C6966742073683E
S3150800C2207574642E0000000043656C6C20616E61B5
S3150800C2306C7973697300000042616C616E63696EA4
S3150800C2406720310042616C616E63696E6720320057
S3150800C25044697363682E204155580000506F77650E
S3150800C2607220646F776E2041434B000043726F77EC
S3150800C2706E204557530000004D61696E20636F6E4E
S3150800C280746163746F720000536572766963652022
S3150800C290726573657400000043686172672E2F44E7
S3150800C2A0697363686172672E0000000052656164F5
S3150800C2B07920746F206368617267650052656164EE
S3150800C2C07920746F2064697363682E00506F7765F0
S3150800C2D0722075700000000045787465726E616C96
S3150800C2E02031000048656174657220284155582937
S3150800C2F00000000070B58CB004460D46DFF8BC653A
S3150800C3003078401E122800F29F81DFE810F01300F3
S3150800C3102A00410058006F0086009D00B400CB003B
S3150800C320DE00F100040119012D013F0153016701E7
S3150800C33079018B010022212103A8FDF775FA212036
S3150800C340019002A8009001AB03AA29462046F9F7F6
S3150800C3502AFD012840F0788103A9F06802F07DFAE9
S3150800C36072E10022212103A8FDF75EFA212001903F
S3150800C37002A8009001AB03AA29462046F9F713FD47
S3150800C380012840F0618103A9F06802F087FA5BE1B1
S3150800C3900022212103A8FDF747FA2120019002A8CF
S3150800C3A0009001AB03AA29462046F9F7FCFC0128B0
S3150800C3B040F04A8103A9F06802F091FA44E10022AC
S3150800C3C0052103A8FDF730FA0520019002A8009080
S3150800C3D001AB03AA29462046F9F7E5FC012840F0F7
S3150800C3E0338103A9F06802F0B9FA2DE1002207218A
S3150800C3F003A8FDF719FA0720019002A8009001ABDF
S3150800C40003AA29462046F9F7CEFC012840F01C81EC
S3150800C41003A9F06802F084FA16E10022052103A8B0
S3150800C420FDF702FA0520019002A8009001AB03AAC5
S3150800C43029462046F9F7B7FC012840F0058103A9EB
S3150800C440F06802F0A9FAFFE00022052103A8FDF72B
S3150800C450EBF90520019002A8009001AB03AA294632
S3150800C4602046F9F7A0FC012840F0EE8003A9F06801
S3150800C47002F0B0FAE8E00022052103A8FDF7D4F996
S3150800C4800520019002A8009001AB03AA2946204680
S3150800C490F9F789FC012840F0D78003A9F06802F073
S3150800C4A0B7FAD1E0002003900420019002A800907A
S3150800C4B001AB03AA2046F9F776FC012840F0C480B0
S3150800C4C00399F06802F06AFBBEE00020039004209E
S3150800C4D0019002A8009001AB03AA2046F9F763FC75
S3150800C4E0012840F0B1800399F06802F073FBABE0D5
S3150800C4F0002003900420019002A8009001AB03AA33
S3150800C5002046F9F750FC012840F09E800399F06810
S3150800C51002F09CFA98E00020ADF80C000220019089
S3150800C52002A8009001AB03AA2046F9F73CFC0128B3
S3150800C53040F08A80BDF80C10F06802F0A3FA83E098
S3150800C5400020ADF80C000220019002A8009001AB73
S3150800C55003AA2046F9F727FC012875D1BDF80C1067
S3150800C560F06802F0ABFA6FE0002003900420019017
S3150800C57002A8009001AB03AA2046F9F714FC01288B
S3150800C58062D10399F06802F0B5FA5DE00020ADF8D3
S3150800C5900C000220019002A8009001AB03AA2046D5
S3150800C5A0F9F701FC01284FD1BDF80C10F06802F02C
S3150800C5B0BDFA49E00020ADF80C000220019002A85F
S3150800C5C0009001AB03AA2046F9F7EDFB01283BD101
S3150800C5D0BDF80C10F06802F0C5FA35E000200390AB
S3150800C5E00420019002A8009001AB03AA2046F9F79F
S3150800C5F0DAFB012828D10399F06802F0E0F823E075
S3150800C600002003900420019002A8009001AB03AA21
S3150800C6102046F9F7C8FB012816D10399F06802F0FD
S3150800C620E8F811E06FF0004003900420019002A89A
S3150800C630009001AB03AA2046F9F7B5FB012803D100
S3150800C6400399F06802F0EFF8022229462046F7F728
S3150800C65019FF7068804730780146132904DBB068F3
S3150800C66080471420307001E0401C30700CB070BD5B
S3150800C6701FB50122914C2378002B01D0142B01D130
S3150800C6801346237023785B1E122B00F20C81DFE819
S3150800C69013F0130020002D003A00470054006100F3
S3150800C6A06E007B0088009500A200AF00BC00C900A0
S3150800C6B0D600E300F000FD0000220292804A0192B3
S3150800C6C00922009201234FF42852F9F75FFB02462C
S3150800C6D0EBE0002202927A4A019209220092002394
S3150800C6E042F6FF72F9F752FB0246DEE0002202929A
S3150800C6F0734A019209220092002341F20A02F9F7CD
S3150800C70045FB0246D1E0002202926D4A01920522BB
S3150800C7100092342344F27002F9F738FB0246C4E06B
S3150800C72000220292664A019205220092352344F2BB
S3150800C7307002F9F72BFB0246B7E000220292604A24
S3150800C7400192052200923C2344F27002F9F71EFB7F
S3150800C7500246AAE000220292594A01920522009254
S3150800C7603D2344F27002F9F711FB02469DE00022D0
S3150800C7700292534A0192052200923E2344F2700225
S3150800C780F9F704FB024690E0002202924C4A019215
S3150800C79008220092062344F27002F9F7F7FA0246D5
S3150800C7A083E000220292464A01920822009213462A
S3150800C7B044F27002F9F7EAFA024676E0002202929B
S3150800C7C03F4A019208220092152344F27002F9F7B3
S3150800C7D0DDFA024669E000220292394A01920622EF
S3150800C7E00092162344F27002F9F7D0FA02465CE08A
S3150800C7F000220292324A019206220092172344F23C
S3150800C8007002F9F7C3FA02464FE0002202922C4A58
S3150800C810019208220092182344F27002F9F7B6FA38
S3150800C820024642E000220292254A0192062200921E
S3150800C830192344F27002F9F7A9FA024635E00022F4
S3150800C84002921F4A0192062200921A2344F27002AB
S3150800C850F9F79CFA024628E000220292184A019249
S3150800C86008220092502344F27002F9F78FFA024622
S3150800C8701BE000220292124A0192082200925123DA
S3150800C88044F27002F9F782FA02460EE0002202929A
S3150800C8900B4A0192042200929E2344F27002F9F791
S3150800C8A075FA024601E000202070104604B010BD5B
S3150800C8B0024BD86059609A6070470000403F0020DC
S3150800C8C0F5C2000810B50446022101F0C7FDDFF8DD
S3150800C8D0480B206004F581704FF6FF710180418096
S3150800C8E0204610BD7CB504460D4604F10C01684689
S3150800C8F006F061FD2878698840EA0120216B4140ED
S3150800C90061632063B5F9040006F05EFDDFF80C1BD1
S3150800C910FEF782F8206595F9060006F055FD606574
S3150800C92095F9070006F050FDA06504F15C0630781D
S3150800C930297A884201D0012000E000207070287A08
S3150800C9403070652801DB64203070688906F04EFD7A
S3150800C950DFF8C81AFEF760F87060A06BE96821F086
S3150800C96080414840E063E86820F08040A063216C7D
S3150800C97028694140616428692064A16C686941405E
S3150800C980E1646869A064684606F03DFD73BD082148
S3150800C99001F046BE00207047704700207047704778
S3150800C9A038B504460D4604F10C01684606F003FD49
S3150800C9B0A4F80251684606F026FD31BD1CB50446AA
S3150800C9C004F10C01684606F0F6FCB4F80241684624
S3150800C9D006F019FD204616BD38B504460D4604F185
S3150800C9E00C01684606F0E7FCA4F80451684606F010
S3150800C9F00AFD31BD1CB5044604F10C01684606F073
S3150800CA00DAFCB4F80441684606F0FDFC204616BD7B
S3150800CA101046012971D0022974D0042977D0082933
S3150800CA207AD010297DD0202900F08080402900F096
S3150800CA308280802900F08480B1F5807F00F08580AF
S3150800CA40B1F5007F00F08680B1F5806F00F0878031
S3150800CA50B1F5006F00F08880B1F5805F00F089803D
S3150800CA60B1F5005F00F08A80B1F5804F00F08B8049
S3150800CA70B1F5004F00F08C80B1F5803F00F08D8055
S3150800CA80B1F5003F00F08E80B1F5802F00F08F8061
S3150800CA90B1F5002F00F09080B1F5801F00F091806D
S3150800CAA0B1F5001F00F09280B1F5800F00F0938079
S3150800CAB0B1F5000F00F09480B1F1807F00F0958009
S3150800CAC0B1F1007F00F09680B1F1806F00F0978099
S3150800CAD0B1F1006F00F09880B1F1805F00F09980A5
S3150800CAE0B1F1005F00F09A80B1F1804F00F09B80B1
S3150800CAF0B1F1004F00F09C809FE00E220FF6003146
S3150800CB00F9F768BC0F220FF24011F9F763BC0F2240
S3150800CB100FF24411F9F75EBC10220FF24C11F9F727
S3150800CB2059BC11220FF25011F9F754BC10220FF21A
S3150800CB305C11F9F74FBC11220FF26011F9F74ABCE4
S3150800CB4010220FF26C11F9F745BC11220FF2701181
S3150800CB50F9F740BC09220FF27C11F9F73BBC0F220A
S3150800CB600FF6AC21F9F736BC10220FF6B421F9F707
S3150800CB7031BC10220FF6B821F9F72CBC11220FF29E
S3150800CB806011F9F727BC0A220FF26811F9F722BCDF
S3150800CB900C220FF26C11F9F71DBC0A220FF26C1168
S3150800CBA0F9F718BC0E220FF27011F9F713BC06221A
S3150800CBB00FF27411F9F70EBC0E220FF27411F9F781
S3150800CBC009BC11220FF27811F9F704BC10220FF2F2
S3150800CBD08411F9F7FFBB0B220FF28811F9F7FABB9C
S3150800CBE00A220FF28C11F9F7F5BB0F220FF28C11FE
S3150800CBF0F9F7F0BB0C220FF29411F9F7EBBB0922F7
S3150800CC000FF29411F9F7E6BB09220FF29811F9F71A
S3150800CC10E1BB10220FF62821F9F7DCBB11220FF62B
S3150800CC203021F9F7D7BB10220FF28411F9F7D2BBDE
S3150800CC3011220FF28C11F9F7CDBB0822DFF87C1B05
S3150800CC40F9F7C8BB000000004D6F64756C65206F6E
S3150800CC5066666C696E650000437269746963616C27
S3150800CC60206572726F720000566F6C74616765207A
S3150800CC70756E622E20434800566F6C746167652096
S3150800CC80756E622E20444348000000004375727298
S3150800CC90656E7420756E622E204348004375727265
S3150800CCA0656E7420756E622E2044434800000000AD
S3150800CCB043482063757272656E7420756E622E0025
S3150800CCC04443482063757272656E7420756E622ED1
S3150800CCD0000000004E6565642041434B00000000DB
S3150800CCE0496E73756C6174696F6E206661756C74D4
S3150800CCF000000000574454207265736574000000F4
S3150800CD004F76657263757272656E7400505357205C
S3150800CD106572726F72000000486967682068756DF1
S3150800CD2069646974790000005761746572000000CF
S3150800CD3053686F72742063697263756974000000C2
S3150800CD404869676820636F6E742E2074656D702E4F
S3150800CD5000000000537475636B20636F6E74616323
S3150800CD60746F72004856494C206572726F720000E3
S3150800CD70414443206572726F7200000043757272F7
S3150800CD80656E742073656E736F7200004D6F756EF5
S3150800CD9074206572726F72004653206572726F72E4
S3150800CDA0000000004856206661756C74000000009B
S3150800CDB0507265636861726765206572726F72008A
S3150800CDC04375722E206C696D6974206572726F7274
S3150800CDD0000000001046012956D0022958D004291F
S3150800CDE05AD008295CD010295ED0202960D0402965
S3150800CDF062D0802964D0B1F5807F65D0B1F5007F17
S3150800CE0066D0B1F5806F67D0B1F5006F68D0B1F51F
S3150800CE10805F69D0B1F5005F6AD0B1F5804F6BD0FD
S3150800CE20B1F5004F6CD0B1F5803F6DD0B1F5003F3C
S3150800CE306ED0B1F5802F6FD0B1F5002F70D0B1F557
S3150800CE40801F71D0B1F5001F72D0B1F5800F73D075
S3150800CE50B1F5000F74D0B1F1807F75D0B1F1007FC4
S3150800CE6076D0B1F1806F77D0B1F1006F78D0B1F19B
S3150800CE70805F79D0B1F1005F7AD0B1F1804F7BD075
S3150800CE80B1F1004F7CD07FE0042241A1F9F7A2BAA4
S3150800CE90042240A1F9F79EBA04223FA1F9F79ABAEB
S3150800CEA004223EA1F9F796BA04223DA1F9F792BAEF
S3150800CEB004223CA1F9F78EBA04223BA1F9F78ABAF3
S3150800CEC004223AA1F9F786BA042239A1F9F782BAF7
S3150800CED0042238A1F9F77EBA042237A1F9F77ABAFB
S3150800CEE0042236A1F9F776BA042235A1F9F772BAFF
S3150800CEF0042234A1F9F76EBA042233A1F9F76ABA03
S3150800CF00032232A1F9F766BA042231A1F9F762BA07
S3150800CF10042230A1F9F75EBA04222FA1F9F75ABA0A
S3150800CF2004222EA1F9F756BA04222DA1F9F752BA0E
S3150800CF3004222CA1F9F74EBA03222BA1F9F74ABA13
S3150800CF4004229AA1F9F746BA042299A1F9F742BA36
S3150800CF50042298A1F9F73EBA042297A1F9F73ABA3A
S3150800CF60042296A1F9F736BA042295A1F9F732BA3E
S3150800CF70042294A1F9F72EBA032293A1F9F72ABA43
S3150800CF80042292A1F9F726BA042291A1F9F722BA46
S3150800CF90424345004D4F460043455200565543000F
S3150800CFA056554400435543004355440043435500F2
S3150800CFB04443550041434B0043434600444346001F
S3150800CFC043444600494E4600574454004F43000028
S3150800CFD050534500484855005748550053484300A4
S3150800CFE0484354005354430048450000104601295D
S3150800CFF056D0022959D004295BD008295DD01029BA
S3150800D0005FD0202961D0402963D0802965D0B1F549
S3150800D010807F66D0B1F5007F67D0B1F5806F68D0A4
S3150800D020B1F5006F69D0B1F5805F6AD0B1F5005FE0
S3150800D0306BD0B1F5804F6CD0B1F5004F6DD0B1F51E
S3150800D040803F6ED0B1F5003F6FD0B1F5802F70D01C
S3150800D050B1F5002F71D0B1F5801F72D0B1F5001F60
S3150800D06073D0B1F5800F74D0B1F5000F75D0B1F15A
S3150800D070807F76D0B1F1007F77D0B1F1806F78D01C
S3150800D080B1F1006F79D0B1F1805F7AD0B1F1005F6C
S3150800D0907BD0B1F1804F7CD0B1F1004F7DD080E0DC
S3150800D0A00C220FF29C11F9F795B9042249A1F9F758
S3150800D0B091B9042248A1F9F78DB9042247A1F9F7D5
S3150800D0C089B9042246A1F9F785B9042245A1F9F7D9
S3150800D0D081B9042244A1F9F77DB9042243A1F9F7DD
S3150800D0E079B9042242A1F9F775B9042241A1F9F7E1
S3150800D0F071B9042240A1F9F76DB904223FA1F9F7E5
S3150800D10069B904223EA1F9F765B904223DA1F9F7E8
S3150800D11061B904223CA1F9F75DB904223BA1F9F7EC
S3150800D12059B904223AA1F9F755B9042239A1F9F7F0
S3150800D13051B9042238A1F9F74DB9042237A1F9F7F4
S3150800D14049B9042236A1F9F745B9042235A1F9F7F8
S3150800D15041B9042234A1F9F73DB9042233A1F9F7FC
S3150800D16039B9042232A1F9F735B9042231A1F9F700
S3150800D17031B9042230A1F9F72DB904222FA1F9F704
S3150800D18029B90422A0A1F9F725B904229FA1F9F724
S3150800D19021B904229EA1F9F71DB904229DA1F9F728
S3150800D1A019B908220FF62431F9F714B94144430096
S3150800D1B0435345004D4E54004653450048564600D5
S3150800D1C0504346004D43460050450000434C450039
S3150800D1D0554B4E004533330045333400453335004F
S3150800D1E04533360045333700453338004533390073
S3150800D1F04534300045343100453432004534330077
S3150800D2004534340045343500453436004534370056
S3150800D2104534380045343900453530004535310048
S3150800D220453532004535330045353400453535003A
S3150800D230453536004535370045353800453539001A
S3150800D240506F776572206661756C74001046012907
S3150800D25056D0022958D004295AD008295CD010295A
S3150800D2605ED0202960D0402962D0802964D0B1F5EB
S3150800D270807F65D0B1F5007F66D0B1F5806F67D045
S3150800D280B1F5006F68D0B1F5805F69D0B1F5005F80
S3150800D2906AD0B1F5804F6BD0B1F5004F6CD0B1F5BF
S3150800D2A0803F6DD0B1F5003F6ED0B1F5802F6FD0BD
S3150800D2B0B1F5002F70D0B1F5801F71D0B1F5001F00
S3150800D2C072D0B1F5800F73D0B1F5000F74D0B1F1FB
S3150800D2D0807F75D0B1F1007F76D0B1F1806F77D0BD
S3150800D2E0B1F1006F78D0B1F1805F79D0B1F1005F0C
S3150800D2F07AD0B1F1804F7BD0B1F1004F7CD07FE07E
S3150800D3000322A2A1F9F766B80422A1A1F9F762B827
S3150800D3100422A0A1F9F75EB804229FA1F9F75AB82A
S3150800D32004229EA1F9F756B804229DA1F9F752B82E
S3150800D33004229CA1F9F74EB804229BA1F9F74AB832
S3150800D34004229AA1F9F746B8042299A1F9F742B836
S3150800D350042298A1F9F73EB8042297A1F9F73AB83A
S3150800D360042296A1F9F736B8042295A1F9F732B83E
S3150800D370042294A1F9F72EB8042293A1F9F72AB842
S3150800D380042292A1F9F726B8042291A1F9F722B846
S3150800D390042290A1F9F71EB804228FA1F9F71AB84A
S3150800D3A004228EA1F9F716B804228DA1F9F712B84E
S3150800D3B004228CA1F9F70EB804228BA1F9F70AB852
S3150800D3C004228AA1F9F706B8042289A1F9F702B856
S3150800D3D0042288A1F8F7FEBF042287A1F8F7FABF4E
S3150800D3E0042209A1F8F7F6BF042208A1F8F7F2BF4C
S3150800D3F0042207A1F8F7EEBF042206A1F8F7EABF50
S3150800D40004227EA1F8F7E6BF4536300045363100DE
S3150800D410453632004536330018C001080000204161
S3150800D420104601293ED0022941D0042944D00829B2
S3150800D43047D010294AD020294DD0402950D08029DC
S3150800D44053D0B1F5807F55D0B1F5007F57D0B1F5EF
S3150800D450806F59D0B1F5006F5BD0B1F5805F5DD0B4
S3150800D460B1F5005F5FD0B1F5804F61D0B1F5004FDF
S3150800D47062D0B1F5803F63D0B1F5003F64D0B1F515
S3150800D480802F65D0B1F5002F66D0B1F5801F67D023
S3150800D490B1F5001F68D0B1F5800F69D0B1F5000F5E
S3150800D4A06AD06DE00E220FF25811F8F793BF0F22DB
S3150800D4B00FF29871F8F78EBF0F220FF2A071F8F7E6
S3150800D4C089BF0F220FF2A471F8F784BF0F220FF25B
S3150800D4D04011F8F77FBF10220FF24411F8F77ABF10
S3150800D4E010220FF24C11F8F775BF0E220FF28C714D
S3150800D4F0F8F770BF0F220FF29471F8F76BBF11227D
S3150800D5000FF29871F8F766BF10220FF23411F8F788
S3150800D51061BF11220FF23811F8F75CBF0A220FF229
S3150800D5209071F8F757BF10220FF29071F8F752BFB3
S3150800D53004229FA1F8F74EBF04229EA1F8F74ABF1E
S3150800D54004229DA1F8F746BF04229DA1F8F742BF21
S3150800D55004229CA1F8F73EBF04229BA1F8F73ABF24
S3150800D56004229AA1F8F736BF042299A1F8F732BF28
S3150800D570042298A1F8F72EBF042297A1F8F72ABF2C
S3150800D58008220FF24871F8F725BF00005046000040
S3150800D59045333300453334004533350045333600CB
S3150800D5A045333700453338004533390045343000B4
S3150800D5B045343100453432004534330045343400AF
S3150800D5C0453435004534360045343700453438008F
S3150800D5D0453439004535300045353100453532008A
S3150800D5E04535330045353400453535004535360073
S3150800D5F0453537004535380045353900554B4E0019
S3150800D6004261747465727920636F766572000000F2
S3150800D610434820636F6E742E20666565642E00008D
S3150800D62044434820636F6E742E20666565642E0039
S3150800D630432F4420636F6E742E20666565642E0042
S3150800D64050434820636F6E742E20666565642E000D
S3150800D6504D61696E20636F6E742E20666565642E53
S3150800D66000000000104601293ED0022940D00429B6
S3150800D67042D0082944D0102946D0202948D040292C
S3150800D6804AD080294CD0B1F5807F4DD0B1F5007FC6
S3150800D6904ED0B1F5806F4FD0B1F5006F50D0B1F5CF
S3150800D6A0805F51D0B1F5005F52D0B1F5804F53D0AD
S3150800D6B0B1F5004F54D0B1F5803F55D0B1F5003FD4
S3150800D6C056D0B1F5802F57D0B1F5002F58D0B1F507
S3150800D6D0801F59D0B1F5001F5AD0B1F5800F5BD025
S3150800D6E0B1F5000F5CD05FE004223CA1F8F772BEEA
S3150800D6F004223BA1F8F76EBE04223AA1F8F76ABEE7
S3150800D700042239A1F8F766BE042238A1F8F762BEEA
S3150800D710042237A1F8F75EBE042236A1F8F75ABEEE
S3150800D7200422B6A1F8F756BE0422B5A1F8F752BEF0
S3150800D7300422B4A1F8F74EBE0422B3A1F8F74ABEF4
S3150800D7400422B2A1F8F746BE0422B1A1F8F742BEF8
S3150800D7500422B0A1F8F73EBE042215A1F8F73ABE96
S3150800D760042214A1F8F736BE042213A1F8F732BE34
S3150800D770042213A1F8F72EBE042212A1F8F72ABE36
S3150800D780042211A1F8F726BE042210A1F8F722BE3A
S3150800D79004220FA1F8F71EBE04220EA1F8F71ABE3E
S3150800D7A004220DA1F8F716BE04229BA1F8F712BEB3
S3150800D7B0493134004931350049313600CCDC00089E
S3150800D7C0493137004931380049313900493230008A
S3150800D7D04932310049323200493233004356520049
S3150800D7E043524500505245004452450043434600C3
S3150800D7F04443460043444600104601296BD002299B
S3150800D8006ED0042971D0082974D0102977D0202920
S3150800D8107AD040297DD0802900F08080B1F5807FBC
S3150800D82000F08180B1F5007F00F08280B1F5806F4D
S3150800D83000F08380B1F5006F00F08480B1F5805F59
S3150800D84000F08580B1F5005F00F08680B1F5804F65
S3150800D85000F08780B1F5004F00F08880B1F5803F71
S3150800D86000F08980B1F5003F00F08A80B1F5802F7D
S3150800D87000F08A80B1F5002F00F08A80B1F5801F8C
S3150800D88000F08A80B1F5001F00F08A80B1F5800F9C
S3150800D89000F08A80B1F5000F00F08A80B1F1807F30
S3150800D8A000F08A80B1F1007F00F08A80B1F1806FC4
S3150800D8B000F08A80B1F1006F00F08A80B1F1805FD4
S3150800D8C000F08A80B1F1005F00F08A80B1F1004F64
S3150800D8D000F08A808CE005220FF2F831F8F77ABD5D
S3150800D8E009220FF2F831F8F775BD0C220FF2F8315C
S3150800D8F0F8F770BD11220FF2FC31F8F76BBD112253
S3150800D9000FF20441F8F766BD11220FF21041F8F73D
S3150800D91061BD0C220FF21841F8F75CBD11220FF217
S3150800D9201C41F8F757BD0E220FF22441F8F752BDF5
S3150800D9300E220FF22C41F8F74DBD0E220FF23041A0
S3150800D940F8F748BD07220FF23841F8F743BD07221A
S3150800D9500FF23441F8F73EBD0F220FF23441F8F7C3
S3150800D96039BD0E220FF23841F8F734BD0D220FF2F9
S3150800D9704041F8F72FBD11220FF24441F8F72ABDAE
S3150800D980042292A1F8F726BD042291A1F8F722BD38
S3150800D990042290A1F8F71EBD04228FA1F8F71ABD3C
S3150800D9A004228EA1F8F716BD04228DA1F8F712BD40
S3150800D9B004228CA1F8F70EBD04228BA1F8F70ABD44
S3150800D9C004228AA1F8F706BD042289A1F8F702BD48
S3150800D9D0042288A1F8F7FEBC042287A1F8F7FABC4E
S3150800D9E0042286A1F8F7F6BC042285A1F8F7F2BC52
S3150800D9F008220FF2D821F8F7EDBC0000494E530073
S3150800DA004A5443004A544400504346004D43460096
S3150800DA10494E540050444E00554B4E0010460129BD
S3150800DA2053D0022955D0042957D0082959D010298E
S3150800DA305BD020295DD040295FD0802961D0B1F51F
S3150800DA40807F62D0B1F5007F63D0B1F5806F64D076
S3150800DA50B1F5006F65D0B1F5805F66D0B1F5005FAE
S3150800DA6067D0B1F5804F68D0B1F5004F69D0B1F5F0
S3150800DA70803F6AD0B1F5003F6BD0B1F5802F6CD0EE
S3150800DA80B1F5002F6DD0B1F5801F6ED0B1F5001F2E
S3150800DA906FD0B1F5800F70D0B1F5000F71D0B1F12C
S3150800DAA0807F72D0B1F1007F73D0B1F1806F74D0EE
S3150800DAB0B1F1006F75D0B1F1805F76D0B1F1005F3A
S3150800DAC077D0B1F1004F78D07BE004224DA1F8F76A
S3150800DAD081BC03224CA1F8F77DBC04224BA1F8F7C0
S3150800DAE079BC04224AA1F8F775BC042249A1F8F7C3
S3150800DAF071BC042248A1F8F76DBC042247A1F8F7C7
S3150800DB0069BC042246A1F8F765BC042245A1F8F7CA
S3150800DB1061BC042244A1F8F75DBC042243A1F8F7CE
S3150800DB2059BC042242A1F8F755BC042241A1F8F7D2
S3150800DB3051BC042240A1F8F74DBC03223FA1F8F7D7
S3150800DB4049BC03223EA1F8F745BC04223DA1F8F7DB
S3150800DB5041BC04221DA1F8F73DBC04221CA1F8F71C
S3150800DB6039BC04221BA1F8F735BC04221AA1F8F720
S3150800DB7031BC042219A1F8F72DBC042218A1F8F724
S3150800DB8029BC042217A1F8F725BC042216A1F8F728
S3150800DB9021BC042215A1F8F71DBC042214A1F8F72C
S3150800DBA019BC042213A1F8F715BC042212A1F8F730
S3150800DBB011BC042211A1F8F70DBC042210A1F8F734
S3150800DBC009BC042220A1F8F705BC00005331370030
S3150800DBD05331380053313900533230005332310053
S3150800DBE05332320053323300533234005332350045
S3150800DBF05332360053323700533238005332390025
S3150800DC0053333100494E4900434800004443480015
S3150800DC104343500044435000432F440050434800B8
S3150800DC20494E4D0046314D0046324D0046334D00B3
S3150800DC3048454100434F4F004D434F0053520000A3
S3150800DC404350000047454D00554B4E0043686172EE
S3150800DC506765207265717565737400005072656337
S3150800DC606861726765207265712E00004469736386
S3150800DC706861726765207265712E0000496E73755A
S3150800DC806C2E207374617475730000004A6F696E98
S3150800DC9020746F2063686172676500004A6F696E59
S3150800DCA020746F20646973636861722E0000000037
S3150800DCB0496E7465726C6F636B000000506F776510
S3150800DCC07220646F776E207265712E00554E4B4E2A
S3150800DCD04F574E00496E6974000000004368617230
S3150800DCE067696E670000000044697363686172675C
S3150800DCF0696E6700434820637572722E20707265DC
S3150800DD0073656E7400000000444348206375722EE4
S3150800DD102070726573656E74000000004368617256
S3150800DD20672E2F44697363686172672E00000000CE
S3150800DD305072656368617267696E6700496E7465DB
S3150800DD40726C6F636B20286D6F642E2900000000CB
S3150800DD5046757365203120286D6F642E29000000F2
S3150800DD6046757365203220286D6F642E29000000E1
S3150800DD7046757365203320286D6F64292E000000D0
S3150800DD804865617465720000436F6F6C65720000C8
S3150800DD904D61696E20636F6E746163746F72000003
S3150800DDA05365727669636520726573657400000051
S3150800DDB0436F6F6C616E742070756D7000000000A3
S3150800DDC047656E2E6572726F7220286D6F642E29F4
S3150800DDD00000000070B58CB004460D46DFF84C66AE
S3150800DDE03078401E142800F2CB81DFE810F01500C9
S3150800DDF02C0043005A00710088009F00B600CD0031
S3150800DE00E000F30006011B013001450157016B01D3
S3150800DE107F019301A501B7010022212103A8FBF781
S3150800DE2003FD2120019002A8009001AB03AA294610
S3150800DE302046F7F7B8FF012840F0A28103A9F06849
S3150800DE4000F00BFD9CE10022212103A8FBF7ECFC66
S3150800DE502120019002A8009001AB03AA294620467A
S3150800DE60F7F7A1FF012840F08B8103A9F06800F0BD
S3150800DE7015FD85E10022212103A8FBF7D5FC212009
S3150800DE80019002A8009001AB03AA29462046F7F79D
S3150800DE908AFF012840F0748103A9F06800F01FFD8D
S3150800DEA06EE10022052103A8FBF7BEFC05200190C0
S3150800DEB002A8009001AB03AA29462046F7F773FF8C
S3150800DEC0012840F05D8103A9F06800F047FD57E19D
S3150800DED00022072103A8FBF7A7FC0720019002A848
S3150800DEE0009001AB03AA29462046F7F75CFF0128F4
S3150800DEF040F0468103A9F06800F012FD40E10022D7
S3150800DF00052103A8FBF790FC0520019002A80090C4
S3150800DF1001AB03AA29462046F7F745FF012840F03A
S3150800DF202F8103A9F06800F037FD29E100220521B9
S3150800DF3003A8FBF779FC0520019002A8009001AB25
S3150800DF4003AA29462046F7F72EFF012840F0188134
S3150800DF5003A9F06800F03EFD12E10022052103A89E
S3150800DF60FBF762FC0520019002A8009001AB03AA0A
S3150800DF7029462046F7F717FF012840F0018103A933
S3150800DF80F06800F045FDFBE00020039004200190B6
S3150800DF9002A8009001AB03AA2046F7F704FF012860
S3150800DFA040F0EE800399F06800F0F8FDE8E0002004
S3150800DFB003900420019002A8009001AB03AA204612
S3150800DFC0F7F7F1FE012840F0DB800399F06800F0CE
S3150800DFD001FED5E0002003900420019002A80090DD
S3150800DFE001AB03AA2046F7F7DEFE012840F0C880F9
S3150800DFF00399F06800F02AFDC2E00020ADF80C0095
S3150800E0000220019002A8009001AB03AA2046F7F768
S3150800E010CAFE012840F0B480BDF80C10F068FEF77F
S3150800E020BFFCADE00020ADF80C000220019002A86C
S3150800E030009001AB03AA2046F7F7B5FE012840F089
S3150800E0409F80BDF80C10F06800F01CFD98E00020D9
S3150800E050ADF80C000220019002A8009001AB03AABB
S3150800E0602046F7F7A0FE012840F08A80BDF80C107C
S3150800E070F06800F023FD83E000200390042001905F
S3150800E08002A8009001AB03AA2046F7F78CFE0128E8
S3150800E09076D10399F06800F02DFD71E00020ADF807
S3150800E0A00C000220019002A8009001AB03AA2046AA
S3150800E0B0F7F779FE012863D1BDF80C10F068FEF772
S3150800E0C08BFC5DE00020ADF80C000220019002A850
S3150800E0D0009001AB03AA2046F7F765FE01284FD149
S3150800E0E0BDF80C10F06800F021FD49E00020ADF8FD
S3150800E0F00C000220019002A8009001AB03AA20465A
S3150800E100F7F751FE01283BD1BDF80C10F06800F076
S3150800E11029FD35E0002003900420019002A8009014
S3150800E12001AB03AA2046F7F73EFE012828D103993A
S3150800E130F06800F044FB23E00020039004200190DF
S3150800E14002A8009001AB03AA2046F7F72CFE012887
S3150800E15016D10399F06800F04CFB11E06FF000400F
S3150800E16003900420019002A8009001AB03AA204660
S3150800E170F7F719FE012803D10399F06800F053FB5D
S3150800E180022229462046F6F77DF9706880473078DE
S3150800E1900146152904DBB06880471620307001E077
S3150800E1A0401C30700CB070BD1FB501229F4C2378FF
S3150800E1B0002B01D0162B01D11346237023785B1E42
S3150800E1C0142B00F22881DFE813F0150022002F0037
S3150800E1D03C0049005600630070007D008A009700E5
S3150800E1E0A400B100BE00CB00D800E500F200FF0095
S3150800E1F00C011901002202928D4A0192092200920D
S3150800E20001234FF42852F7F7C1FD024605E1002223
S3150800E2100292874A019209220092002342F6FF726F
S3150800E220F7F7B4FD0246F8E000220292804A01920E
S3150800E23009220092002341F20A02F7F7A7FD0246D7
S3150800E240EBE0002202927A4A0192052200923423D8
S3150800E25044F27002F7F79AFD0246DEE000220292C7
S3150800E260734A019205220092352344F27002F7F7A9
S3150800E2708DFD0246D1E0002202926D4A01920522E6
S3150800E28000923C2344F27002F7F780FD0246C4E090
S3150800E29000220292664A0192052200923D2344F228
S3150800E2A07002F7F773FD0246B7E000220292604A51
S3150800E2B00192052200923E2344F27002F7F766FDAA
S3150800E2C00246AAE000220292594A019208220092C6
S3150800E2D0062344F27002F7F759FD02469DE0002234
S3150800E2E00292534A019208220092134644F270029F
S3150800E2F0F7F74CFD024690E0002202924C4A019242
S3150800E30008220092152344F27002F7F73FFD0246F1
S3150800E31083E000220292464A0192062200922023B6
S3150800E32044F27002F7F732FD024676E000220292C6
S3150800E3303F4A019206220092162344F27002F7F72A
S3150800E34025FD024669E000220292394A0192062218
S3150800E3500092172344F27002F7F718FD02465CE0B4
S3150800E36000220292324A019208220092182344F2AD
S3150800E3707002F7F70BFD02464FE0002202922C4A84
S3150800E380019206220092212344F27002F7F7FEFC5E
S3150800E390024642E000220292254A01920622009293
S3150800E3A0192344F27002F7F7F1FC024635E0002221
S3150800E3B002921F4A0192062200921A2344F2700220
S3150800E3C0F7F7E4FC024628E000220292184A019276
S3150800E3D008220092502344F27002F7F7D7FC02464F
S3150800E3E01BE000220292124A01920822009251234F
S3150800E3F044F27002F7F7CAFC02460EE000220292C7
S3150800E4000B4A019204220092522344F27002F7F753
S3150800E410BDFC024601E000202070104604B010BD85
S3150800E420024BD86059609A6070470000503F002040
S3150800E430D5DD000840EA010C1CEB0C0F4FF0807C80
S3150800E44007D305D01CEB400F9CBF1CEB410F88423D
S3150800E45070471CEB400F98BF814270471CE02DE9BE
S3150800E460F0419DF918609DF91C70089D099CDDF81E
S3150800E47028C0DDF82CE0DDF830800170428083800A
S3150800E4808671C77105724481C0F80CC0C0F810E0E7
S3150800E490C0F81480BDE8F08138B504460D4604F18D
S3150800E4A00C00FBF7DFF9002020636063A063E063DC
S3150800E4B020646064A064E06420656065A06504F17A
S3150800E4C05C0000210170417041608160C1606FF09D
S3150800E4D00041016104F17000062104F09BFF04F17C
S3150800E4E07600042104F096FF04F17A00042104F072
S3150800E4F091FF04F17E00042104F08CFF04F18200F0
S3150800E500042104F087FF04F18600202104F082FF2D
S3150800E51004F1A600202104F07DFF04F1C6002021A5
S3150800E52004F078FF04F1E800002101604FF6FF715E
S3150800E5308180C180002282608181C181114601618A
S3150800E540416101764576204632BD001D70471CB5EF
S3150800E550044604F10C01684604F02DFF94F80141C5
S3150800E560684604F050FF204616BD38B504460D46E9
S3150800E57004F10C01684604F01EFF84F80051684651
S3150800E58004F041FF31BD1CB5044604F10C01684690
S3150800E59004F011FF94F80041684604F034FF204661
S3150800E5A016BD38B504460D4604F10C01684604F05C
S3150800E5B002FF206B05402C46641EA441E443E40F89
S3150800E5C0684604F020FF204632BD38B504460D469D
S3150800E5D004F10C01684604F0EEFE606B05402C461B
S3150800E5E0641EA441E443E40F684604F00CFF204689
S3150800E5F032BD38B5044604F10C01684604F0DBFE6A
S3150800E6000025284605E0216BC140C90700D56D1CC9
S3150800E610401C1828F7DB684604F0F5FE284632BD8C
S3150800E62038B504460D4604F10C01684604F0C3FEED
S3150800E630A06B05402C46641EA441E443E40F6846DB
S3150800E64004F0E1FE204632BD38B5044604F10C015B
S3150800E650684604F0B0FE0025284605E0A16BC140D7
S3150800E660C90700D56D1C401C2028F7DB684604F056
S3150800E670CAFE284632BD7CB504460D46164604F148
S3150800E6800C01684604F097FE002E01D0606801E090
S3150800E6904FF0FF30216C0D4005402C46641EA44106
S3150800E6A0E443E40F684604F0AEFE204676BD7CB52A
S3150800E6B004460D46164604F10C01684604F07BFE36
S3150800E6C0002E01D0A06801E04FF0FF30A16C0D408C
S3150800E6D005402C46641EA441E443E40F684604F052
S3150800E6E092FE204676BD7CB504460E4604F10C0122
S3150800E6F0684604F060FE0025300001D0606801E03D
S3150800E7004FF0FF3001D0A16801E04FF0FF312A46F3
S3150800E7100CE001239340266C1E40064200D06D1C77
S3150800E720A66C33400B4200D06D1C521C202AF0DB2D
S3150800E730684604F068FE284676BD1CB5044604F112
S3150800E7400C01684604F037FE246D684604F05BFE4B
S3150800E750204616BD1CB5044604F10C01684604F0B3
S3150800E7602AFE646D684604F04EFE204616BD1CB5AA
S3150800E770044604F10C01684604F01DFEA46D6846C3
S3150800E78004F041FE204616BD1CB5044604F10C01F2
S3150800E790684604F010FE94F85C40684604F033FEC0
S3150800E7A0204616BD1CB5044604F10C01684604F063
S3150800E7B002FE246E684604F026FE204616BD38B5CD
S3150800E7C004460D4604F10C01684604F0F4FD65663E
S3150800E7D0684604F018FE31BD1CB5044604F10C0168
S3150800E7E0684604F0E8FD646E684604F00CFE2046B0
S3150800E7F016BD38B504460D4604F10C01684604F00A
S3150800E800DAFDA566684604F0FEFD31BD1CB5044672
S3150800E81004F10C01684604F0CEFDA46E684604F0C7
S3150800E820F2FD204616BD38B504460D4604F10C0126
S3150800E830684604F0C0FDE566684604F0E4FD31BDAF
S3150800E8401CB5044604F10C01684604F0B4FDE46EF8
S3150800E850684604F0D8FD204616BD38B504460D4670
S3150800E86004F10C01684604F0A6FD1F22294604F1AE
S3150800E870C60004F0D3FD002084F8E500684604F0DD
S3150800E880C2FD31BD1CB5044604F10C01684604F00E
S3150800E89092FD04F0B8FD04F1C60016BD38B504466D
S3150800E8A00D4604F10C01684604F085FD1F22294631
S3150800E8B004F1A60004F0B2FD002084F8C5006846FD
S3150800E8C004F0A1FD31BD1CB5044604F10C016846EF
S3150800E8D004F071FD04F097FD04F1A60016BD38B5E5
S3150800E8E004460D4604F10C01684604F064FD1F2237
S3150800E8F0294604F1860004F091FD002084F8C5003D
S3150800E900684604F080FD31BD1CB5044604F10C01CF
S3150800E910684604F050FD04F076FD04F1860016BD45
S3150800E92038B504460D4604F10C01684604F043FD6B
S3150800E9300622294604F17000F7F74CFD684604F0F4
S3150800E94062FD31BD1CB5044604F10C01684604F0AD
S3150800E95032FD04F058FD04F1700016BD38B50446C2
S3150800E9600D4604F10C01684604F025FD04222946EB
S3150800E97004F17600F7F72EFD684604F044FD31BD34
S3150800E9801CB5044604F10C01684604F014FD04F0B5
S3150800E9903AFD04F1760016BD38B504460D4604F175
S3150800E9A00C01684604F007FD0422294604F17A00A2
S3150800E9B0F7F710FD684604F026FD31BD1CB5044680
S3150800E9C004F10C01684604F0F6FC04F01CFD04F1A1
S3150800E9D07A0016BD38B504460D4604F10C016846A2
S3150800E9E004F0E9FC0422294604F17E00F7F7F2FC5C
S3150800E9F0684604F008FD31BD1CB5044604F10C0157
S3150800EA00684604F0D8FC04F0FEFC04F17E0016BD4E
S3150800EA1038B504460D4604F10C01684604F0CBFCF3
S3150800EA200422294604F18200F7F7D4FC684604F06C
S3150800EA30EAFC31BD1CB5044604F10C01684604F035
S3150800EA40BAFC04F0E0FC04F1820016BD38B50446B1
S3150800EA500D4604F10C01684604F0ADFCC4F8E85014
S3150800EA60684604F0D0FC31BD1CB5044604F10C011F
S3150800EA70684604F0A0FCD4F8E840684604F0C3FCF5
S3150800EA80204616BD38B504460D4604F10C01684605
S3150800EA9004F091FCA4F8EC50684604F0B4FC31BDCF
S3150800EAA01CB5044604F10C01684604F084FCB4F86D
S3150800EAB0EC40684604F0A7FC204616BD38B5044667
S3150800EAC00D4604F10C01684604F075FCA4F8EE50F6
S3150800EAD0684604F098FC31BD1CB5044604F10C01E7
S3150800EAE0684604F068FCB4F8EE40684604F08BFC0F
S3150800EAF0204616BD38B504460D4604F10C01684695
S3150800EB0004F059FCC4F8F050684604F07CFC31BDAA
S3150800EB101CB5044604F10C01684604F04CFCD4F814
S3150800EB20F040684604F06FFC204616BD38B504462A
S3150800EB300D4604F10C01684604F03DFCA4F8F450B7
S3150800EB40684604F060FC31BD1CB5044604F10C01AE
S3150800EB50684604F030FCB4F8F440684604F053FC08
S3150800EB60204616BD38B504460D4604F10C01684624
S3150800EB7004F021FCA4F8F650684604F044FC31BDC4
S3150800EB801CB5044604F10C01684604F014FCB4F8FC
S3150800EB90F640684604F037FC204616BD38B50446EC
S3150800EBA00D4604F10C01684604F005FCC4F8F8505B
S3150800EBB0684604F028FC31BD1CB5044604F10C0176
S3150800EBC0684604F0F8FBD4F8F840684604F01BFCE5
S3150800EBD0204616BD38B504460D4604F10C016846B4
S3150800EBE004F0E9FBC4F8FC50684604F00CFC31BD9F
S3150800EBF01CB5044604F10C01684604F0DCFBD4F8A5
S3150800EC00FC40684604F0FFFB204616BDEFF305807E
S3150800EC10401E8041C043C00F7047EFF310800028A4
S3150800EC2006D1EFF31180401E8041C043C00F7047E4
S3150800EC300120704710B5002806D16FF0030420465E
S3150800EC4004F024FC204610BD0146132002F095FB73
S3150800EC50002801D0002010BD4FF0FF3004F016FC4C
S3150800EC604FF0FF3010BD000010B50446FFF7CEFF89
S3150800EC70002803D1FFF7D1FF002805D06FF005045F
S3150800EC80204604F003FC04E003488446204600DFDF
S3150800EC900446204610BD000035EC0008F8B50446C9
S3150800ECA00D4616461F4604F0F2FB0B482060201D51
S3150800ECB004F0F8FBE56026616761204600F00EF86F
S3150800ECC02046F2BD10B5044603482060201D04F016
S3150800ECD0EAFB204610BD0000C4C001081CB5044666
S3150800ECE000200190009001AAE168204600F0AAF8E9
S3150800ECF06A462169204600F0A5F804F506700199D0
S3150800ED00009A914204D3002101700199416003E001
S3150800ED1001210170009941600078002801D1E1685D
S3150800ED2000E021694FF4007204F11800F7F752FB6E
S3150800ED30002016BD2DE9F84304460D46104619462F
S3150800ED40DDE90823861841EB030740F2FF184FF068
S3150800ED5000094F450AD801D3464507D2204400F199
S3150800ED6018012846F7F736FB484601E04FF0FF3012
S3150800ED70BDE8F2832DE9F8438046894614461D46C8
S3150800ED80DDE90867A01945EB070140F2FF120023E9
S3150800ED90994253D801D3904250D208F1040004F0A6
S3150800EDA083FB00284AD13246494608F11800204418
S3150800EDB0F7F710FB684604F0DBFC002407E008F1CF
S3150800EDC0180050F82410684604F0D6FC641C7E2C03
S3150800EDD0F5DB08F50474E168491CE160684604F04F
S3150800EDE0CBFC684604F0D6FCE068206000986060BA
S3150800EDF0207A002802D1D8F8105001E0D8F80C5033
S3150800EE00D8F81420294608F1040004F04DFC00281F
S3150800EE1014D14FF400732A4608F1180108F10400CA
S3150800EE2004F099FB002809D1207A401E8041C00FC2
S3150800EE30207208F1040004F066FB01E04FF0FF3091
S3150800EE40BDE8F2837CB50C461546684604F090FC8E
S3150800EE50002605E054F82610684604F08DFC761C5A
S3150800EE607F2EF7DB684604F095FC04F5FC704168D4
S3150800EE70009A914201D0002076BD006828600120E2
S3150800EE8076BD000038B504460D4600221C21FAF767
S3150800EE90CBFC2946204604F0BDFC204632BD70B5A1
S3150800EEA004460D46164600221C21FAF7BDFC3246DA
S3150800EEB02946204604F0ADFC204670BD38B5044608
S3150800EEC00D4600221C21FAF7AFFC2946204604F01D
S3150800EED09FFC204632BD010D10B586B00446684633
S3150800EEE01821FBF7F3F8201D04904020059004F143
S3150800EEF044000290342003906A460421084604F030
S3150800EF00C9FF2060002804D14A2203490348FAF7BA
S3150800EF10EDFB204606B010BD08C5010820D401083F
S3150800EF202DE9FF4F81B00446BDF93C50BDF940605C
S3150800EF30BDF94470BDF94880BDF94C90BDF950A0A3
S3150800EF40BDF954B005F020F833482060BDF9081023
S3150800EF50201DFFF797FFBDF90C1004F12000FFF7FD
S3150800EF6091FFBDF9101004F13C00FFF78BFF01205B
S3150800EF70009000230246BDF9381004F1580000F04D
S3150800EF809DFA0120009000230246294604F17400E8
S3150800EF9000F094FA0120009000230246314604F15D
S3150800EFA0900000F08BFA01200090002302463946B3
S3150800EFB004F1AC0000F082FA01200090002302461A
S3150800EFC0414604F1C80000F079FA012000900023B8
S3150800EFD00246494604F1E40000F070FA0120009068
S3150800EFE000230246514604F5807000F067FA0120B6
S3150800EFF0009000230246594604F58E7000F05EFA2A
S3150800F00004F59C701421017000214170817020461E
S3150800F01005B0BDE8F08F000010C9010810B5044618
S3150800F02004F1580004F0B2FF04F1740004F0AEFFD6
S3150800F03004F1900004F0AAFF04F1AC0004F0A6FF66
S3150800F04004F1C80004F0A2FF04F1E40004F09EFFF6
S3150800F05004F5807004F09AFF04F58E7004F096FFAC
S3150800F0603220FAF7EFF83A21204600F011FA052087
S3150800F070FAF7E8F83A21204600F00AFA0120FAF7EA
S3150800F080E1F83A21204600F003FA0821204600F06C
S3150800F090FFF90121204600F0FBF90621204600F081
S3150800F0A0F7F90C212046BDE81040F1E110B50446F9
S3150800F0B094F839010A4690423BD084F8391108463B
S3150800F0C00028204602D0BDE81040A7E72168496914
S3150800F0D088470021201D00F053FA002104F1200082
S3150800F0E000F04EFA002104F13C0000F049FA04F160
S3150800F0F0580004F057FF04F1740004F053FF04F1BC
S3150800F100900004F04FFF04F1AC0004F04BFF04F14B
S3150800F110C80004F047FF04F1E40004F043FF04F5D7
S3150800F120807004F03FFF04F58E70BDE8104004F0CF
S3150800F13039BF10BD90F83901704790F83931002B66
S3150800F14015D0002903D1A2F18001C9B2A0E1012995
S3150800F15003D1A2F14001C9B29AE1022903D1A2F171
S3150800F1606C01C9B294E1A2F12C01C9B290E17047D1
S3150800F17090F83911002900D1704780B5012100F0B7
S3150800F18087F90720BDE80240FAF75CB890F83921FC
S3150800F190002A00D087E17047F8B504460E461D469A
S3150800F1A004F59C77787800281CD012F1010F0AD153
S3150800F1B0284604F003FF02463878821A002A01DD41
S3150800F1C0521000E00022314620462368DB68984743
S3150800F1D005E015F8011B20462268D2699047287871
S3150800F1E00028F6D1F1BD2DE9F84F04460D46114623
S3150800F1F0491E8941C943C90F201D00F0C1F90021E4
S3150800F20004F1200000F0BCF904F1580004F0BEFE39
S3150800F21004F1740004F0BAFE04F19006304604F0D6
S3150800F220B5FE04F1AC07384604F0B0FE04F1C80890
S3150800F230404604F0ABFE04F1E409484604F0A6FE95
S3150800F24004F5807A504604F0A1FE04F58E7B5846F4
S3150800F25004F09CFE05F0010104F1580000F067FA7D
S3150800F2602946490801F0010104F1740000F05FFA2B
S3150800F2702946890801F00101304600F058FA294666
S3150800F280C90801F00101384600F051FA2946090972
S3150800F29001F00101404600F04AFA2946490901F001
S3150800F2A00101484600F043FA2946890901F001019F
S3150800F2B0504600F03CFAED092946584600F037FA60
S3150800F2C0012104F13C0000F05BF9022004F092FEF3
S3150800F2D0002104F13C0000F053F9012104F1580023
S3150800F2E000F025FA012104F1740000F020FA01214A
S3150800F2F0304600F01CFA0121384600F018FA0121C0
S3150800F300404600F014FA0121484600F010FA01219F
S3150800F310504600F00CFA01215846BDE8F44F00F0BB
S3150800F32006BA2DE9F84F04460846401E8041C043F8
S3150800F330C00F0146201D00F023F9012104F1200029
S3150800F34000F01EF904F1580004F02CFE04F17400D4
S3150800F35004F028FE04F19005284604F023FE04F183
S3150800F360AC06304604F01EFE04F1C807384604F021
S3150800F37019FE04F1E408404604F014FE04F5807909
S3150800F380484604F00FFE04F58E7A504604F00AFE4D
S3150800F390012104F13C0000F0F3F8022004F02AFEF3
S3150800F3A004F1580004F046FEB0F1010B6BEB0B0BB1
S3150800F3B06FEA0B0B04F1740004F03CFE002801D040
S3150800F3C0022000E0002040EADB7B284604F032FEFB
S3150800F3D0002801D0042000E0002040EA0B0B30464C
S3150800F3E004F028FE002801D0082000E0002040EAAA
S3150800F3F00B0B384604F01EFE002801D0102000E052
S3150800F400002040EA0B0B404604F014FE002801D009
S3150800F410202000E0002040EA0B0B484604F00AFED4
S3150800F420002801D0402000E0002040EA0B0B50469F
S3150800F43004F000FE002801D0802000E0002040EA09
S3150800F4400B0B002104F13C0000F09AF8022004F0AE
S3150800F450D1FD5846BDE8F28F38B5054695F83A010C
S3150800F460002801D0002032BD4FF47A7400212846C6
S3150800F470FFF757FF000606D5641EF7D1012085F869
S3150800F4803A01002032BD00212846BDE8344048E74D
S3150800F49038B504460D46FFF7DFFF00222946204609
S3150800F4A0BDE838409FE638B504460D46FFF7D4FF59
S3150800F4B0012229462046BDE8384094E6F8B50446B8
S3150800F4C00D4616461F4600221C21FAF7ADF9069886
S3150800F4D000903B4632462946204604F09FF92046CE
S3150800F4E0F2BD38B504460D4600202076F7F7FCFB3A
S3150800F4F02946204604F0A0FDF7F707FC204632BD52
S3150800F50070B504460D46164604F07EFF0348206093
S3150800F5106560A66001202073204670BD94CF01085F
S3150800F5200173704710B504466068227B002A08D12B
S3150800F530002100F038F80021A068BDE8104000F06E
S3150800F5401FB80A2908D17D2100F02DF80121A068ED
S3150800F550BDE8104000F014B8642908D17D2100F0F8
S3150800F56022F80021A068BDE8104000F009B8002183
S3150800F57000F019F80021A068BDE8104000F000B8B6
S3150800F58010B5044604F042FF204610BD38B50446BF
S3150800F5900D46F7F7A9FB2946204604F037FEBDE8D5
S3150800F5A03140F7F7B2BB38B504460D46F7F79CFB72
S3150800F5B02946204604F0CDFEBDE83140F7F7A5BB45
S3150800F5C038B504460D46F7F78FFB2946204604F062
S3150800F5D0C7FFBDE83140F7F798BB040092B202486E
S3150800F5E000EB810002607047006C004038B50400EB
S3150800F5F001D1012032BD4CF6CC402168086045F2A5
S3150800F600555021680860606821684860A0682168CC
S3150800F6108860FAF794F805462168C868002806D075
S3150800F620FAF78DF8401B3128F6D3032032BD4AF687
S3150800F630AA200860002032BD4AF6AA2100680160A7
S3150800F64000207047F8F771BC38B504460D46F7F741
S3150800F6504BFB204604F09EFF2946204604F066FD33
S3150800F660BDE83140F7F751BB10B50446F7F73CFB48
S3150800F670204604F0B1FD0446F7F747FB204610BDC7
S3150800F680F8F753BC0E4A13684FF6FF010B40000209
S3150800F69000F4E06018430B49084310607047BFF355
S3150800F6A04F8F07490A6802F4E062074802430A6076
S3150800F6B0BFF34F8F00BFFDE7E4E7FFF7F0FF00BF9A
S3150800F6C00CED00E00000FA050400FA0502B519463B
S3150800F6D013460A466946006804F0F6FB02BD0000B8
S3150800F6E038B584B004460D461346002000900246FD
S3150800F6F06946286804F006FCC01C03280AD8DFE817
S3150800F70000F0050709021020009905E0002003E033
S3150800F710402001E06FF003002A68019002910392ED
S3150800F72001A890E80E0084E80E0005B030BD10B5BB
S3150800F730044604F039FF204610BD000003000020EF
S3150800F74013F0030F09D0521E22BF13F8010B11F84C
S3150800F75001CBB0EB0C00F3D0704711F0030F14D1B6
S3150800F760121F22BF53F8040B51F804CB6045F7D09B
S3150800F770121D0AD200BA9CFA8CFCB0EB0C0038BFFA
S3150800F7806FF0000088BF01207047521E22BF13F891
S3150800F790010B11F801CBB0EB0C00F6D0521C08BFD8
S3150800F7A0104670475CE080B500F002F8002002BD04
S3150800F7B07CB5044604F50A75B5F9000010F1010F89
S3150800F7C002D0204600F024F80F4E3346002241F2BC
S3150800F7D005012046F6F790FC3346002241F2060161
S3150800F7E02046F6F789FC6868006840000AD5A868CC
S3150800F7F00368002B06D00093044A00212046F6F73A
S3150800F800A1FC288073BD0000A7F70008A5F700082B
S3150800F81010B5044600231A4641F20501F6F76CFCBA
S3150800F82000231A4641F206012046F6F765FCB4F9AC
S3150800F8302802F6F7D6FCA4F8280210BDF8B500F59C
S3150800F8400B70C1698DF8001000680068ADF80200F9
S3150800F8500020ADF804006846F6F74EFD05B000BD79
S3150800F86038B50446FFF7EAFF0546204600F002F8D9
S3150800F870284632BD70B5044604F50D7529688847D3
S3150800F88094F9E600002801D1002070BD0121204628
S3150800F890F8F75CFF0646204669688847304670BD1B
S3150800F8A07047704730B400F51C7211680978002952
S3150800F8B00ED1002106E0002354680D46EDB244F847
S3150800F8C02530491C0B4690F86D42DBB2A342F2D3B1
S3150800F8D0002030BC704710B50446054B002241F2A3
S3150800F8E00301F6F709FC0020D4F87012087010BD61
S3150800F8F0A5F8000870471CB54A79082A0DD101F108
S3150800F900090200920B7A8A79CC7942EA042289782C
S3150800F91001F07F01D0F8A042A04713BD7047000050
S3150800F92030B40A4600F58273196851F82210090C9A
S3150800F9304FF0FF345D6825F8124001220C46E4B208
S3150800F940044484F81821C9B21A6930BC10472DE955
S3150800F950FF4106468F7807F07F070879012827D1E7
S3150800F9603068007801468F4271D100F5E06006F5EF
S3150800F9700F71CA688DF80020ADF8020001208DF8D5
S3150800F980050000208DF8040096F8E0208DF8062082
S3150800F990087A002806D042F080028DF8062000205A
S3150800F9A0087201E0012008726846F6F7A5FC4EE0E9
S3150800F9B08D7905F07F0538463418D6F8A401007805
S3150800F9C084F8A80194F818012946884208D02A46DE
S3150800F9D03946304606F50F735B68984784F8185120
S3150800F9E094F81801002804D139463046D6F83C2246
S3150800F9F0904794F818010F2829D04FF0000806F10F
S3150800FA00E00420E0606A50F8285038462946090C78
S3150800FA10C9B2884213D1ADB2A06A30F91800F6F718
S3150800FA20E0FB002000904FF47A7045432B46814A4C
S3150800FA3041463046F6F786FBA16A21F8180008F118
S3150800FA4001085FFA88F8206A00788045DADBBDE8A5
S3150800FA50FF811FB500F1E004E16A0988002916D084
S3150800FA600168097801F5E061D0F848028DF80000D0
S3150800FA70ADF8021001208DF8050000208DF804006D
S3150800FA8020788DF806006846F6F736FC1FBDB4F9EF
S3150800FA903000F6F7A6FB20861FBD70B5054605F5AE
S3150800FAA0CC74A068008800282CD00026802E2EDA78
S3150800FAB0A81990F818010F2821D0286800788642DE
S3150800FAC01DD0A81990F8A80100280BD16268002A51
S3150800FAD004D030460146C9B2284690470120A919E4
S3150800FAE081F81801A81990F8A801401EA91981F8EB
S3150800FAF0A80130460146C9B2284600F070F9761CBE
S3150800FB00F6B2D3E7B4F90000F6F76BFB208070BDB8
S3150800FB1010B5044600F0B2F8204600F052F800206E
S3150800FB2010BD38B5044604F58675B5F90400F6F730
S3150800FB3058FBA8802868008800280AD04FF47A71F4
S3150800FB404843009000233C4A19462046F6F7FAFA3D
S3150800FB50A880002032BD7CB50446384B002241F20D
S3150800FB601701F6F7C9FA002084F84402064604F598
S3150800FB70807513E0686830F82630002B0CD000201A
S3150800FB8000904FF47A7043432A4A31462046F6F7E6
S3150800FB90D9FAA96821F81600761CF6B22868007802
S3150800FBA08642E7DBE8680388002B09D04FF47A70B1
S3150800FBB043430093204A00212046F6F7C3FA2882D9
S3150800FBC073BD38B504461E4D2B46002241F20C0182
S3150800FBD0F6F792FA2B46002241F20D012046F6F777
S3150800FBE08BFA04F5CC75A8680388002B21D0E86841
S3150800FBF0007800281DD04FF47A7043430093114AC9
S3150800FC0000212046F6F79EFA288000200FE02118EA
S3150800FC1091F818110F2908D021680978884204D06C
S3150800FC20E9680978221882F8A811401CC0B2802811
S3150800FC30EDDB31BD21F9000853FA000823FB000863
S3150800FC4011FB00089BFA000870B50446002504F568
S3150800FC50807609E0B06830F91500F6F7C2FAB1689F
S3150800FC6021F815006D1CEDB2306800788542F1DB8D
S3150800FC70B6F91000F6F7B5FA308270BD10B504462D
S3150800FC80B4F99801F6F7ADFAA4F8980110BD10B5C5
S3150800FC900446FFF760FF2046BDE8104091E710B51F
S3150800FCA00446FFF7D1FF2046BDE81040E6E7704757
S3150800FCB070477047704770B5044604F1E0052A7826
S3150800FCC07F2A03D0052A01D0042A51D1C8790028F1
S3150800FCD003D023681B7898424AD18879012808D02E
S3150800FCE0022810D0802818D0812820D0822829D030
S3150800FCF070BD7F2A01D0042A3AD105212046BDE8E5
S3150800FD007040F8F7C3BF7F2A01D0052A30D10421F5
S3150800FD102046BDE87040F8F7B9BF052A01D0042A85
S3150800FD2026D17F212046BDE87040F8F7AFBFA96904
S3150800FD30002901D02046884700212046BDE87040AA
S3150800FD40F8F7A4BF2046F8F7F6FF0646E969002942
S3150800FD5001D020468847FF20216808703146204692
S3150800FD60F8F7ECFF00212046BDE87040F8F78EBF93
S3150800FD7070BD1FB50446F6F721FD002801D1002005
S3150800FD8015E0D4F848028DF800002068007840F4A1
S3150800FD90E060ADF8020000208DF8040001208DF81F
S3150800FDA0050000208DF806006846F6F7A5FA04B0A7
S3150800FDB010BDF8B5D0F848028DF800000020ADF85F
S3150800FDC002008DF8040002208DF805008DF8062043
S3150800FDD08DF807106846F6F78FFA05B000BDF8B536
S3150800FDE0D0F848028DF8000041F4E061ADF8021041
S3150800FDF001208DF8040000208DF805006846F6F706
S3150800FE007BFA05B000BD000040F0200070472DE9E0
S3150800FE10F14FB0B0924604910DF142013A9A2B91F6
S3150800FE2099464A7000200AE01AF8011B0498309A8D
S3150800FE3090470028049000F031860D98401C0D90DC
S3150800FE409AF8000050B12528EED10021002207912A
S3150800FE50089209910A920B910C9204E00D9800F011
S3150800FE601FBE41F001011AF8010F2028F9D02328F6
S3150800FE700CD02B2804D02D2805D0302809D00BE02B
S3150800FE8041F00201EFE741F00401ECE741F0080117
S3150800FE90E9E741F01001E6E72A280FD1D9F8002052
S3150800FEA052F8040BC9F8002000280F9003D54042E9
S3150800FEB00F9041F004010AF1010A14E00F92DFF8ED
S3150800FEC0E83B0AE00F98984205DA00EB800402EB5B
S3150800FED04402303A0F920AF1010A9AF80020A2F178
S3150800FEE030000A28EED39AF800002E2803D04FF0E7
S3150800FEF0FF320E9229E01AF8010F2A2809D1D9F8FB
S3150800FF00000050F8042BC9F800000E920AF1010A05
S3150800FF101BE02D280CBF0AF1010A002000220E92D0
S3150800FF20DFF8844B0BE040B90E9AA24205DA02EBE1
S3150800FF30820503EB4503303B0E930AF1010A9AF852
S3150800FF400030A3F130020A2AEDD3ADF840100FF6BF
S3150800FF505C309AF8001004F029FB08B11AF8010B76
S3150800FF608DF842009DF84200682805D19AF80000ED
S3150800FF7068280CD1622106E06C2804BF9AF80000B4
S3150800FF806C2804D171218DF842100AF1010A12A8D1
S3150800FF9006901AF801BBBBF125012CD01C3900F0DC
S3150800FFA09481091F022940F29081133900F0A88430
S3150800FFB0093900F08A81891E00F03D85491E00F046
S3150800FFC0EA84491E022940F28081091F00F0E38471
S3150800FFD0491F00F0EF80491E00F09284491E00F088
S3150800FFE0D780C91E0CD0891E00F08A84C91E00F06D
S3150800FFF0878400F02BBD01220792252100F023BD3E
S31508010000D9F8000050F8044BC9F80000002C0594F3
S3150801001040F0AB802B994878002800F0A1804FF07A
S31508010020FF340FF6902004F0CDFA201A40F03685F9
S3150801003000F018BD01236A4602A9304600F0FEFD0C
S31508010040002840F02B856D1EF4D13096079D12AF1E
S3150801005075B1309E17F8011B0498B0470028049023
S3150801006000F01C850D98401C6D1E0D90F2D130963E
S315080100700A9D3021002D8DF800100CDD309E0123DC
S315080100806A4602A9304600F0D9FD002840F00685E7
S315080100906D1EF4D13096059F089D75B1309E17F8EF
S315080100A0011B0498B0470028049000F0F7840D98C6
S315080100B0401C6D1E0D90F2D130960B9D3021002DFE
S315080100C08DF800100CDD309E01236A4602A93046E0
S315080100D000F0B4FD002840F0E1846D1EF4D130969D
S315080100E005980899099D471875B1309E17F8011B9F
S315080100F00498B0470028049000F0D0840D98401C5D
S315080101006D1E0D90F2D130960C9D3021002D8DF883
S3150801011000100CDD309E01236A4602A9304600F024
S315080101208DFD002840F0BA846D1EF4D130969DF8F5
S31508010130400041077FF584AE2020002C8DF8000091
S315080101407FF77EAE309D01236A4602A9284600F054
S3150801015075FD002840F0A284641EF4D130956FE63F
S315080101600FF63830059000F07DBC0E9D002D04D5A4
S31508010170204603F023FF044607E02A46204604F0FA
S3150801018041FA002814BF041B2C46089400F06ABCE7
S31508010190D9F8001051F8040BC9F8001020F0000432
S315080101A0002121F0FF35CDE9024512AB05937821EF
S315080101B000F03DBC2B99487820B14FF0FF340FF67B
S315080101C0AC2030E79DF84200622860D0682817D035
S315080101D06A283FD06C2806D0712847D074282CD0BD
S315080101E07A281DD062E0D9F8001051F8040BC9F835
S315080101F00010002866D14FF0FF340FF6882012E769
S31508010200D9F8001051F8040BC9F8001020B94FF0BD
S31508010210FF340FF6702006E70D99018000F022BC25
S31508010220D9F8001051F8040BC9F80010002849D173
S315080102304FF0FF340FF64C20F5E6D9F8001051F8C7
S31508010240040BC9F8001000283CD14FF0FF340FF613
S315080102503420E8E6D9F8001051F8040BC9F8001063
S3150801026080B94FF0FF340FF61C20DCE6D9F80010F0
S3150801027051F8040BC9F8001020B94FF0FF340FF6F6
S315080102800420D0E60D9AD317C0E90023EAE3D9F88A
S31508010290001051F8040BC9F8001020B94FF0FF34CB
S315080102A00FF6E010BFE60D990170DBE3D9F80010EF
S315080102B051F8040BC9F8001020B94FF0FF340FF6B6
S315080102C0C410B0E60D990160CCE39DF842004C28B4
S315080102D007BFD9F80010CB1DD9F80000C31D23F0BC
S315080102E00703C9F80030D3E900010833C9F800301B
S315080102F0CDE90201C80F02D007982D210AE0BDF801
S315080103004000810702D507982B2103E0C00705D5D0
S315080103100798202112AB1954401C079012A8079977
S31508010320DDE9024543184BF020006128059321AE0B
S315080103300BD00E98002802D506200E9005E001BFC5
S315080103404BF02000672801210E91DDE902014F00DB
S315080103507F1517F1010F0DD108030BD0ABF161021F
S3150801036003201A2A089002D20FF634110FE00FF66D
S3150801037034110CE017F1010F0ED109030CD1ABF1C1
S31508010380610203201A2A08901CD30FF620110322B2
S315080103901846F6F71FF865E3DDE902016A4604F037
S315080103A05DF9CDE902014BF02000612811D10598CC
S315080103B030210170821C0592BBF1610F0CBF7821B7
S315080103C0582102E00FF6E001E1E741700798801C29
S315080103D00790DDE9020120F0000231F0004308BF71
S315080103E0002A02D10025002445E14BF02008B8F186
S315080103F0610F40F095800E98002847BF2121019191
S31508010400401C0190019F7F1C20462946002200239B
S31508010410DDE9024504F05AF938BF85F0004500992F
S315080104208DF88420091F002F00910DF1850034DD18
S315080104300646204629460022002304F061F92BD2FC
S315080104401C2204F077F904460D4604F011FAFF1F41
S31508010450002F804609DD04F027FA02460B4620469E
S31508010460294604F0F1FA04460D46F01D0721B8F1B4
S31508010470000F0CDD491E5EBF08F00F0200F8012DC2
S315080104804FEA2818F3D502E0002200F8012D491E8B
S31508010490FAD5C61D002FCCDC30460DF18501401A70
S315080104A001990DF1850605468842C8BF0D46002DFE
S315080104B02FD4854206DA0DF18500415D0829A8BFCA
S315080104C00F2000DA0020294621AA0A4400E06D1E01
S315080104D012F80139491E8342F9D00F2804D10DF1CA
S315080104E08500425C521C4254002904D50098001D1F
S315080104F021AE6D1C0090681E0BD431180A78303273
S31508010500D3B23A2BA4BF5A443A3A401E01F80129FC
S31508010510F4D50E98002840F1AD80691E0E91A9E028
S315080105200099DFF8082747F29750414391FBF2F209
S31508010530009225F00045C2F10702002A04DD204693
S31508010540294600F04FFB0BE052420020DFF8E01687
S3150801055000F048FB02460B462046294604F0E6FA17
S3150801056004460D46B8F1660F06BF009F0A370627EF
S315080105700E983F18142FC8BF142730208DF8840011
S315080105800DF1850000E03046002F35DD0646204690
S31508010590294604F0EFFB01460A4606F10803042042
S315080105A00A26B2FBF6F606EB860EA2EB4E023032AF
S315080105B003F8012C0A22B6FBF2F202EB820EA6EB35
S315080105C04E063036401E03F8026DE9D1083F002F6A
S315080105D003F10806D7DD084604F0DEFB02460B46A2
S315080105E02046294604F030FA0022DFF8483604F09E
S315080105F0E1FB04460D46CAE70DF18501401A0DF1E6
S31508010600850604E00099491E401E0091761C317842
S315080106103029F7D0B8F1660F02D10099491C04E0D8
S31508010620B8F1650F0CBF012100210E9D4D19A84295
S31508010630B8BF451E002D1DD4854204DA705D3428E5
S31508010640C8BF392000DC30202946721E531800E045
S315080106506D1E13F80149491E8442F9D0392802D181
S31508010660705C401C7054002904D50098401C16463D
S315080106706D1C0090009C04F073FC406A0778DDF855
S31508010680388028B2002802DC01250FF224664BF0D7
S315080106902000662808BF641C16D0672846D120B2F8
S315080106A010F1040F48DB404546DA9DF84000641C0A
S315080106B0010703D428B24045D8BF804620B2B8EB1B
S315080106C0000848BF4FF000080FFA84FBBBF1000F82
S315080106D000F3B5800898411C0891302205990A54FF
S315080106E0B8F1000F03DC9DF84000010704D508980E
S315080106F0411C089105990F5418EB0B0FB8BFC8F1A7
S31508010700000424B26042A0442AB20B909045B8BFB7
S315080107104546059B08982DB209952A46314618443F
S31508010720F5F758FEA8EB05000C90D2E0BBF1610F76
S3150801073017D14FF0700B19E028B2404504DA9DF83D
S3150801074040100A0758BF8046B8F1010848BF4FF064
S315080107500008BBF1670F14BF4FF0450B4FF0650B4F
S3150801076004E0BBF1410F08BF4FF0500B0898411C3C
S315080107700891B8F1000F059916F8012B0A5403DC04
S315080107809DF8400001071AD50898411C0891B8F14F
S31508010790000F05990F5412DD6D1E28B28045B8BFAA
S315080107A045460598089B2AB231461844F5F712FEC4
S315080107B008992DB269180891A8EB05000B900598C0
S315080107C00899084421B2002980F800B003D42B22E5
S315080107D04270821C04E02D2242700C46821C64423F
S315080107E000212CAB20460AE004460A2094FBF0F0CF
S315080107F000EB8005A4EB450403F8014B491C00B244
S315080108000028F1DC012906DC4BF02000652804BF2D
S31508010810302002F8010B00292CAB08D1302002F850
S31508010820010B06E0491E585C303002F8010B00291D
S31508010830F8DC059908980844121A099249E028B281
S3150801084021B288421CDA0598089B2AB23146184417
S31508010850F5F7C0FD08992DB269180891ABEB0500AB
S31508010860B8F1000F0B9003DC9DF84000020704D590
S31508010870059847540999491C0991CDF8308028E013
S315080108800598089B22B231461844F5F7A3FD089846
S315080108902D1B5844B8F1000F089003DC9DF8401051
S315080108A00A0703D5411C089105990F5428B28045BA
S315080108B0B8BF45460598089B2AB206EB0B011844B2
S315080108C0F5F788FD08982DB228180890A8EB0500B9
S315080108D00B909DF8400000F01400102840F0C280EB
S315080108E0079A08990B988A18099982180C988A18F0
S315080108F082180F98824280F2B580821A0A92B1E074
S315080109009DF84200622808D068280ED06A2814D0BB
S315080109106C281FD0712810D01CE0D9F8001051F8A6
S31508010920040BC9F80010C0B21AE0D9F8001051F842
S31508010930040BC9F8001080B212E0D9F80000C21DF4
S3150801094022F00702C9F80020D2E900010832C9F8E5
S31508010950002006E0D9F8001051F8040BC9F8001078
S315080109600021CDE902019DF8400001075AD5DDE9CC
S315080109700223002B08BF002A54D04BF02000782808
S3150801098050D1079812A930220A54401C431C0793D8
S3150801099001F800B046E09DF84200622808D06828B0
S315080109A00ED06A2814D06C281FD0712810D01CE0EC
S315080109B0D9F8001051F8040BC9F8001040B21AE032
S315080109C0D9F8001051F8040BC9F8001000B212E06A
S315080109D0D9F80000C21D22F00702C9F80020D2E9A1
S315080109E000010832C9F8002006E0D9F8001051F8CC
S315080109F0040BC9F80010C117CDE90201002902D577
S31508010A0007982D210AE0BDF84000810702D507980D
S31508010A102B2103E0C00705D50798202112AA1154F6
S31508010A20401C079012A8079901440591594602A846
S31508010A3000F04EF816E001200790D9F8000050F8AA
S31508010A40041BC9F800008DF848100BE00121252286
S31508010A50BBF1000F07918DF8482003D002220792B7
S31508010A608DF849B00F9A07980A990C9C121A08989A
S31508010A70521A0B99121A0998521A121A9DF840001D
S31508010A80141B41073FF5E2AA2020002C8DF800002F
S31508010A907FF7DCAA309E2546FFF7CCBA4FF0FF3028
S31508010AA031B0BDE8F08F0000CBCCCC0C686A6C7411
S31508010AB07A4C00007072696E74665F733A206261DF
S31508010AC06420257320617267756D656E7400000078
S31508010AD02DE9FC4707468A463C6950466F2808BFF8
S31508010AE0082505D0FFF790F9782814BF0A2510259F
S31508010AF0D7E900013C2680468946BAF1640F18BF3A
S31508010B00BAF1690F05D1002903D5D8F1000869EBB7
S31508010B104909B9F1000F08BFB8F1000F0CD1386BBC
S31508010B2050B9082D3AD197F83800010736D5302241
S31508010B303B2684F83B2031E08DF800A04046494623
S31508010B402A46EB1702F010FB3032D0B2761E3A284D
S31508010B5001960EDAA255404649462A46EB1702F097
S31508010B6003FB80465FEA010908BFB8F1000F05D10A
S31508010B7008E09DF800001218513AEBE7F868A11948
S31508010B808842DBD3082D09D197F83800010705D526
S31508010B90A05D302802D0761E3020A055C6F13C0251
S31508010BA0BA61A119F960386B824208DA821A3A6287
S31508010BB04FF6EF70398F01403987BDE8F387002872
S31508010BC00ED597F8380000F01400102808D17B6B71
S31508010BD07969386A5B1A1B1A9A1A002AC8BF3A62D7
S31508010BE0BDE8F3872DE9D04306460F4614464FF074
S31508010BF00008DFF8449012E0E00707D542464B4665
S31508010C003046394604F0D6F806460F464046494668
S31508010C1042464B4604F0CEF8641080468946002CBD
S31508010C20EAD130463946BDE8D0830000A0860100E6
S31508010C300000F03F84D7974100002440F8B50546E7
S31508010C400E4617461C4600205CB117F8011BB06812
S31508010C50A847B06030B1F06A401CF0620020641EFB
S31508010C60F3D1F2BD4FF0FF30F2BD00007072696E2C
S31508010C7074665F733A20256E20646973616C6C6FC4
S31508010C80776564007072696E74663A2062616420E1
S31508010C90256E20617267756D656E7400000000002F
S31508010CA06E616E004E414E00696E6600494E460001
S31508010CB03000000038B504460D4600221021F8F729
S31508010CC0B3FD21460420F9F758FF002801D0296809
S31508010CD001600148E06031BD2CD2010870B50446B7
S31508010CE01D46DFF8AC022060DFF8A802006800287C
S31508010CF001D0204670BDDFF8A062304604F03EF907
S31508010D002946304604F0E9F9204670BD70B50C460F
S31508010D101546002605E0A15DDFF87C0204F060FABD
S31508010D20761CAE42F7D3284670BD10B5DFF86C4283
S31508010D302078C0070ED4204604F06CFA002809D0A2
S31508010D404FF4E1330A220921201DFFF7C7FF204688
S31508010D5004F06DFA201D10BD10B5044604F070FAB2
S31508010D60002807D1204604F06DFA002802D1BDE813
S31508010D701040DAE710BD10B5102801DB002010BDC0
S31508010D80DFF8081201EB8004216A11F1010F05D180
S31508010D90032803DAFFF7E0FF01462162084610BD82
S31508010DA000BF10B50446FFF7E6FF0021DFF8DC2196
S31508010DB002EB84021162002806D104F055FA0921D2
S31508010DC001604FF0FF3010BD01684969884704008A
S31508010DD006D504F049FA644204604FF0FF3010BDAD
S31508010DE0002010BD002070472DE9F04780460D46CA
S31508010DF01646B6F1004F06D304F036FA16210160FD
S31508010E004FF0FF304FE00024FFF7ECFF002831D008
S31508010E10DFF8787107EB080090F810A0A14627E0E3
S31508010E2015F809000A281FD150460D281CD04C4533
S31508010E300EDAA9EB04022919404600F036F8002813
S31508010E402DD404194C452DDB07EB080080F810A0BA
S31508010E50012224A1404600F028F800281FD421DDEC
S31508010E600D2007EB0801087415F809A009F1010915
S31508010E70B145D5DBB44215DA361B32462919404647
S31508010E8000F013F800280AD40419002C0ADD2819E1
S31508010E9010F8010CDFF8F4104144087402E04FF031
S31508010EA0FF3000E02046BDE8F08738B50C46154608
S31508010EB0FFF761FF002806D104F0D6F90921016080
S31508010EC04FF0FF3032BD2A4621460368DB68984752
S31508010ED0040005D504F0C8F9644204604FF0FF30F8
S31508010EE032BD00000D00000000BF38B50C4615469E
S31508010EF0FFF741FF002806D104F0B6F90921016080
S31508010F004FF0FF3032BD2A46214603681B699847D0
S31508010F10040005D504F0A8F9644204604FF0FF30D7
S31508010F2032BD1CB50146684604F0AAF904F0E4F995
S31508010F30040006D104F098F9132101604FF0FF303F
S31508010F4016BD684604F0C8F90146204622681269AA
S31508010F509047040006D504F087F9644204604FF00F
S31508010F60FF3016BD002016BD38B5054604F0DFF979
S31508010F70040007D10020009003462A4609A1084823
S31508010F80F9F79CFA204632BD04F05ABA60180020D7
S31508010F9064BF0108BC3A0020C03A00208C3F0020FB
S31508010FA01F0101804F70657261746F72206E6577DB
S31508010FB05B5D206F7574206F66206D656D6F727944
S31508010FC00D0A00004FF08070704720207047EFF33C
S31508010FD00580401E8041C043C00F7047EFF3108063
S31508010FE0002806D1EFF31180401E8041C043C00F8F
S31508010FF0704701207047000010B4024652E8000FFE
S3150801100000EA01038B4203D0BFF32F8F002005E0CE
S3150801101020EA010342E8003404B1EFE710BC704747
S3150801102010B4024652E8000F084203D1BFF32F8FCE
S31508011030002005E020EA010342E8003404B1F1E7A3
S3150801104010BC70477047704770477047DFF87C07D8
S31508011050007A7047DFF8740740697047DFF86C1744
S3150801106048617047930705D4D20701D52830C3E7ED
S315080110702830D5E7806AD30703D501EA00038B42F6
S3150801108003D1D20702D4084200D10020704738B5EF
S315080110900C4694F92050FFF7D7FF816801E008460E
S315080110A08968002903D091F92020AA42F7DAE0607D
S315080110B0A1608460002900D0CC6031BD10B5846878
S315080110C0A1688160A168002903D0FFF7BDFFA16867
S315080110D0C8600020E060204610BD00E0C0680178C5
S315080110E0F129FBD0704738B5054600E0C0680028ED
S315080110F002D00178F129F9D0FFF7A5FF040007D03E
S31508011100284600F006F829462046BDE83440BEE7E1
S3150801111031BDC168002908D082688A6081680029C2
S3150801112001D0C268CA600021C1607047014601202A
S315080111304870DFF89C06AAE730B4DFF8904611F14B
S31508011140010F12D10022216B01E00A460969002923
S31508011150FBD14FF0FF31C161426100210161002AD3
S3150801116001D010611AE0206318E00023E26A02E068
S31508011170491B13461269002A02D0D569A942F7D23A
S31508011180C16143610261002B01D0186100E0E06290
S31508011190002A03D0D369591AD161506130BC70470E
S315080111A00169C26912F1010F0BD1002901D0426907
S315080111B04A61416900290FD10169DFF810261163D7
S315080111C014E0002905D0CB69D218CA6141690269C0
S315080111D051614169002905D00169426911610021FE
S315080111E0416103E00169DFF8E425D1620021C161AB
S315080111F0704738B5DFF8D455EC6A002C4AD0E06957
S31508011200401EE06146D1607843280AD053280ED0A3
S31508011210632817D073281BD083281FD0932823D07F
S3150801122027E02046FFF759FFFFF70DFF21E020468B
S31508011230FFF753FFFFF707FFFFF707FF214600F008
S315080112404CFE16E02046FFF748FFFFF7FCFE10E0CC
S315080112502046FFF742FFFFF7F6FE0AE02046FFF7B2
S315080112603CFFFFF7F0FE04E02046FFF736FFFFF7E5
S31508011270EAFE2046FFF74DFF2046FFF757FF246990
S31508011280002C02D0E0690028BDD0002C01D0002036
S315080112906061EC6231BD10B5044694F82200FFF78F
S315080112A094FEA16B401810BD38B504460120607044
S315080112B094F92050DFF81805FFF7C6FE816801E0AA
S315080112C008468968002903D091F920209542F7DB61
S315080112D0E060A1608460002900D0CC6031BD0221A4
S315080112E04170DFF8E8148861704770B50446FFF766
S315080112F0ADFE0646FFF7AEFE0546002C16D1DFF811
S31508011300CC04446A022E24D1002C22D095F920005F
S3150801131094F9201088421CDA2046FFF7FAFE28467F
S31508011320FFF7C2FF2046BDE87040D8E7022E0CD170
S3150801133095F9200094F92010884206DA2846FFF725
S31508011340B3FF2046BDE87040C9E72046BDE87040B6
S31508011350ECE670BD70B504460D461646FFF79BFFD1
S3150801136005602046FFF71CFF002E204602D0BDE887
S315080113707040BAE7BDE87040D8E670B504460D4638
S31508011380FFF764FE022801D0002070BDDFF83C6437
S31508011390706A002801D1002070BDFFF75BFE44701A
S315080113A02946FFF7C9FE06F11C00FFF787FEFFF77E
S315080113B096FF012070BD016B806B814204D20868DB
S315080113C0DFF8CC14884201D000207047012070470D
S315080113D010B50446607833280CD194F82320616A45
S315080113E02046FFF73FFE010004D000222046BDE853
S315080113F01040AFE710BD2DE9F34F81B080460028B4
S3150801140006D16FF00301002004F01CF80020F7E074
S31508011410002A2ED0D2F80090506800909468156979
S3150801142056699769002C10D014F0030010D1D068C2
S3150801143044280DD3002D04D015F007002CD1002E19
S315080114402AD0002F0BD118271BE0D0680028F1D02D
S315080114506FF00801002003F0F5FF0020D0E0781EA8
S3150801146038280ED36FF00B01002003F0EBFF0020A4
S31508011470C6E04FF000094846009004460546064670
S315080114801827002E0FD016F0070F05D1A6F1480030
S31508011490DFF83414884206D36FF00A01002003F0FE
S315080114A0D1FF0020ACE0002C14D1DFF8203303F182
S315080114B084004068002803D000F0ACFA044606E030
S315080114C001224421D3F8800001F0ADFC04464FF017
S315080114D0010B01E04FF0000B002C2FD0002D2DD170
S315080114E0DFF8E8A2002E0DD1DFF8E003466DDAF841
S315080114F08400002806D000F08DFA050009D04BF0CB
S31508011500100B06E000223146DAF8740001F08BFC74
S315080115100546002D10D15846C0070CD50AF184009E
S3150801152040680028214602D000F084FA03E0DAF880
S31508011530800001F0D5FC00244BF0020B002C54D09E
S31508011540F12020700120607084F802B00098E070E4
S31508011550C4F804900020A060E06020616061A06189
S31508011560E06184F8207004F121000770FD214170C3
S315080115700021817004F12401002008604860886018
S31508011580CD600E6170194038486142468A61DFF8BC
S3150801159000032860DFF834030068430708D5B60856
S315080115A0113E4FF0CC3302E045F8043F761EFBD1DD
S315080115B04D6900210B4602E045F82130491C0D29E9
S315080115C0FAD1029E0FF2B1216963AA6308F00108F4
S315080115D0414600F00100FFF7F5FCE8632E62DFF8EB
S315080115E0F002DFF8E811086604E06FF00401002054
S315080115F003F028FF002C02D02046FFF776FE20468E
S31508011600BDE8FE8F26E510B50446A069002803D07B
S3150801161000221146FFF79EFE6078232802D100209A
S31508011620A168886110BD10B504460020607020705D
S31508011630A07881070CD5216BDFF89822C00604D55E
S31508011640D2F8840000F0F6F902E0506F01F048FC88
S31508011650A078C00711D5DFF87C2202F18400406822
S315080116600028214603D0BDE8104000F0E3B9D2F8BE
S315080116708000BDE8104001F033BC10BDC178C90730
S3150801168000D4D0E7042141700021C160DFF844226B
S31508011690516B8160516B002900D0C8605063704757
S315080116A038B5FFF7D3FC022829D1DFF82842606A4A
S315080116B0002824D0FFF7CEFC0546E86A00F0E8FBCF
S315080116C02846FFF7A0FF04F11C00FFF7F7FCFFF718
S315080116D006FEEFF30980A8632846FFF76CFE00288B
S315080116E006D1A069FFF7BAFC29460120F7F74BFF97
S315080116F00020FFF7B3FC2846BDE83240BEE731BDFE
S3150801170070B5FFF79FFC040002D02078F12807D0B6
S315080117106FF003052946204603F094FE284670BD5E
S31508011720607800F00F0001280ED01AD3032810D0D4
S3150801173017D2FFF78BFC022813D1DFF89801406A0C
S3150801174000280ED0002512E02046FFF7E2FC00250E
S315080117500DE02046FFF7DDFC2046FFF721FD0025B9
S3150801176005E06FF002052946204603F06BFE002DC1
S3150801177029D1E06A00F08CFB2046FFF744FF607828
S3150801178002281AD1DFF84C6106F11C00FFF796FC16
S31508011790FFF7A5FDEFF30980A0632046FFF70BFECF
S315080117A0002806D1B069FFF759FC21460120F7F751
S315080117B0EAFE0020FFF752FC02E00020FFF795FD44
S315080117C02046FFF75BFF284670BD0000241A00205B
S315080117D0401A002070B50024DFF8F050AA6D2146A2
S315080117E0DFF8F400FFF707FEDFF8E860FFF72AFCE9
S315080117F0B062686E00280ED0804700280CD1EA6DC9
S31508011800F16C286EFFF7F7FDFFF71CFCB0640028A2
S3150801181002D0012400E00124204670BD000000002A
S3150801182070B504460D461646FFF7D1FB002803D1CD
S31508011830FFF7D4FB002806D06FF00501002003F05E
S3150801184001FE002070BDDFF8940084463246294621
S31508011850204600DF70BD000080B5FFF7B8FB002801
S3150801186003D1FFF7BBFB002802D0BDE80140C9E65A
S315080118701B48844600DF02BD00F094F919488446E6
S3150801188000DF4FF0FF31002003F0DCFDFEE700002A
S31508011890A52E5AE238B5044600F08AF9FFF797FBF8
S315080118A0002803D1FFF79AFB002806D06FF005053B
S315080118B02946204603F0C6FD04E00B488446204627
S315080118C000DF0546284632BDB8FFFF7F18BE01086E
S315080118D0D1130108241A0020ED1A0108F71301088B
S315080118E005160108A116010801170108F8F7C4BB76
S315080118F003F0A9BD70B5054608461146049C059A2C
S3150801190003F00F062E73AC736A7328601A46281DF6
S31508011910F4F760FD284670BD704770B504460D465C
S31508011920002C07D014F0070004D115F0070F01D1D8
S31508011930182D01D2002070BD204603F097FD0560E1
S31508011940102141600821204603F091FD0646083D15
S315080119502946204603F08BFD306000203168086077
S3150801196010203168486000207060012070BD0000B9
S31508011970014651E8000F421C41E8002303B1F8E78C
S3150801198070470000014651E8000F421E41E8002356
S3150801199003B1F8E770470000014651E8000F10B996
S315080119A0BFF32F8F04E0026841E8002303B1F4E78F
S315080119B07047000010B402680A60BFF35F8F50E8F1
S315080119C0002F0B689342F6D140E8001404B1F2E700
S315080119D010BC704710B4002805D0002903D0002A8E
S315080119E001D0002B01D1002012E0016000244460DF
S315080119F08260C360436102FB01F41C44046102E096
S31508011A00981818600346491EFAD10020186001206B
S31508011A1010BC704738B5050001D1002032BD05F16B
S31508011A201400FFF7B9FF040002D0281DFFF7A0FF35
S31508011A30204632BD10B5040006D00846E268904239
S31508011A4002D32269904202D36FF0030010BD04F15C
S31508011A501400FFF7AFFF201DFFF794FF002010BD0C
S31508011A60002802D14FF0FF3070470B490968B1FBD6
S31508011A70F0F0401EB0F1807F02D34FF0FF3070477F
S31508011A80FF21064A1170064906220A6048600020AD
S31508011A908860044908707047F018002023ED00E0BB
S31508011AA010E000E05A4000204FF0FF307047000078
S31508011AB007490878002805D0002008704FF0806093
S31508011AC0044908600448016841F001010160704752
S31508011AD05A40002004ED00E010E000E070470000E5
S31508011AE024490968002900D00847704703F0D0FC4B
S31508011AF000BF000082B00246401E042831D8DFE844
S31508011B0000F0030C151E2700002000900346012251
S31508011B1019491A48F8F7D2FC2AE000200090034632
S31508011B20022217491748F8F7C9FC21E0002000905E
S31508011B300346032214491548F8F7C0FC18E00020AB
S31508011B4000900346042212491248F8F7B7FC0FE041
S31508011B5000200090034605220F491048F8F7AEFC0D
S31508011B6006E000200090034612A10D48F8F7A6FCEE
S31508011B70FEE70000DC3F002038AA010825010280A3
S31508011B805CAA01082601028084AA010827010280AD
S31508011B90BCAA010828010280F8AA01082A010280C4
S31508011BA00001028080B5FFF757FEBDE8024097E7BE
S31508011BB096E70000434D5349532D52544F53206520
S31508011BC072726F723A20556E6B6E6F776E000000F7
S31508011BD0704700F5A0614A88104609880B4691426C
S31508011BE001D3181A7047C0F1400018187047EFF36F
S31508011BF0108000F0010080F001007047010007D451
S31508011C00012200F01F018A405149400941F820206C
S31508011C107047504A1268103002EB80021160704713
S31508011C20416941F0020141617047000053A07047C4
S31508011C3049484A4908600169890707D5C16889077A
S31508011C4004D56FF002010161F8F764BC70471CB551
S31508011C504348C16841F00401C160C16801F004014B
S31508011C6000910099016841F004010160016821F0C1
S31508011C700401016003F012FC384C374820604FF626
S31508011C80FF70E060374800683749B0FBF1F0401E45
S31508011C90606000202061A0606061A061204603F0B9
S31508011CA039FC0021204603F05BFC30491E20FFF772
S31508011CB0B0FF1E20FFF7A2FF204603F044FC206870
S31508011CC0C16821F00201C16000202949086029493B
S31508011CD0086013BD21480168CA6822F00202CA6079
S31508011CE0002103F03DBC2448006870471B490A6877
S31508011CF050636FF002000A6810610868C16841F014
S31508011D000201C160704710B5144C6FF002002168DA
S31508011D1008612068FFF784FF2068C16841F0020165
S31508011D20C16010BD0D480068C16821F00201C1609B
S31508011D3070476FF00200094909680861704780B564
S31508011D400021064803F022FCBDE80140EAE700004D
S31508011D5000E100E008ED00E000080040F83B002043
S31508011D6010100240F018002040420F00311C0108F3
S31508011D70843F0020883F00202408004040420F008D
S31508011D8010000000284803F0FABD284803F0F7BD03
S31508011D90274803F0F4BD244803F0F7BD234803F0B0
S31508011DA0F4BD234803F0F1BD70B51F4D2868F0B1A5
S31508011DB003F056FE0446002003F054FE012C0646A5
S31508011DC005DB304603F020FE361D641EF9D1284690
S31508011DD003F0CCFD281D03F0C9FD05F1080003F049
S31508011DE0C5FD05F10C00BDE8704003F0BFBD70BD2F
S31508011DF070B500240C4D05EB840003F091FD641CBD
S31508011E00042CF8DB03F02CFE0546002003F02AFE1D
S31508011E100646002404E006EB840003F0BBFD641CBF
S31508011E20AC42F8DB70BD0000603F0020643F002033
S31508011E306C3F0020002800D1704780B503F012FEE0
S31508011E40BDE8024003F0E9BD002800D1704780B51E
S31508011E5003F008FEBDE8024003F0E5BDEFF3058097
S31508011E60401E8041C043C00F7047EFF31080002821
S31508011E7006D1EFF31180401E8041C043C00F704761
S31508011E800120704770477047DFF85C044069704766
S31508011E9070B504001FE06569E07800071AD50020CF
S31508011EA02076A068002815D02046FFF7ECFFFFF73B
S31508011EB005F9064600221146FFF74CFAE6600020AE
S31508011EC02061F06A6061F06A002800D00461F4625A
S31508011ED0012020762C00DED170BDC278920700D48D
S31508011EE0704718B4C06890F92140C36ADA78920736
S31508011EF00AD59A688A4200D19268002A04D092F9D2
S31508011F002020A24200DB14465B69002BEED190F932
S31508011F1020102246914204D080F8204012BCFFF7D7
S31508011F20E2B811BC704770B5002815D00568466837
S31508011F308468002C06D014F0030106D1C0681C2859
S31508011F400DD202E0C068002809D06FF00801002010
S31508011F5003F092FD002070BD00252E462C46002C6C
S31508011F6010D1DFF888335869002803D0FFF752FDEE
S31508011F70044605E001221C21186800F054FF0446B6
S31508011F80012000E00020002C0BD0F5212170A07063
S31508011F90E67065600020A060E060206160612076DF
S31508011FA004E06FF00401002003F066FD204670BDD1
S31508011FB070B50C46FFF766FF0646FFF765FF050095
S31508011FC007D16FF00701304603F056FD4FF0FF3099
S31508011FD070BD002E02D03078F52807D06FF00304C3
S31508011FE02146304603F048FD204670BD307E002864
S31508011FF00DD1F56000203061E86A7061E86A002851
S3150801200000D00661EE6201203076002070BDF178BD
S31508012010CA0710D5F268AA420DD1FF2807D16FF079
S315080120200F01304603F028FD6FF0020070BD401C19
S315080120303076002070BD002C1CD088070BD595F989
S315080120402000F16891F92020824204DA81F8200003
S31508012050F068FFF748F821465320FFF78EF9002864
S3150801206005D03046FFF70FFF2946FFF710F86FF046
S31508012070010070BD6FF0020070BD38B5FFF702FFB1
S315080120800446FFF701FF020007D16FF0070120465A
S3150801209003F0F2FC4FF0FF3032BD002C02D020785D
S315080120A0F52807D06FF003052946204603F0E4FC1E
S315080120B0284632BD207E002807D16FF00E01204642
S315080120C003F0DAFC6FF0020032BDE168914207D0F5
S315080120D06FF00D01204603F0CFFC6FF0020032BD10
S315080120E0401E2076C0B200283BD16069002801D085
S315080120F02169016161692069002801D0416100E017
S31508012100D16292F92130D16A0BE0C878800707D5E8
S315080121108868002804D090F92000984200DB03461D
S3150801212049690029F1D182F82030A068002815D024
S315080121302046FFF7A8FEFEF7C1FF05460022114615
S31508012140FFF708F9E56000202061E86A6061E86A3E
S31508012150002800D00461EC62012020760020FFF7F8
S31508012160C4F8002032BD38B5FFF78CFE040002D052
S315080121702078F52807D06FF003052946204603F095
S315080121807BFC284632BD207E002839D0E26860698A
S31508012190002801D02169016161692069002801D0FF
S315080121A0416100E0D16292F92130D16A0BE0C87829
S315080121B0800707D58868002804D090F9200098423E
S315080121C000DB034649690029F1D192F92000194635
S315080121D088420FD082F820301046FEF784FF09E0C6
S315080121E02046FFF750FEFEF769FF00226FF0020155
S315080121F0FFF7B0F8A0680028F2D10020FFF775F8BC
S3150801220000202070A078C0070AD5384A50690028EE
S31508012210214602D0FFF70EFC02E0106800F060FECE
S31508012220002032BD0000000010B50446FFF716FE77
S31508012230002803D1FFF719FE002806D06FF0050123
S31508012240002003F019FC002010BD294884462046C9
S3150801225000DF10BD38B504460D46FFF7FFFD00281F
S3150801226003D1FFF702FE002806D06FF005052946BF
S31508012270204603F001FC05E01E488446294620460F
S3150801228000DF0546284632BD38B50446FFF7E6FDA8
S31508012290002803D1FFF7E9FD002806D06FF00505F0
S315080122A02946204603F0E8FB04E013488446204605
S315080122B000DF0546284632BD38B50446FFF7CEFD90
S315080122C0002803D1FFF7D1FD002806D06FF00505D8
S315080122D02946204603F0D0FB04E0084884462046F8
S315080122E000DF0546284632BD241A0020A41A00201C
S315080122F0271F0108B11F01087B2001086721010872
S3150801230078B58DB004460D46002C00D4704C129E4B
S31508012310002234216846F7F787FA00940196029558
S315080123206C4840690390C16B0491416B0591006B40
S31508012330069068460790F4F7D7FC674C6068401C1E
S315080123406060012805D13422694604F10800F4F7D2
S3150801235041F83422694604F13C00F4F73BF8216F51
S31508012360002902D004F13C008847F4F7CEFC00208E
S315080123700EB070BD0020704757480078704700209E
S3150801238070470000002800D155A070472DE9FE438B
S3150801239005460E4614461F462968C1F341700328AF
S315080123A002D1C1F1000901E01FFA81F9DFF82C8198
S315080123B0C1F307434A46404603F060FB40F2311039
S315080123C0B9EB000918D0B9F101091BD0B9F1010916
S315080123D01ED0B9F1010921D0B9F1010924D0B9F109
S315080123E001092DD0B9F1010924D0B9F101092DD07E
S315080123F0B9F10C0930D032E0D5F808103BA003F04A
S315080124003DFB2CE0D5F808103EA003F037FB26E08B
S31508012410D5F808103FA003F031FB20E0D5F80810E5
S3150801242040A003F02BFB1AE0D5F8081042A003F0F0
S3150801243025FB14E0D5F8081044A003F01FFB0EE0B5
S31508012440D5F8081046A003F019FB08E0D5F80810DE
S3150801245047A003F013FB02E04BA003F00FFB304645
S3150801246003F02CFBD5F804104CA003F007FB002C55
S315080124700AD000BF4DA003F021FB204603F01EFB46
S31508012480394612A003F0FAFAD5F8081049A003F064
S31508012490F5FAE8684068FFF775FFE9690291A969E5
S315080124A00191696900912B69EA68014608F15400AE
S315080124B003F0E4FA296808F1A80003F0DFFA00BF7F
S315080124C041A0BDE8FE4303F0D9BA00002B256400FC
S315080124D00101FF80241A00209827002038AB010843
S315080124E03C756E6E616D65643E0000004B65726EEB
S315080124F0656C204572726F723A20307825582C2007
S31508012500000000005468726561643A2030782558E5
S315080125102C2000004D757465783A20307825582CA2
S315080125202000000053656D6170686F72653A20304E
S315080125307825582C200000004D656D6F7279506F13
S315080125406F6C3A20307825582C2000004576656E48
S3150801255074466C6167733A20307825582C20000040
S3150801256054696D65723A20307825582C2000000090
S315080125704D65737361676551756575653A20307880
S3150801258025582C2000000000417373657274696F29
S315080125906E206661696C65643A2000000A4C6F63B7
S315080125A06174696F6E3A2030782558000A46696C5D
S315080125B0653A20000A4572726F722056616C75651C
S315080125C03A203078255800000A2D2D204D62656481
S315080125D04F53204572726F7220496E666F202D2DFA
S315080125E00A00000038B504460D4600221021F7F707
S315080125F01BF9EA68002A03D0294620465268904703
S31508012600E868E060204632BD2DE9F0410446002520
S315080126102F46002C01D101208BE004F13C063078CD
S31508012620002804D128467070204603F063FA022078
S3150801263030702068016821F0020101602068016894
S3150801264041F001010160F7F77AF880462068416890
S31508012650C9070BD4F7F773F8A0EB08000B28F5D3D5
S315080126600320307028467070032062E04168C9076C
S3150801267054D5A169012901D180210F46E1690129B2
S3150801268002D147F0400701E027F04007216A0129F6
S3150801269002D147F0200701E027F02007616A0129E6
S315080126A002D147F0100701E027F01007A16A0129B6
S315080126B002D147F0080701E027F00807E16A012976
S315080126C002D147F0040701E027F00407016821F069
S315080126D0FC010F430760A168E068014320690143D3
S315080126E0606901436068401E01432068C161206832
S315080126F00168490849000160F7F721F8074620688B
S315080127004168C90705D5F7F71AF8C01B0B28F6D390
S31508012710A6E74068C00701D401200546012D05D169
S315080127200020706001203070002002E00420307023
S315080127300120BDE8F08170B401224B6902FA03F366
S315080127400268D2F8004224F47C544D6A44EA05240E
S3150801275044F00104C2F80042DC430268D2F81C5274
S315080127602540C2F81C52CA69002A1BD10268D2F850
S315080127700C522540C2F80C5202684D6902EBC5029B
S31508012780CD684E68B6B246EA0546C2F840620268A6
S315080127904D6902EBC5028D680E68B6B246EA054672
S315080127A0C2F84462CA69012A1BD10268D2F80C52DE
S315080127B01D43C2F80C5202684D6902EBC5020D6849
S315080127C04E68B6B246EA0546C2F8406202684D69E5
S315080127D002EBC5028D68CE68B6B246EA0546C2F86E
S315080127E0446205688A69002AD5F8042203D1224081
S315080127F0C5F8042202E01A43C5F8042205680A69E5
S31508012800002AD5F8142203D11440C5F8144202E06F
S315080128101A43C5F81422096A012905D10168D1F8B4
S315080128201C221343C1F81C320068D0F8001249086B
S315080128304900C0F80012002070BC70470EB43CB5C0
S315080128400446104D0121284600F074FC002816D1D3
S31508012850002000900346024601460B48FFF750FD4B
S3150801286000231A46094905F13C00FFF78FFD05A922
S31508012870204603F00BF90021284600F05BFC33BC27
S315080128805DF810FB982700200001FF80CCCE0108D7
S315080128901CB504464FF0FF32904201D113BD0C31ED
S315080128A0B1F9000010F1010F0CD022469042F6D181
S315080128B08968204600F0C0F900212046BDE81C4081
S315080128C000F020BA002000900346224638A1374876
S315080128D0F7F7F4FD13BD0000884200D1704780B5B3
S315080128E010F1010F01D1084602BD11F1010F09D0FE
S315080128F0002100910B46024632A12C48F7F7DEFD6E
S315080129004FF0FF3002BD034600E00C31B1F900205B
S3150801291012F1010F03D09A42F7D1486870474FF078
S31508012920FF3070471CB502464FF0FF339A4201D17A
S31508012930184616BDFFF7E7FF044614F1010F09D142
S31508012940002000904FEA00034FF0FF3222A11748FA
S31508012950F7F7B4FD204616BD034600E00C31B1F980
S31508012960002012F1010F03D09A42F7D18868704707
S315080129704FF0FF30704700001CB502464FF0FF3399
S315080129809A4201D1184616BDFFF7E6FF044614F12F
S31508012990010F09D1002000904FEA00034FF0FF32E2
S315080129A015A10248F7F78AFD204616BD30010180B8
S315080129B0636F756C64206E6F742070696E6F7574C1
S315080129C00000000070696E6D6170206D69732D6D70
S315080129D0617463680000000070696E6D6170206E35
S315080129E06F7420666F756E6420666F7220706572EB
S315080129F06970686572616C0070696E6D6170206ED0
S31508012A006F7420666F756E6420666F722066756EC8
S31508012A106374696F6E00000010B400EB116091FADF
S31508012A20A1F1B1FA81F1890003680F248C40A3430F
S31508012A308A401A43026010BC704791FAA1F2B2FAB1
S31508012A4082F2920000EB116000680F219140084064
S31508012A50D040704710B400EB116091FAA1F1B1FAB8
S31508012A6081F18900036803248C40A3438A401A43F1
S31508012A70026010BC704710B400EB116091FAA1F125
S31508012A80B1FA81F18900036804248C40A3438A4082
S31508012A901A43026010BC7047C368090A8B4391FA4E
S31508012AA0A1F1B1FA81F18A401A43C260704781B037
S31508012AB0BA490A6842F001020A60096801F001018F
S31508012AC00091009901460D2901D00E2906D1B44974
S31508012AD00A6822F0E06242F080620A6001460F2924
S31508012AE003D0132901D0142806D1AD48016821F075
S31508012AF0E06141F00071016001B0704781B0A748FB
S31508012B00016841F001010160006800F001000090D0
S31508012B100098002A60D0521E092A5DD8DFE802F023
S31508012B20050D151D252F39434B539D48016841F065
S31508012B30E06141F0010101604EE09948016841F008
S31508012B40E06141F00201016046E09548016841F003
S31508012B50E06141F0040101603EE09148016841F0FD
S31508012B60E06141F00801016036E08D48016821F015
S31508012B70300141F0E06141F0100101602CE0884824
S31508012B80016821F0C00141F0E06141F040010160B6
S31508012B9022E08348016821F4406141F0E06141F493
S31508012BA00061016018E07E48016841F0E06141F486
S31508012BB04071016010E07A48016841F0E06141F432
S31508012BC04061016008E07648016821F4C04141F09E
S31508012BD0E06141F48041016001B0704770B5044677
S31508012BE00D461646FFF729FF012E02D0022E0DD0FB
S31508012BF019E0042804D1082229462046FFF70CFFCC
S31508012C00012229462046BDE8704045E7042804D13B
S31508012C10082229462046FFF7FFFE002229462046BC
S31508012C20BDE8704038E7082805D104222946204620
S31508012C30BDE87040F0E670BD2DE9F84F04460F4631
S31508012C40DFF860814FF0FF31884206D15FF03E021E
S31508012C5008F1400154A0F6F749FD07F00709C7F343
S31508012C60032A00F00F0158F821504FF0000BC0F36A
S31508012C70031001F0DFFB0646B9F1010F03D1032268
S31508012C802946FFF7E7FE4846032825D8DFE800F07E
S31508012C9002191C044FF0080B5A4629463046FFF71D
S31508012CA0BBFEB9F1010F02D0B9F1020F1FD1C7F36B
S31508012CB0C000002816D0042229463046FFF7DBFE5D
S31508012CC015E04FF0010BE7E74FF0090B5246214695
S31508012CD03046FFF713FFDFE76D2208F140012EA00A
S31508012CE0F6F704FD002229463046FFF7C4FEC7F36E
S31508012CF0011229463046FFF771FF2046BDE8F24F1B
S31508012D00D5E6000070B50C46264902464FF0FF335A
S31508012D109A4204D18E22403123A0F6F7E7FC00F04F
S31508012D200F0251F82250C0F3031001F083FB064647
S31508012D302946FFF782FE012801D0092811D120462C
S31508012D40042803D0032801D0052805D104222946E1
S31508012D503046FFF790FE04E0002229463046FFF789
S31508012D608AFE2046032801D0012805D101222946D9
S31508012D703046BDE8704031E7052801D0022C05D15F
S31508012D80022229463046BDE8704027E70022294637
S31508012D903046BDE8704021E73000000018100240B7
S31508012DA004000140CCB8010870696E20213D202835
S31508012DB050696E4E616D65294E430000C0E90023D6
S31508012DC08160704738B504460D4600221021F6F792
S31508012DD02BFD21460C20F7F7D0FE002803D095E8F5
S31508012DE00E0080E80E000148E06031BD38D20108C6
S31508012DF0C0E900238160704738B504460D460022B4
S31508012E001021F6F711FD21460C20F7F7B6FE00282A
S31508012E1003D095E80E0080E80E000148E06031BD58
S31508012E2044D2010870472DE9F04105460C4617467C
S31508012E30002D43D0002C41D0B80880003ED10F3474
S31508012E40E4080821284602F012FB06463068811B71
S31508012E5072689208B1EB8201B1EBC40F04D206463F
S31508012E6030680028F2D129E0284602F0FFFA4168C5
S31508012E7011EBC4014160284602F0F8FA01680839E5
S31508012E80284602F0F4FA8046284602F0EFFAD8F806
S31508012E9004104068814205D2284602F0E7FA4068E4
S31508012EA0C8F8040057EAC4047168002908D1746097
S31508012EB008213046BDE8F04102F0D9BA00200DE0FC
S31508012EC089088900304602F0D2FA31680160446007
S31508012ED030600821BDE8F04102F0C9BABDE8F081C9
S31508012EE0F8B506460846002E12D0002810D0002153
S31508012EF002F0BDFAA0F1080700250821304602F0C4
S31508012F00B6FA0446BC4205D025462468002CF9D1F8
S31508012F100020F2BD304602F0A9FA416862689208BB
S31508012F20B1EB82014160002D02D10020606001E011
S31508012F30206828600120F2BD4FF080507B49086067
S31508012F407047000010B40246D2E85F0F814202D8EA
S31508012F50BFF32F8F04E0431CC2E8543F04B1F3E7E3
S31508012F6080B210BC7047000010B40246D2E85F0F69
S31508012F70431C994200D80023C2E8543F04B1F5E73F
S31508012F8080B210BC704700000146D1E85F0F10B946
S31508012F90BFF32F8F04E0421EC1E8532F03B1F4E7B4
S31508012FA080B27047704770477047704770477047DF
S31508012FB05F48007A7047F8B504465D4D05F1540639
S31508012FC03788394605F15600FFF7BCFF394688426E
S31508012FD008D205F15800FFF7C7FFB16841F820404C
S31508012FE00120F2BD0020F2BD70B5514C04F1540523
S31508012FF02E8804F15600FFF7C7FF00280AD031468C
S3150801300004F15A00FFF7B0FFA96851F82000BDE89E
S315080130107040C7E7002070BD38B502F06DFD444D1C
S31508013020E868401CE860FEF7E4F80020FEF75DF961
S31508013030286D002800D08047296C00292AD0AA6962
S31508013040E86B824204D0EA63D069002800D1D161D5
S31508013050D069002801D0401ED061D069002819D155
S31508013060FFF7A6FF022815D16C6A002C12D094F935
S315080130702000E96B91F9201088420BD12046FEF712
S3150801308048F8E86BFEF752F82046FEF728F9EC6394
S31508013090286CE06131BD80B504E0FFF784FF24495F
S315080130A0096E8847FFF7A0FF002811D00178F1299A
S315080130B0F3D0F32911D0F62904D0F72913D0F92929
S315080130C017D0EFE7FFF771FF1949896E8847E9E7D6
S315080130D00020BDE80240FEF708B9FFF765FF14496D
S315080130E0496E8847DEE7FFF761FF1149C96E8847D0
S315080130F0D8E7FFF75CFF0E49096F8847D2E710B595
S315080131000446FFF758FF002809D00949487A0028DC
S3150801311002D1BDE810400FE70120887210BD214693
S315080131200220BDE81040F6F72EBA000004ED00E0D3
S31508013130241A00200246D2E84F0FC2E8431FC0B244
S3150801314070470000D2B2203A22BF00FA02F10020ED
S3150801315070475242D041D2F1200291404140D040BD
S315080131609040414070470000BBBBE1B1B2F5803FDA
S3150801317080F07E80022A1ED98C46B1FBF2F102FB51
S3150801318011C31B0443EA1043B3FBF2FC02FB1C33D5
S3150801319080B240EA0343B3FBF2F002FB103240EA85
S315080131A00C4000237047022A05D98446B0FBF2F089
S315080131B002FB10C270474AB105D100F00102490865
S315080131C05FEA3000704700220023704702F09ABC7C
S315080131D00B000200002100207047904271EB030C9E
S315080131E0F6D3B3F5803F2FD2F0B5B3FA83F7B1FA28
S315080131F081F4A7F10F0E3D1B5340CEF1200602FACA
S315080132000EF2F3415340B5F10F0746D80F3C2C4453
S315080132104140C4F12006A040F1414140B1FBF3F61B
S3150801322003FB1611A2FB0645001BA94102D2761E15
S315080132308018594180EA010221FA0EF362FA0EF268
S3150801324000215A403046F0BD30B4B1FBF3FC03FB14
S315080132501C11A2FB0C45001BA94103D2ACF1010CC0
S315080132608018594130BC02460B466046002170471A
S31508013270B2F1807F65D3F0B5B2FA82F7B1FA81F47B
S31508013280C7F10F063D1B22FA06F307F1110EF241AB
S3150801329020355A40B5F10F07B8D94140C4F1200687
S315080132A0A040F1414140B1FBF3FC03FB1C11A2FB19
S315080132B00C45001BA94103D2BCF1010C80185941E8
S315080132C00F2F12D30F3FC90341EA5041B1FBF3F661
S315080132D003FB1611A2FB0645D4EBC030A94102D265
S315080132E0761E8018594146EACC3C07B34140C7F1DE
S315080132F02006B840F1414140B1FBF3F603FB161134
S31508013300A2FB0645001BA94102D2761E8018594127
S3150801331080EA010221FA0EF3C7F1200462FA0EF2DD
S315080133200CFA07F05A402CFA04F13043F0BD80EA52
S31508013330010221FA0EF3002162FA0EF260465A40A2
S31508013340F0BD8C46B1FBF2F102FB11C31B0243EA45
S315080133501063B3FBF2FC02FB1C331B024CEA002090
S3150801336043EA1063B3FBF2FC02FB1C331B024CEA73
S31508013370002043EA1063B3FBF2FC02FB1C331B0279
S315080133804CEA002043EA1063B3FBF2FC02FB1C3251
S315080133904CEA002000237047D2B2203A22BF21FA14
S315080133A002F0002170472032D141D0404840914077
S315080133B0D1404840704710B5044621600846F6F7E3
S315080133C07FFA204610BD000010F0004C68B148BFD6
S315080133D04042B0FA80F18840D1F19D014CEAC15CC6
S315080133E0010671F100414CEB1020704750B1B0FA5B
S315080133F080F18840C1F19D01C905020672F10042BA
S3150801340041EB1020704710B504462068F6F776FAA6
S31508013410204610BD002202F07BBB000001B58B07D8
S315080134201AD1830724D1121F21D351F8043BA3F1E2
S31508013430013C2CEA030C1CF0803C04BF40F8043B19
S31508013440F1E79CFA8CFCBCFA8CF1C1F118018B40AE
S31508013450CB4040F8043B13E0042A09D311F8013B99
S31508013460521E00F8013B5BB18B07F7D1D9E7121D54
S315080134705AB111F8013B521E00F8013B03B1F8D1CC
S3150801348011001CBF002202F043FB01BD704702F088
S315080134906EBB0000B0FBF1F201FB1200401E804139
S315080134A0C00F7047704770477CB504460025AE4E7D
S315080134B0304602F05DFBF6F703FA0DF1010002F062
S315080134C059FB684602F057FB204602F069FB0028C3
S315080134D001D04FF0FF35684602F04AFC0DF10100B4
S315080134E002F047FC204600F041F9FDF73DFD60601A
S315080134F0002801D14FF0FF35304602F039FBF6F7C7
S31508013500FDF9284676BD7CB504460025964E30461B
S3150801351002F02EFBF6F7D4F90DF1010002F02AFBB1
S31508013520684602F028FB204602F03CFB002801D041
S315080135304FF0FF35684602F01BFC0DF1010002F061
S3150801354018FC6068FDF720FD304602F011FBF6F71E
S31508013550D5F9284676BD2DE9FC4F83B005460C46BC
S31508013560164600F003F90290284602F0F0FB804661
S31508013570284602F0E9FB8146274602993046FFF7BD
S3150801358089FF002806D0002C04D0C8440498801965
S31508013590804502D24FF0FF3083E00024DFF8C8816E
S315080135A0404602F0E5FAF6F78BF92AE04FF0FF34C8
S315080135B00DF1050002F0DCFB01A802F0DAFB09F1C6
S315080135C00109B9F1100F15D201A802F0D3FA0DF1CC
S315080135D0050002F0D0FA53465A463146284602F00B
S315080135E027FB0400E2D10DF1050002F0C1FB01A899
S315080135F002F0BFFB04990098091A049100988619EC
S3150801360007440498002846D0002C44D13146284660
S3150801361002F071FBB9088900B94202D04FF00109DD
S3150801362001E04FF00009811BB6FBF0F200FB021026
S31508013630019004A901A802F09DFB00680090B9F168
S31508013640000F02D1029988421AD202A9684602F0ED
S3150801365091FB00680090024639466868F2F7BAFE9F
S3150801366000980299884206D2FF22091A6868009BC7
S31508013670184402F049FAD5F804B0DDF808A007E0C5
S31508013680B0FBF1F1029841430091BB46DDF800A079
S315080136904FF0000995E7404602F06AFAF6F72EF967
S315080136A0204605B0BDE8F08F2DE9F84306460F46DA
S315080136B0154602F04CFB0446304602F045FB20183D
S315080136C0EC19A0420BD384420CD22146304602F0B3
S315080136D012FB01462046FFF7DDFE002802D14FF016
S315080136E0FF303DE00024DFF88080404602F040FAD2
S315080136F0F6F7E6F827E04FF0FF340DF1010002F086
S3150801370037FB684602F035FB09F10109B9F1100FDB
S3150801371013D2684602F02EFA0DF1010002F02BFAD7
S315080137203946304602F040FA0400E4D10DF10100B1
S3150801373002F01EFB684602F01CFB3946304602F0D1
S31508013740DAFA2D1AC719002D04D0002C02D14FF030
S315080137500009DBE7404602F00BFAF6F7CFF82046F8
S31508013760BDE8F28300000000C03D002002F0EABA7D
S315080137704FF0FF31016070470268054B514001F077
S31508013780FF0153F8211081EA1221016070470000F8
S31508013790408B010802684FF0FF314A4002607047CA
S315080137A00268002902D0806802607047C06802601A
S315080137B0704770B504460D46164600F09AFE4FF05E
S315080137C0FF30854209D00021204600F0CDFE314662
S315080137D02046BDE8704000F0C3BE70BDF8B504468A
S315080137E00D4616461F4600F084FE4FF0FF3085420F
S315080137F00DD039462046FFF7D3FF0121204600F0B8
S31508013800B3FE31462046BDE8F44000F0A9BEF1BD3D
S315080138100022CEE7002213460022DFE770B50446F0
S315080138200D4610461A46049E00280BD12046FFF77E
S31508013830C0FF4FF0FF30854209D031462046BDE82A
S315080138407040ADE733462046BDE87040C6E770BD17
S31508013850EFF30580401E8041C043C00F7047EFF368
S315080138601080002806D1EFF31180401E8041C04325
S31508013870C00F7047012070470246D2E84F0FC2E8D1
S31508013880431F03B1F9E7C0B270470000014651E88A
S31508013890000F421C41E8002303B1F8E77047000016
S315080138A0014651E8000F10B9BFF32F8F04E0421EFD
S315080138B041E8002303B1F4E7704770477047DFF822
S315080138C0B0064069704730B4026B002A16D000234F
S315080138D0CD7801E013465268002A02D0D478AC426A
S315080138E0F8D34A608B60002A01D0916000E0C1627A
S315080138F0002B01D0596006E0016304E000224A600A
S315080139008A60C1620163283030BCBFE710B504463E
S3150801391004F12800FFF7C4FF00280AD0E46A002C46
S3150801392008D00121A01CFFF7A7FF002802D0A46830
S31508013930F5E70024204610BD8B684A68002A01D0A5
S31508013940936000E0C3624A688968002901D04A6029
S3150801395070470263704770B50446A078002833D0D3
S31508013960E56821462846FFF7E7FF00202070214633
S3150801397005F10C00FEF75EF8A868002852D005F19B
S315080139800C00FEF747F804004CD02846FFF796FFCF
S31508013990FDF794FB064600221146FDF7DBFC30468F
S315080139A0FDF779FC06466A6AB16804F10C00F2F77C
S315080139B011FDF92020700020A070F068E070214602
S315080139C02846BDE870407EE7A568A868002824D087
S315080139D04078832821D12846FFF770FFFDF76EFB53
S315080139E0064600221146FDF7B5FC3046FDF753FCA5
S315080139F006466A6A04F10C01B068F2F7EBFCF06856
S31508013A00002801D0E178017000202070214605F1D7
S31508013A100C00BDE87040FEF70DB821462846BDE802
S31508013A20704050E770BD2DE9F84F060008D00F0029
S31508013A3006D0B6FA86F1B7FA87F04118202906D2D8
S31508013A406FF00301002002F09BF9002097E007F1CF
S31508013A5003084FEA98084FEA880808F10C0808FB9A
S31508013A6006F00090002A28D0D2F8009094681569CB
S31508013A705169002C0ED014F003000ED1D0683428F9
S31508013A800BD3002D10D015F003000FD100988142F9
S31508013A9017D20BE0D0680028F3D06FF00801002098
S31508013AA002F06EF900206AE000290AD06FF00901D8
S31508013AB0002002F065F9002061E04FF000094C464C
S31508013AC02546002C13D1DFF8A834D3F8A000002826
S31508013AD003D0FDF79FFF044606E001223421D3F8FF
S31508013AE08000FFF7A0F904464FF0010A01E04FF004
S31508013AF0000A002C22D0002D20D1DFF874B4002250
S31508013B000099DBF87C00FFF78EF9050010D15046C5
S31508013B10C0070BD5DBF8A0000028214602D0FDF727
S31508013B2089FF03E0DBF88000FFF7DAF9002403E0F8
S31508013B300022009901F0E8FF4AF0020A002C18D089
S31508013B40FA20207084F802A0C4F804900020A0602E
S31508013B506762A062E06220632B464246314604F161
S31508013B600C00FDF737FFDFF80C04DFF804140867CB
S31508013B7004E06FF00401002002F002F92046BDE8D6
S31508013B80F28F2DE9F0410C4690461D46FFF795FE4A
S31508013B90060004D03078FA2801D1002C07D16FF03D
S31508013BA003042146304602F0EBF8204652E0B0689D
S31508013BB000281CD04078832819D13046FFF77EFEAD
S31508013BC0FDF77CFA054601220021FDF7C3FB2846CD
S31508013BD0FDF761FB0546726A2146A868F2F7FAFB0A
S31508013BE0E868002801D080F80080002032E006F15C
S31508013BF00C00FDF70FFF070011D0726A214607F185
S31508013C000C00F2F7E7FBF92038700020B87087F846
S31508013C10038039463046FFF756FE00201AE0002D8C
S31508013C2016D029469320FDF7A8FB00280DD0FFF7EB
S31508013C3046FE05463046FFF741FE2946FDF727FAB7
S31508013C40EFF309808460C0F80C806FF0010001E091
S31508013C506FF00200BDE8F0812DE9F0410C461546EA
S31508013C601E46FFF72AFE070004D03878FA2801D144
S31508013C70002C07D16FF003042146384602F080F87C
S31508013C80204660E03846FFF741FE8046B8F1000F4E
S31508013C903FD041463846FFF74FFE7A6A08F10C01D4
S31508013CA02046F2F797FB002D02D098F803002870FA
S31508013CB0002088F80000414607F10C00FDF7BAFE1E
S31508013CC0B868002823D007F10C00FDF7A3FE04000D
S31508013CD01DD03846FFF7F2FDFDF7F0F9054601223A
S31508013CE00021FDF737FB2846FDF7D5FA05467A6A1E
S31508013CF0A96804F10C00F2F76DFBF9202070002089
S31508013D00A070E868E07021463846FFF7DCFD002020
S31508013D1019E0002E15D031468320FDF72EFB002829
S31508013D200CD0FFF7CCFD06463846FFF7C7FD3146EE
S31508013D30FDF7ADF9EFF309808460C5606FF0010006
S31508013D4001E06FF00200BDE8F08138B5FFF7B5FD77
S31508013D50040002D02078FA2807D06FF00305294617
S31508013D60204602F00DF8284632BDA06800280FD07B
S31508013D702046FFF7A3FDFDF7A1F900226FF0020126
S31508013D80FDF7E8FAA0680028F2D10020FDF7ADFAA0
S31508013D9000202070A078800704D5A1697448C06FF7
S31508013DA0FFF79EF8A078C0070CD5714AD2F8A00093
S31508013DB00028214602D0FDF73DFE03E0D2F8800037
S31508013DC0FFF78EF8002032BDF8B50C4617461D469A
S31508013DD0FFF773FD060006D03078FA2803D1002CC8
S31508013DE001D0002D07D06FF003042146304601F0BB
S31508013DF0C7FF2046F2BD06F10C00FDF70BFE0500D4
S31508013E0013D0726A214605F10C00F2F7E3FAF9209C
S31508013E1028700020A870EF706C60AE602846FFF726
S31508013E204DFDFFF76CF90020F2BD6FF00200F2BDFF
S31508013E30F8B50E4615461C46FFF73FFD070006D0A6
S31508013E403878FA2803D1002E01D0002C07D06FF05C
S31508013E5003042146384601F093FF2046F2BD384651
S31508013E60FFF754FD040011D07A6A04F10C013046BB
S31508013E70F2F7B0FA002D01D0E0782870E760204605
S31508013E80FFF71CFDFFF73BF90020F2BD6FF00200BA
S31508013E90F2BD000070B504460D461646FFF7D8FC7C
S31508013EA0002803D1FFF7DBFC002806D06FF00501D7
S31508013EB0002001F065FF002070BD2F488446324678
S31508013EC02946204600DF70BDF8B504460D4616465C
S31508013ED01F46FFF7BDFC002803D1FFF7C0FC0028E9
S31508013EE007D03B4632462946204601B0BDE8F04098
S31508013EF06AE7224884463B4632462946204600DF81
S31508013F00F2BD0000F8B504460D4616461F46FFF7F2
S31508013F109FFC002803D1FFF7A2FC002807D03B46E7
S31508013F2032462946204601B0BDE8F04080E71448EC
S31508013F3084463B4632462946204600DFF2BD00004C
S31508013F4038B50446FFF784FC002803D1FFF787FC40
S31508013F50002806D06FF005052946204601F010FF16
S31508013F6004E008488446204600DF0546284632BD57
S31508013F70241A002057390108273A0108833B01080A
S31508013F80593C01084B3D010801F0FBBE10B504463A
S31508013F90F2F7AAFE0121204600F0E6FABDE8104034
S31508013FA0F2F7B3BE10B50446F2F79EFE002120468D
S31508013FB000F0DAFABDE81040F2F7A7BE00F10103F6
S31508013FC0810704D010F8011B820781B1FAD1026872
S31508013FD0A2F10131914311F0803104BF50F8042F49
S31508013FE0F6E709BAB1FA81F100EBD100401CC01A13
S31508013FF0704700007CB5044642F21170844207DB23
S31508014000002000900346024608490948FEF7B7F919
S31508014010F6F77EFA0546F6F7C9FC06462846F6F788
S31508014020C5FC801BA042F9D373BD00001CC701085B
S315080140300001018001F0A6BE7CB504460D46DFF8F5
S31508014040386331462846FEF76DFC206010F1010FF2
S3150801405006D12E22DFF824130FF24830F5F746FB76
S3150801406031462846FEF788FC10F1010F06D13222A7
S31508014070DFF808130FF24430F5F738FB0146090B50
S3150801408001F01F012175400C00F0010060752068E0
S31508014090DFF8EC12884209D1BA48016841F4006197
S315080140A00160006800F40060009000982068B0F193
S315080140B0804F09D1B348416841F001014160406828
S315080140C000F00100009000982068AF49884209D1A4
S315080140D0AC48416841F002014160406800F00200C5
S315080140E0009000982068A949884209D1A5484168E5
S315080140F041F004014160406800F004000090009816
S3150801410031462846FEF7C4FBA5800020E060206101
S315080141100120A06044F620612046BDE87C4075E098
S315080141200021B0F90400FEF787BD0000F0B587B09D
S3150801413006460F460024964D3068286038462146C3
S3150801414001F02AFE01D20F4605E09249FAF772F903
S3150801415001D84FF07E57F068FFF748F9394601F064
S315080141602FFE01F099FE22468B4B00F0AFFB00F0C3
S3150801417001FE3061602000903069B168B0FBF1F052
S315080141800190204602900490059003900690307D98
S31508014190401E03281ED8DFE800F003020F1104248D
S315080141A022466946284601F04BFA002808D000BF86
S315080141B089A0FEF743FB0DE00824F1E70C24EFE79D
S315080141C0707D00282146284602D001F089FE01E0CB
S315080141D001F01DFA07B0F0BD38B50022C468002CFD
S315080141E00BD00069FFF702F905462046FFF7FEF8EE
S315080141F001462846F6F710FC024610466549FAF7C5
S3150801420019F901D84FF07E52104632BD2DE9F8430F
S3150801421086B004460F46D4F800905D4DC5F8009067
S31508014220002000902046FFF7D7FF06464FF000080A
S31508014230D9F8200041F2111108420BD1D9F8200012
S3150801424040F24441084205D1D9F80000400840002F
S31508014250C9F80000694601A8F2F7DCFF4F4A01E0F8
S3150801426008F101084146C9B252F83100236898425B
S31508014270F6D1002804D100BF5DA0FEF7DFFA65E09C
S31508014280101D10F83100002804D1F2F7ADFF009097
S31508014290049803E0F2F7B3FF009005980121A160A5
S315080142A00028009905D13E4AB1FBF2F1491E696021
S315080142B005E049003A4AB1FBF2F1491E69607A1EE6
S315080142C0EA604FF6FF71EB688B4202D86B688B4246
S315080142D026D9A3685B00A3600028DDF800C008D1D1
S315080142E0DFF8BCE0BCFBFEFC03FB0CF35B1E6B605A
S315080142F009E04FEA4C0CDFF8A8E0BCFBFEFC03FB27
S315080143000CF35B1E6B60A368B2FBF3F3EB608B42A5
S31508014310D9D26B688B42D6D92FA0FEF78FFA15E052
S3150801432000202861A860284601F058F9002803D022
S3150801433029A0FEF783FA09E0E76031462046FFF730
S31508014340F5FE2868016841F00101016007B0BDE882
S31508014350F08338B504460846FFF736F80546E0689F
S31508014360FFF744F801462846F6F756FB014620466C
S31508014370BDE83440DAE6000018A00108B8C1010812
S31508014380002C0140181002400004004000080040BB
S31508014390503D00200100803F0000E03F48CA010867
S315080143A040420F006F626A2D3E70776D20213D20D5
S315080143B02850574D4E616D65294E430066756E63EB
S315080143C074696F6E20213D202875696E7433325FDA
S315080143D074294E430000000043616E6E6F742069B4
S315080143E06E697469616C697A652050574D0A0000D7
S315080143F0556E6B6E6F776E2050574D20696E7374CC
S31508014400616E63650000000001F089BDF3F784BDA4
S3150801441010B400EB116091FAA1F1B1FA81F18900AA
S3150801442003680F248C40A3438A401A43026010BCD8
S31508014430704700001CB50024042840D8DFE800F0C6
S31508014440030F1B2733003D4C3D48016841F0040129
S315080144500160006800F004000090009832E0394CD1
S315080144603748016841F008010160006800F008005A
S315080144700090009826E0344C3148016841F010015B
S315080144800160006800F01000009000981AE02F4CB7
S315080144902B48016841F020010160006800F0200006
S315080144A0009000980EE02A4C2548016841F0400129
S315080144B00160006800F040000090009802E025487D
S315080144C0FEF7BCF9204616BD10B504464FF0FF317C
S315080144D0884204D17622204929A0F5F707F9002157
S315080144E0FEF7AAFB012004F00F0400FA04F42046A3
S315080144F010BD70B504460D46258228464FF0FF319A
S31508014500884219D0C0F30310FFF794FF06462846E0
S31508014510FFF7DAFF206066611048217C01F00F0180
S3150801452050F82100A06106F10800606006F110004C
S31508014530A06006F11400E06070BD000000080140AB
S3150801454018100240000C01400010014000140140FF
S3150801455000180140BCCA010810C10108CCB80108FD
S31508014560B0F91000FEF7CEBB43698069002903D173
S315080145700822014618464BE701220146184647E735
S3150801458070696E20213D202850696E4E616D65293E
S315080145904E43000010B50446207E002803D1F5F7E6
S315080145A068FD0120207610BDF3F7B6BCC9B20278C2
S315080145B08A421AB11CBF10F8012FF9E718BF00206B
S315080145C07047000080B500B906A005490B681BB104
S315080145D022220021984701E001F0A2FC222002BD17
S315080145E0F03F0020636F6E73747261696E742068A0
S315080145F0616E646C65723A20626164206D657373DD
S3150801460061676500C9B2830706D0521E22D310F826
S31508014610013B9942F7D11FE0083A13D302F104028C
S3150801462041EA012141EA014150F8043B121F21BF29
S315080146304B40A3F1013C2CEA030C1CF0803FF3D05C
S31508014640C9B2001F083210F8013B521E28BF91EA71
S31508014650030FF8D818BF0120401E704710B514463D
S3150801466000F002F8226010BDC1F30A5343B14A00B3
S3150801467012F5001F28D2A3F2FE32A1EB02517047B0
S3150801468050EA410C20D001F0004C31EA0C01B1FA94
S3150801469081F204BFB0FA80F3D2180B3AB2F12003C3
S315080146A02CBF00FA03F1914041EA0C013EBFC2F169
S315080146B0200C20FA0CF319439040524240F2FD3384
S315080146C0D21A01EB035170470022704741EA030CE5
S315080146D050EA4C0C52EA0C0C4FF4001C09D307D0D3
S315080146E01CEB410F9CBF1CEB430F8B4208BF824258
S315080146F070471CEB430FFBD8994208BF904270479D
S3150801470041EA030C50EA4C0C52EA0C0C4FF4001C1B
S3150801471009D307D01CEB410F9CBF1CEB430F9942F1
S3150801472008BF904270471CEB410FFBD88B4208BF6C
S3150801473082427047124254D440F2FF7C1CEA11535C
S315080147400FD0634531D09B1863453CBF01EB02513D
S31508014750704701F0004141EA0C51002000F07BBD91
S31508014760704750EA410320D001F0004C91EA0C0150
S315080147701CD0B1FA81F30B3B9A420DD9D21A994052
S3150801478051EA0C01C3F1200C20FA0CFC6144984053
S31508014790531C40F2FF7CD7E7914041EA0C01C2F174
S315080147A0200C20FA0CF3194390407047B0FA80F3B5
S315080147B01533202BE0D3202AEED3203A203B9A4208
S315080147C009D9D21A00FA03F141EA0C010020531C57
S315080147D040F2FF7CB8E700FA02F141EA0C01002039
S315080147E07047524240F2FF7C1CEA11530DD06345D3
S315080147F0DBD0B2EB030C3CBFA1EB025170470CF1C5
S31508014800010221EA035141F4801150EA410CCCD04E
S3150801481001F0004C352A27DC30B481EA0C01B2F1EB
S31508014820200309DAC2F12003044601FA03F5D04050
S315080148302843D1409C400CE0C3F12002450020FAF0
S3150801484003F418BF44F0010421FA03F091400C4324
S31508014850002174F1004550F1000051EB0C0124428E
S3150801486030BC7FF47BAF70476146002076E70000D5
S31508014870C1F30A5340F21E42D31A0CDDCA0283F36E
S31508014880070342EA505242F00042DA4002EBE17273
S3150801489082EAE17070476FEAE17203F2E13008B12A
S315080148A082F000407047000010F0004160B148BF37
S315080148B04042B0FA80F29040D21CC2F5846241EAC5
S315080148C0025202EBD02140057047000070B491EA0C
S315080148D0030F4FF0004540F1BF806B40841A71EB1E
S315080148E0030604D26E40001BB141121973414FF4FD
S315080148F0001C1CEB410F34BF7CEB430683E00C0D17
S31508014900A4EB1356362E00F37C80012E45EAC32309
S3150801491041DC43EA525312BFD20292025B082405D4
S3150801492045EAC12141EA5051D2EBC020994125D42B
S3150801493007D1B0FA80F610FA06F162D000202036C7
S3150801494008E0B1FA81F6B140C6F1200220FA02F276
S315080149501143B0404FEAF474B4EB465434F00106FF
S315080149604FEA74040AD8D6F50016760D04F0004409
S31508014970F04061FA06F25040F1404840C00A40EA68
S31508014980415021F0004128BF5FEA500550F100006F
S3150801499044EBD12135E0DB0A45EAC121C90AB6F162
S315080149A020050EDD42EA0242120CC5F1200603FA81
S315080149B006F6EB4042EA06056D42984161F10001AF
S315080149C00DE062FA06F5F240554063FA06FC82EA02
S315080149D00C02F3405A406D42904161EB030111F418
